:020000040800F2
:10000000902C0020A90D010885960108859601080D
:100010008596010885960108859601088596010850
:100020008596010885960108859601088596010840
:100030008596010885960108859601088596010830
:100040008596010885960108859601088596010820
:100050008596010885960108859601088596010810
:100060008596010885960108859601088596010800
:1000700085960108859601088596010885960108F0
:1000800085960108859601088596010885960108E0
:1000900085960108859601088596010885960108D0
:1000A00085960108859601088596010885960108C0
:1000B00085960108859601088596010885960108B0
:1000C00085960108859601088596010885960108A0
:1000D0008596010885960108859601088596010890
:1000E0008596010885960108859601088596010880
:1000F0008596010885960108859601088596010870
:10010000859601088596010885960108859601085F
:10011000859601088596010885960108859601084F
:10012000859601088596010885960108859601083F
:10013000859601088596010885960108859601082F
:10014000859601088596010885960108859601081F
:10015000859601088596010885960108859601080F
:1001600085960108859601088596010885960108FF
:1001700085960108859601088596010885960108EF
:1001800085960108859601088596010885960108DF
:1001900085960108859601088596010808B5034CE7
:1001A00000F0ACF8204610F05CFCF9E788D90108B3
:1001B000004870474CFA010810EE103AC3F3C752DA
:1001C00022B95B0014BF032002207047FF2A04D12C
:1001D0005B020CBF0120002070470420704710EE26
:1001E000103AC3F3C752952A18DCDFED0D7ADB0F06
:1001F00015BF30EE670A30EE270A30EE270A30EEE0
:10020000670AB5EE400AF1EE10FA07D1DFED057A84
:100210009FED050A002B08BFB0EE670A704700BFCC
:100220000000004B000000000000008053EC102B89
:10023000C3F30A5131B992185B41134314BF032031
:100240000220704740F2FF70814206D11B0353EA3F
:1002500032530CBF0120002070470420704770B556
:100260008EB0054602A80E4600F070F80446D0B9DC
:10027000284610F001FD234602462946352000F0AD
:1002800078FF056801463246684601F0E4FA01232A
:1002900022462946684603F069FD05F0F3FA00F0AE
:1002A00071F80EB070BD0399014806F0ABF9F8E79C
:1002B00030DA010830B58FB0054602A800F046F8E4
:1002C0000446A0B9284600F062FF056801460122F5
:1002D000684601F0C0FA012322462946684603F029
:1002E00045FD05F0CFFA00F04DF80FB030BD039991
:1002F000014806F087F9F8E730DA010808B505F09B
:1003000051F801210348FFF7AAFF05F067F8002024
:1003100008BD00BFACD901080020704708B50446ED
:1003200010F050F8224602494C3010F02DFAFEE74A
:10033000CFD90108FEE710B51C4602460B4602481D
:10034000214610F07CFBFEE7E3D90108C46005619B
:1003500046618761C0F81C80C0F82090C0F824A0D6
:10036000C0F828B0C0F82CD0C0F808E000F001B800
:100370000020034B9A68026098600020704700BF1D
:100380003C210020024B9A6812689A60704700BFB7
:100390003C2100200D4A93680BB9FFF7BFFF196895
:1003A000586091601846C468056946698769D0F845
:1003B0001C80D0F82090D0F824A0D0F828B0D0F835
:1003C0002CD0D0F808E001207047FEE73C21002047
:1003D000014810F034BB00BF9DEB010870B5054625
:1003E00008460E4610F048FC044620B102466B68F1
:1003F000286831469847204670BD2DE9F74F019196
:100400009DF8301091460D9A11F0DF0F0646A2EBD1
:1004100009023DD030290CA9244F0EBF4FF010081F
:100420000F464FF0010813F0800435D0022492FBF0
:10043000F4F4151B002C36DDA246D045C346A8BFF8
:10044000D346736830685A463946AAEB0B0A984778
:10045000BAF1000FF1DCB9F1000F05D07368019912
:1004600030684A4698474C44002D0DDD2C44A84581
:10047000C146A8BFA946736830684A463946A5EB0D
:1004800009059847002DF2DC204603B0BDE8F08F47
:10049000074F4FF01008C6E713F0010501D11446CD
:1004A000C8E71546D7E70024D5E700BF1DDA0108E5
:1004B0000CDA01082DE9F04389B00746119D9DF83B
:1004C0004880139E42BB00228DF80F2051BB08AC20
:1004D000302304F8013D15F040099DF80F303FD05E
:1004E000002B46D001220192CDF800802B460DF161
:1004F0000F013846FFF781FF013E814608AA0196A9
:10050000CDF800802B46121B21463846FFF775FFB9
:10051000484409B0BDE8F083002919DA2D228DF88E
:100520000F204942109A08ACA2F10A0E0DF1100CEE
:10053000B1FBF3F003FB1012092ACCBF7244303236
:1005400004F8012D64450146C5D00028F0D1C2E76A
:10055000A80701D52B22B7E76A07B4D52022B3E755
:10056000002BCBD004AA9442C8D904F8013C013C2A
:10057000C4E79946C2E72DE9F04F91B011F0010FA1
:100580008246884691461A9D9DF86CB01C9F1D9E20
:100590000ED111F0030F03D10A6883498A4207D0B4
:1005A0004046059306F0E8F8059B400040F001083E
:1005B00015F0810206D1BBF1300F03D1B742B8BFAD
:1005C000374616464046059308F087F9002808A9E3
:1005D000059B17DBAC0711D52B228DF820200DF1E0
:1005E0002104EA061DD5B9F1020F0DD122463020B3
:1005F00002F8020B581C6070144612E0680701D51F
:100600002022EAE70C46ECE7B9F1080F3ED1A80535
:100610004FF03002227045BF03F10E0262700134C8
:100620000234611A002215F0200F05910CBF11460B
:100630002C21012E0CA8C8BF45F04005227009905E
:10064000DBB2102015F040040A900B928DF81F20A9
:100650000391029324D00192CDF8009043460BAA57
:100660000AA909A807F0EAFF03782D2B814671D16A
:100670000B9C8DF81F30013C012E00F101090B94F9
:1006800000F38D804FF00008444617E0B9F1100FD9
:10069000C7D12246302002F8020B03F11700AAE767
:1006A00008AB0193CDF8009043460BAA0AA909A80C
:1006B00007F0C4FF012E814647DCA04669061BD522
:1006C0009DF81F3053B101220023019200930DF1D8
:1006D0001F015046FFF791FE013F0444059B5BB1AB
:1006E0000123019300230093059A08A95046FFF7C0
:1006F00084FE059B0444FF1A012EC8BF37460197AC
:10070000CDF800B02B460B9A49465046FFF775FED0
:100710000444B8F1000F0AD0202300930023CDF841
:1007200004801A4621495046FFF767FE04440998A1
:100730000CAB984201D00DF0A7FD204611B0BDE8EA
:10074000F08F4FF00008444619E00B9CB442B8BF4C
:1007500034460BE0012E95DD0B9C9DF81F30B44212
:10076000B8BF344603B10134059B1C44A742E8DD01
:1007700015F00108A7EB040401D0A046002425F0E1
:1007800001054CB120230093002301941A46074928
:100790005046FFF732FE04464FF0300B8EE7B4426E
:1007A000B8BF3446DFE700BF74F7010872110208D2
:1007B0002DE9F04316468BB0B20780469946129F4A
:1007C0003DD416F0040F0CBF0023202300930A46EB
:1007D000139B202102A804F0C9F9F30504460DD5A6
:1007E000431C1F2B0AD80AAA1444252204F8202CE3
:1007F0000AAA1A44002102F8201C1C4616F04005E3
:100800001FD09DF808302F2B4FF000031BD801227A
:1008100002A9019200934046FFF7EFFD013F054614
:10082000013C0DF109010197CDF8009033462246B5
:100830004046FFF7E2FD28440BB0BDE8F0832B23D0
:10084000C4E702A9EFE702A91D46ECE72DE9F04F46
:10085000814689B0144600250E46334613F8012B15
:10086000CAB9B14208D2771AD9F80430D9F80000D1
:100870003A4698473D4431460B78002B00F01081F2
:10088000013120234FF000080E780F464A1C36B97C
:100890004FF0FF3245E0252AE3D01E46DDE72D2E3E
:1008A00003D148F001081146EEE72B2E02D148F0A3
:1008B0000208F8E7202E02D148F00408F3E7212EC1
:1008C00002D148F00808EEE7302E1DD000264FF088
:1008D0000A0E0F4611F8012BA2F13000092817D992
:1008E0002E2AD5D17A782A2A16D000224FF00A0C67
:1008F0000F4611F8010BA0F1300EBEF1090F10D810
:100900000CFB0202303AF3E748F040083346CAE7EE
:100910000EFB0626303EDCE72268023722EAE2724E
:10092000043439786C2908BF013797F800A0BAF170
:10093000000F00F0B580BAF1640F00F08B8023D86F
:10094000BAF1500F2AD00ED8AAF14501022940F27F
:100950009080D9F80430D9F8000001223946984730
:100960000135A34648E0BAF1620F38D04AD8BAF14F
:10097000580FEED1029304F1040B0396CDF80480D6
:1009800041230093102363E0BAF1710F45D00DD8D5
:10099000BAF1670F6DD9BAF1700FDAD1029304F191
:1009A000040B0396CDF804806123EAE7BAF1750FD2
:1009B00045D0BAF1780FF1D0BAF1730FC9D1511CFB
:1009C00004F1040B246805D12046049310F054F977
:1009D000049B02468DE848002146434608E0226811
:1009E00004F1040B8DE84800434642B12E4904222D
:1009F0004846FFF702FD0544791C5C462CE70522BA
:100A00002A49F5E708A9226801F8042D04F1040B2E
:100A10008DE8480001224346EAE707A920680592CD
:100A200004930DF051FD059A049B0146501C8DE87E
:100A3000480004F1040B08BF079A4346D8E7029325
:100A40006123009304F1040B0396CDF804800A237C
:100A5000002209E002936123009304F1040B039642
:100A6000CDF804800A23012221684846FFF722FDC1
:100A7000C1E7073424F00704D4E900010592049388
:100A80001CF05AFD059A019200EE100A0096049B94
:100A900042465146484604F1080BFFF789FEAAE793
:100AA000284609B0BDE8F08F38DA01083DDA0108C0
:100AB0000EB403B503AA52F8041B0192FFF7C6FE59
:100AC00002B05DF804EB03B0704700BF0369272B49
:100AD0001DD0222B1BD0752B03D023F01002622ACD
:100AE00004D14269272A12D0222A10D0722B10D1A9
:100AF0004369622B0FD18069272808D0A0F1220317
:100B000058425841C0B270474369722BF2E7012046
:100B1000F8E7622BF8D00020F4E703690A2B10B540
:100B2000044622D1C3690133C3610123236263698F
:100B30002361A36963616068A36898476369A061E2
:100B40000D2B07D10A239842636103D1A368606823
:100B50009847A061A369013306D163695A1C03D089
:100B60000A2B1CBF0A23A36110BD092B036A04BF13
:100B7000073323F007030133D8E770B504460E4668
:100B800000252069431C01D1284670BD0A2808D1E0
:100B900016B1A36A002BF7D02046FFF7BEFF012550
:100BA000EFE70DF008FE18B12046FFF7B6FFE8E7C3
:100BB0002369232B08D12046FFF7AFFF23695A1C76
:100BC000DFD00A2BF7D1DCE75C2BDDD163690A2B80
:100BD000DAD12046FFF7A1FFE6E72DE9F74F0446FB
:100BE00000218164FFF7C9FFE369A363636A256A93
:100BF000E563002B04DA062284F84020013304E088
:100C000007D0052284F84020013B636203B0BDE8B1
:100C1000F08F002832D0A36A83BB0423226B84F8B0
:100C200040306FF00043606BD118013D30F8111077
:100C30008D42EBD017D9E16A8A4207D308314900C7
:100C40000DF013FBE36A60630833E362236B626BAE
:100C5000591C216322F81350636ACFE7013A2263DB
:100C6000626A013A6262226BD11830F811108D422B
:100C7000F4D3CBD0022384F84030C7E72169481C65
:100C800001D10023F7E72046FFF720FF002800F0FE
:100C90000E81002384F840304FF001092369752B41
:100CA0005CD0622B51D16369722B0CBF02250125E8
:100CB0004FF00B030CBF0127002794F84020002AB7
:100CC00055D184F840303DB12046FFF726FF022D74
:100CD00002D12046FFF721FF23692046222B0CBFBB
:100CE0004FF0220A4FF0270AFFF717FF23695345F9
:100CF00040D163699A453DD12046FFF70EFF20465B
:100D0000FFF70BFF4FF00308002504F14406D4F869
:100D100010B0BBF1FF3F00F0C480B8F1010F03D168
:100D2000BBF10A0F00F0BD80454526D3294604F1EA
:100D300044000DF0F1FC01212046FFF71EFF204684
:100D4000FFF7C4FE0028A9D160E7722B0AD16369BE
:100D5000622B09D001250A230127AEE701250A23CA
:100D60000027AAE70025FAE702250B23F4E79342C0
:100D7000A9D04BE74FF00108C6E7DA4508D1514644
:100D8000304601350DF0ACFC2046FFF7C6FEBEE74D
:100D9000BBF15C0F40F082802046FFF7BEFE256964
:100DA00027B15C2130460DF09BFC5AE0622D00F02B
:100DB0008E812ED84E2D6ED01BD8222D3ED0272DC1
:100DC0003CD00A2D53D0A5F13003072BE9D84FF0C2
:100DD000030B1D466369303B072B42D8BBF1010B67
:100DE0003FD02046FFF799FE2369303B03EBC50552
:100DF000F0E75C2D22D0612D00F06F81552DE2D1FE
:100E000094F840300B2B22D15C2130460DF068FC69
:100E100014E0742D00F05D8107D86E2D0DD0722D79
:100E200013D0662DCFD10C2508E0762D0BD0E7D35B
:100E3000782DC8D14FF0020B0FE00A25E9B23046F9
:100E40000DF047FC13E00B25F8E70D25F6E7752DAF
:100E500014BF4FF0080B4FF0040B00251BF1FF3BB4
:100E600007D2691C03D0FF2DE8D984F840900025F3
:100E70008AE72046FFF751FE2369019318460DF0DB
:100E8000B9FC002800F01F81019B18460DF0F2FC10
:100E90002D010544E2E7924805F0E8F95FFA8BF18D
:100EA000CDE745453CBF032384F840303EE7084684
:100EB0000DF08CFC216918B95F2901D07F293DD93B
:100EC000072384F8403004F14405C9B228460DF0E8
:100ED00000FC2046FFF721FE2069421C1AD128465B
:100EE0000DF0E8FB7F4F0646002557F825103046E9
:100EF0000FF0B7FE00281BD10D35EDB2102D84F890
:100F000040507FF483AE784B5B6F002B14BF0D23F2
:100F10000F23B0E60DF05AFC40B920695F2805D0D8
:100F20007F2803D80DF05CFC0028D8D0217CCDE7C9
:100F3000FFF66CAE0135222DD7D167E608460DF0DD
:100F40004FFCA8B923692E2B0DD0684D00262F78B1
:100F500017B12369BB4263D12046FFF7DEFD002FA6
:100F600066D1012387E660690DF03AFC0028ECD0D9
:100F700021692E2904D1092384F84030002511E08D
:100F80000823302984F84030F8D1656945F0200500
:100F9000A5F16203162B9DBF554DDD4005F00105FF
:100FA0000025EDB204F1440630460DF099FB2046D1
:100FB000FFF7B3FD09272069431C3FF427AEC5B9ED
:100FC000652801D0452814D16521304684F8407049
:100FD0000DF086FB2046FFF7A0FD21692B2901D0EB
:100FE0002D29E8D130460DF07BFB2046FFF795FD1B
:100FF000E1E70DF0EBFB28B121692E290BD184F834
:101000004070EFE720690DF0EBFB0028F4D1236975
:101010002E2BF1D0FAE521F020034A2BE2D1EEE7A6
:10102000652F01D0632F00D10135013601358EE7E0
:10103000212F07D123693D2B93D12046FFF76DFD6A
:10104000412318E62E2F0DD123692E2B43D163693E
:101050002E2B40D12046FFF760FD2046FFF75DFDB7
:101060000C2308E60335324615F8027C632F11D0B5
:10107000652F0FD01B4B134493F8883084F8403011
:1010800003F0FB02422A01D0442B14D1A36A01339E
:10109000A362BBE515F8013C2169994206F10106FE
:1010A00007D12046FFF739FD3246652FE2D00235E1
:1010B000DAE7632FFAE7432A02D0452B7FF4A6AD87
:1010C000A36A013BE4E784F840900546B6E60825AC
:1010D000B4E60925B2E64A23CDE50725AEE600BF12
:1010E00037DB010844DA01083C210020F6DA010868
:1010F000012040007FB5064601AD542085E80E0072
:101100000DF096F80446034695E8070043F8046B93
:1011100083E807006FF001020025012322620A2202
:10112000E262E36123636562A56214200DF080F83A
:101130002021606304F144000DF047FA636B204600
:101140001D80A56165612561FFF7E7FC2046FFF77B
:10115000E4FC2046FFF7E1FC2046FFF73EFDE36B91
:10116000012B18BF0523204618BF84F8403004B077
:1011700070BD30B585B001AC054620460EF0C5FC0B
:1011800094E80E002846FFF7B5FF05B030BD30B536
:1011900085B001AC0146054620460EF0F5FC284618
:1011A0000DF054F994E80E00FFF7A4FF05B030BD30
:1011B00030B585B001AC054620460EF0BDFC94E884
:1011C0000E002846FFF796FF05B030BD10B5044667
:1011D00070B1C3684068984704F144000DF022FAEA
:1011E000606B0DF051F82046BDE810400DF04CB892
:1011F00010BD00BF03694269013B036152F823003F
:101200007047C1F17F5101F57F11036901F57F51ED
:101210003F311944436953F821007047F8B5446AD7
:1012200005460E46B4B194E809000B44834222D926
:1012300008310022014420460DF021F80246B8B9D9
:101240006168204608310DF01AF8636823602B6A44
:1012500063602C62102E374638BF102707F1080054
:101260000CF0E6FF0023076043600446686202E07A
:101270002368334423606068064466600834204471
:10128000F8BD38B50D460369C1688B42044608D3E2
:101290001031890040690CF0E8FFE36860611033A9
:1012A000E36023696269591C216142F8235038BD0B
:1012B000F8B50D461F4690E80A008B4204461646D4
:1012C00008D31031C90080680CF0CFFF2168A060FE
:1012D000103121606168A0684B1C636050F83120B8
:1012E00065F3170240F8312000EBC1033278DA7061
:1012F0005F60F8BD10B4C1F30B018469034A002399
:1013000052F82120A16B5DF8044BD1E7D8DB01082E
:10131000F7B586690F4696F84010072905461FD194
:10132000B16CF06C0DF03AF83B78882B04460ED186
:101330008100002241F0020105F1280004F0E5FFE0
:1013400028B14468E3071FD544F0010002E0200102
:1013500040F002000146284603B0BDE8F04090E7A7
:10136000082907D133460022B16CF06C03F03AFE35
:101370000446E7E7092912D1009600230122B16C47
:10138000F06C03F0ABFE04460C212846B66BFFF769
:1013900045FF40F23513066043608460DAE7A1F14F
:1013A0000A03012B1CD8B16CF06C0A290BD80CF085
:1013B000F5FF96F8403048B10A2B0CBF06210A21F0
:1013C00041EA0010C6E70CF0B9FFF2E7064C074807
:1013D000B26CF16C0A2B08BF204608F0BDFAD2E7C8
:1013E000090141F00E00B5E724FB0108D0FA01081D
:1013F000DE2807D010F0010306D043080CBF0120FF
:10140000002070470120704718467047FE2807D01B
:1014100010F0010306D0430814BF012000207047DC
:10142000012070471846704710F0010204D040F0C8
:101430000100086001207047B0B110F0030310D123
:101440000279352A0FD183680B6013F0010006D1B1
:101450009A0704D11868054BC31A58425841C0B2C4
:101460007047104670471846704700BF74F7010870
:101470002DE9F04F92F80090B9F12A0F85B004469B
:10148000884617461D460AD10021FFF7BAFE30B143
:10149000810740F05E8103798A2B40F05A81A9F1DF
:1014A0001C03012B5AD82E46AA4666B1013E31468E
:1014B0002046FFF7A6FE23696269A3EB0A03834671
:1014C00042F8230076BB0AF1FF390026B14540D827
:1014D000A5EB0905012D00F03C813B78A3F1210229
:1014E000022A69D8691E2046FFF78BFE01A9FFF783
:1014F0009BFF002800F08D803B78212B49D0222BC8
:101500000CBF4FF016094FF01709AE1E002E43DA3C
:10151000002D40F06A81019EF30740F16B8146F097
:10152000010130E0B9F11C0F0BD1FFF76FFF00286C
:10153000C9D15846FFF75CFF0028B6D10AF1FF3A3F
:10154000B3E7FFF755FF0028BDD15846FFF75EFF10
:10155000F2E72046FFF74EFE0136B7E7B9F11E0F5E
:10156000BBD100212046FFF74CFE0646FFF740FFA7
:1015700068B93046FFF74AFF0028AED0DE25204686
:10158000FFF738FE29462046FFF77BFEE1E0FE2507
:10159000F5E74FF01509B8E731462046FFF731FE71
:1015A00002A9FFF741FFA0B3029A0199484604F04F
:1015B000CFFC013E0190A9E7A3F12402022A48D8FA
:1015C000691E2046FFF71DFE01A9FFF72DFF00B39E
:1015D000DFF858A2AE1E002E9ADD711E2046FFF7DE
:1015E00010FE02A9FFF720FF98B131462046FFF711
:1015F00008FEC0F30710504490F85D92B9F1FF0F58
:1016000007D0029807F069F9B9F1190F14D800282A
:1016100017DAAE1CB60031462046FFF7FFFDC0F8D2
:1016200000803B7843EA0523814643600644002D51
:1016300040F0EB804946A6E7B9F11C0F01D900281C
:10164000E7D0029A0199484604F082FC023E0190DC
:10165000C1E7272B1BD100212046FFF7D2FD01A9AE
:10166000FFF7E2FE0028D4D001212046FFF7C9FD94
:10167000C0F307102F2808D030280CBF012002200B
:10168000019904F071F8019042E70020F8E7052B7A
:1016900069D100212046FFF7B4FD06460028B8D0E6
:1016A00010F0030A03D10379513B012BB1D9012179
:1016B0002046FFF7A6FD00F00F03022BA9D1BAF1D7
:1016C000000FA6D13379292BA3D1B36803F00F0201
:1016D000022A9ED11B096F2B9BD1F368002B98D057
:1016E0009A0796D11A792D2A93D1D3F808B04FEAE8
:1016F000101902A95846FFF797FE68B946494748AE
:1017000006F05AF9A169326809680546534606F0A1
:1017100091F92846FEF73EFE4FEA8901012241F089
:10172000020104F1280004F0F0FD029B43604846EA
:101730000CF0C5FE03785F2B20460DD1FFF75AFD54
:101740002046FFF757FD0023354A19462046FFF78C
:101750008FFE05B0BDE8F08FFFF74CFD59462046DF
:10176000FFF78FFD55E7292B7FF453AF012120466A
:10177000FFF747FD002106462046FFF742FD06F031
:101780000F03022B7FF445AF00283FF442AF10F067
:1017900003027FF43EAF03792F2B7FF43AAF310978
:1017A0008900D0F808901F4841F0020104F0ADFD17
:1017B00000283FF42EAF02AA4FEA1911406803F047
:1017C00069FE029B002B3FF424AFD90707D49A0788
:1017D0007FF41FAF1968144A91427FF41AAF039A3D
:1017E000002A7FF416AF019392E62046FFF702FD30
:1017F000013D8DE60C212046FFF710FD40F2351328
:101800000146056043608660BDE62046FFF7F2FCB6
:10181000013D46F8040D0AE702E301085CEF010808
:1018200070DE010874DE010874F70108D8DB0108D6
:10183000036830B513B91360184630BD9C0702D059
:101840001060012030BD5C68E5B28D42F8D10833EC
:101850001360200A30BD2DE9F04F95B000244023DD
:1018600002904FF400700F460192079308940CF019
:10187000DFFC2023099080200A930B940CF0D8FC05
:1018800021460C9011A80D970F94109404F0F6FCCB
:10189000019B002B54D0022B0CBF38222246AC4CAB
:1018A000B96B54F82220DFF8B8A2002307A8FFF78D
:1018B000FFFC4FF000080494089C002C00F05281BB
:1018C000099B621E03EBC201049CC87853F83230B6
:1018D00054F820500892C3F317096B784C6803F052
:1018E0003002102A03F00F062CD0202A5ED0B8F167
:1018F000000F40F0FF8003F001020392039A2240A0
:1019000005EB4201B1F802B00BEA0A01B1F5805FC4
:1019100040F0138197F84010CBF30B0B594504F1BD
:10192000010440F0E7802AB9294607A80593FFF78C
:10193000EFFC059B05933846FFF74FF9059BDDE764
:101940003622ACE734B905EB4402A64208D84FF082
:101950000108B1E7B8F1000FF5D14FF00008ABE78F
:1019600032F8023F03EA0A01B1F5805F0DD197F822
:101970004010C3F30B03994216D107A82946FFF77D
:10198000C7FC3846FFF729F9E7E7631C9E4204D9F4
:101990002A46494607A8FFF78BFC05EB440407A835
:1019A0006188FFF7A7FCD8E70134CEE7B8F1000F54
:1019B0000AD035F814300AEA0303B3F5405F1FD1AB
:1019C000002107A8FFF75DFC05EB4408A6422BD8D1
:1019D000019B93B12B78052B0FD1002107A8FFF7AE
:1019E00010FC50B9012107A8FFF70BFC10F003040D
:1019F00037D000F00F00022837D1002422464EE0F5
:101A0000012CA4D997F84030052B40F0DA805149D9
:101A1000514805F0D1FF00230446BA6B396806F03F
:101A200009F82046FEF7B6FC38F8023F03EA0A023E
:101A3000B2F5805F13D197F84020DBB29A420AD109
:101A4000072A03D1294607A8FFF762FC3846FFF7AB
:101A5000C4F80134BAE7002C3FF479AFD2E7631C35
:101A600096E790B30379352BC8D107A8FFF7C2FBDF
:101A700007A8FFF7BFFB394A0023494607A8FFF72D
:101A8000F7FC6AE735F8163003EA0A01B1F5805F22
:101A900013D1DBB2072B01D101340132013E002EFC
:101AA000F0D1012A1AD16B785A0617D53146A642D1
:101AB00007A80CD1FFF7E5FB4FE7214607A8FFF782
:101AC000A0FB00B101320134E8E7044696E7FFF7D6
:101AD00091FB0136002818BF0146E8E795F901306F
:101AE000002B04DA002107A8FFF7CBFB01342346C3
:101AF0002A46C2E7022E15D1012C3FF428AF00225E
:101B0000DB0704F1FF3106D5AB880AEA0303B3F51E
:101B1000805F08BF6108012902D1002A3FF41DAF90
:101B20000B46E5E7012C3FF412AF14F00102E7D0B9
:101B3000032E7FF467AF0122E2E7494607A8631C42
:101B40002A46FFF7B5FB594607A8FFF7D3FBB3E6D4
:101B5000D8DB01081EE3010820EF010870DE010850
:101B600000F0FFFF11A804F0ABFB109850B14168E2
:101B7000224608310CF083FB109B5A681A600F9ABA
:101B80005A600F9397F84030002B7FF43BAF0B9BCC
:101B9000002B3FF437AF0C9B09981B680E930CF099
:101BA00073FB0C980CF070FB3846FFF70FFB0EAB85
:101BB00093E80300029B83E80300184615B0BDE8D4
:101BC000F08F022B01D1024922E70249024820E7A7
:101BD00030E3010864E301085CEF010810B54068D8
:101BE00000B910BD44680CF04FFB2046F8E700BF79
:101BF000838B426A0133918C9BB29942838338BFB5
:101C0000938470472DE9F04180461F46C1B111F021
:101C1000030510D14E68F3B293420CD1360A01F19C
:101C20000804B54201DBBDE8F08154F8041B4046CE
:101C3000B8470135F5E740463B46BDE8F041184757
:101C4000BDE8F081014B89689022DBE7D3370008BB
:101C5000014B89686522D5E73D3D000810B5044673
:101C60000846114622680DF0A5FF636A4360002311
:101C70008360236A13B9206210BD13469A68002A54
:101C8000FBD1986010BD8968806A090902F010BD17
:101C90004279012A0B4602D1406A02F09BB9426A9E
:101CA0000149806A02F0BFB904E701084279012ABC
:101CB0000B4602D1406A02F09EB9426A0149806A2D
:101CC00002F0B1B9F4E601084279012A0B4602D1CB
:101CD000406A02F090B9426A0149806A02F0A3B9F1
:101CE000E4E601088968806A02F0C6BC2DE9F74F76
:101CF000B3F1000AC2BF0B7E43F008030B76436AC0
:101D00000C461B78E283064691469BB10025A84607
:101D1000736A1A8D954216DBB8F1000F0AD0CDF820
:101D200000A04B4642462146B06A02F0AEFE03B028
:101D3000BDE8F08FB06A53464A46214603B0BDE87D
:101D4000F04F02F08BBEDB6A13F83520033A012A0C
:101D500003EBC50B03D80027238D9F4201DB013520
:101D6000D6E7E36A03EBC70213F83730042B0BD135
:101D7000DBF804105368994206D1BBF80220B06A20
:101D800002F0F1FA08F101080137E5E72DE9F04129
:101D90000446884611461A4600238779868AC58AF2
:101DA00083718382C3820D4BFFF72CFFA36893B925
:101DB000E18A39B1A38A2BB9A06A02F0FAFDA06AC0
:101DC00002F06EFCA38AE28A41462046FFF78EFFAE
:101DD000A771A682E582BDE8F08100BF0D2C000846
:101DE00070B54379012B05460C4606D1436A0A4675
:101DF0005B7E0221FFF732FF2061A268216928463D
:101E00004623BDE87040C1E770B513464279012A08
:101E100006460C4604D10A460721FFF71FFFA061C2
:101E2000A569E26830463E232946FFF7AFFF688A7E
:101E300070BD10B5436A5A7E0446FFF7E5FF0146C0
:101E40002046BDE8104031E7036823B919B18B077C
:101E500004BF0B680360704738B5836804460D46BD
:101E600053B91146054805F0A7FD2946A06004F1C5
:101E70000C00BDE83840E7E738BD00BF5CEF010863
:101E8000004AE9E76CE40108428B4FF6FF739A427F
:101E900010B5044602D1064AFFF7DEFFA28BE38BA2
:101EA000618BA06AD21ABDE8104002F0AFBC00BF3F
:101EB00089E40108028B4FF6FF739A4210B504467D
:101EC00002D1064AFFF7C8FFA28BE38B218BA06AE1
:101ED000D21ABDE8104002F099BC00BFA1E401088D
:101EE00073B50646406A047E0D46A10706D5234A0F
:101EF00029463046FFF7B0FF02B070BD05F00F0174
:101F0000022915D12909B3791BB1838B013383834E
:101F100002E0438B0133438301240029ECD00DF10F
:101F200007020DF089FE9DF807301BBB144ADFE75E
:101F30002979914202D1A9680909E4E7994212D1AD
:101F4000B379002BD3D10123B371A9680029D3D071
:101F500001F00F0344F001040476022B18BF8968D6
:101F600003240909D9E7A96844F0020404760909A1
:101F70000524D2E7022303704470BDE764E301083F
:101F8000B6E4010849234822AAE741234022A7E7F3
:101F900037B505460C4629B1CA0705D54910806AF0
:101FA00002F01AFB03B030BD8B072CD001F00F04F8
:101FB000062C4FEA111307D00A2C0AD0022C1BD191
:101FC0001946FFF765FEEDE71946806A02F04AFB05
:101FD000E8E74279042A04D01149806A02F04CFBF8
:101FE000E0E701A918460CF06FFA0199AC6A08F015
:101FF00059F801462046F1E7042BD3D0D9B2806AC4
:1020000002F0C3FACEE70968806A02F040FA22794A
:10201000044B214653F8223028469847C2E700BFB8
:102020004CFA010874E301082DE9F14F0D46A907A8
:102030000446164610D005F00F03022B15D12909CE
:102040000AB1022A04D1204601B0BDE8F04F2DE6C6
:1020500001B0BDE8F04F1BE66968CBB22A2B79D0FE
:102060000AD8062B0CD0292B11D0534A29462046DA
:1020700001B0BDE8F04FEFE62B2B7CD0902BF4D1D4
:10208000002EF2D105F108030A0A002185E0022A98
:1020900002D0A968FFF77CFFEF68002FE5D017F0AA
:1020A0000309E2D17B68DAB2862AB84607D1022E4C
:1020B0004FEA132812D108F1010857F8288098F840
:1020C00004302E2B28D1022E16D1A06A02F05EFB1E
:1020D000A06A01B0BDE8F04F02F020BB07F1080A8A
:1020E00008F1FF3BD945E6DA5AF8041B2046FFF712
:1020F0004FFF09F10109F5E72046D8F80810FFF76E
:1021000047FF012EA06AE4D102F019FBA06A01B0DA
:10211000BDE8F04F02F0EEBA2F2BA6D1012E0BD165
:10212000A06A02F004FBD8F80810A06A090901B0FF
:10213000BDE8F04F02F0BCBA022E02D1A06A02F054
:102140000FFBD8F80810A06A090901B0BDE8F04FEC
:1021500002F0D9BAA868002887D0002A85D1C168C2
:1021600031B311F0030323D14A68D6B28D2E16D1B4
:102170001A46816811E0002A7FF477AFA96821B977
:102180000B4601B0BDE8F04F18E08B0703D10B7987
:102190008A2B0846E3D000231A462046F1E78E2E0C
:1021A00003D101F10803120AE3E79F2E3FF45DAF6C
:1021B00000F10803022268E7CFE401082DE9F84F97
:1021C0000F1E06469046994614BF012500251DD0D6
:1021D00017F003041AD13B79202B17D12146806ACE
:1021E00002F02FFC08F1FF3BA9EB8509AA46BBF1E1
:1021F000FF3F0ED1631CA84425D14146B06A02F0CE
:1022000015FC4FBB45452AD1BDE8F88F4FF0FF3490
:10221000E8E759F82A1061B18A070AD10B79202B17
:1022200007D101340AD15A465146B06A02F009FC7E
:1022300054460AF1010A0BF1FF3BD8E730460F4A3A
:10224000BDE8F84F08E6002FDCD02CB9B96822466B
:102250003046FFF7E9FED5E700223946F8E7AC4201
:1022600009BF59F8243059F825109968002218BF81
:1022700000223046FFF7D8FE0135C3E7EAE4010843
:102280002DE9F74F06460D4614461F462846FFF730
:10229000AFF810B1002C4DD105E02846FFF7B6F895
:1022A00040B1012C46D1B06A394603B0BDE8F04FC9
:1022B00002F080BA002D58D0AB0756D16B684FEAB8
:1022C000132BDBB21C2B38D1002C3AD1D6F810805E
:1022D00008F1010333610BF1FF3305F1080A4FF0F8
:1022E00000090193019B99450FDB0BF10101304679
:1022F00055F821103B462246FFF7C2FFB06A41461F
:1023000003B0BDE8F04F02F013B9B4FA84F24346CB
:1023100052095AF8041B3046FFF7B2FF09F10109D0
:10232000E0E73B46224658F8041B3046FFF7A8FF7B
:102330004545F6D103B0BDE8F08F1D2B08D1002C28
:10234000C4D10BF1020305F1080805EB8305EFE7A3
:102350001E2B04D1B4FA84F46409AD6896E72A2BE5
:1023600003D1AB68002B9CD194E729463046FFF798
:102370000FFEB06A3A46214603B0BDE8F04F02F0C6
:1023800023BA2DE9F843066904461F46B31C0361CE
:102390000D46806A314606F10108914602F0C8F800
:1023A0004146A06A02F098FAA96800222046FFF789
:1023B0003BFE2D6905BB49462046FFF7E9FD636AF0
:1023C0001978062912D1A06A02F0ABFBA06A02F0CC
:1023D000BEF93146A06A02F0EDF9A06A414602F06A
:1023E000A7F8A06ABDE8F84302F080BABA00053247
:1023F000A06A02F00BFBECE72B79A02B07D1A968B0
:10240000334600222046FFF73BFFED68D2E7E9683C
:102410002046FFF7BDFDA06A012102F04EFA7B1CA9
:102420004A4629462046FFF7ACFFD2E72DE9F341A3
:1024300004460D46627100260661114645622A4631
:10244000806A01F0C4FE6779012F04BF6E84AE84F8
:10245000EE6866B1B2070AD13379382B07D1B1687B
:102460002046FFF795FDA06A02F043FB1FE02B78A2
:1024700043B931462046FFF78BFD0E21A06A02F0DA
:1024800084F8F0E7072B18D1012F07D10023A3719F
:102490003E224C4BF1682046FFF7B4FB20467169A1
:1024A000FFF776FDA06A01F04EFF0028E5D0A06A94
:1024B00001F01AFF02B0BDE8F081022B14D1012F08
:1024C00007D10023A37146223F4BB1682046FFF796
:1024D00099FBF1682046FFF75BFD2B7E5B07C2D5B9
:1024E000A06A02F034F9C8E7033B032B3DD8012F63
:1024F000D6F80C8008D10DF107023946606A0DF05C
:102500009BFB022303706F832B78032B1DD10021CB
:10251000A06A02F05AFA2B78062B1DD1A06A02F0AD
:10252000BFF801212046FFF7B3FBA06A02F0B8F81C
:10253000A06A02F0B5F80023B26841462046FFF7D2
:1025400020FF2B78062B8ED197E7042BE3D10021B7
:10255000A06A02F046FADEE720460121FFF798FB69
:102560000121A06A02F0A9F9E5E7012F07D10DF1D9
:102570000702062128460DF05FFB022303701B2192
:102580002046FFF785FB1A212046FFF78FFBB16835
:10259000A06A090902F066F81F212046FFF786FBB2
:1025A00031692046FFF7F4FC062128460DF034FB84
:1025B0000378022B3FF461AF4288A06A062101F044
:1025C000D2FE50E78B1F0008851F000838B50C4667
:1025D0000546C968FFF7DCFCA1682846BDE838401D
:1025E000D6E410B504468968FFF7D2FCA06ABDE8BE
:1025F000104002F07FB82DE9F84F0669B0F818B026
:10260000B0F81AA0B0F81E900683B31C036106F15F
:102610000108838BA0F81A800446C38388680D469E
:10262000FEF7E6FEE0B927697B1C2361A868FEF788
:10263000EDFE18B94146A06A02F0BCF83946A06A1E
:1026400001F076FFE9682046FFF7A2FC4146A06A48
:1026500001F06EFF3B460122A9682046FFF710FEFD
:102660002969A4F818B02046A4F81AA0A4F81E906E
:10267000FFF78EFC3146A06ABDE8F84F01F058BF65
:1026800010B504468968FFF783FCA06ABDE81040D6
:1026900002F05DB84B682DE9F04106460F461D0A71
:1026A00001F108080024AC4201DBBDE8F08158F8D4
:1026B000041B3046FFF76CFCB36843B1023406F1EB
:1026C0000C0057F82410BDE8F041FFF7BDBB013402
:1026D000E9E710B50446FFF7DDFFA06A2021BDE859
:1026E000104002F041B92DE9F3470669731C0361FC
:1026F000044688680D46FEF77BFE0246F8B9276956
:102700007B1C2361A9683B462046FFF7B9FD2046A4
:10271000E968FFF73DFCA868FEF778FEE8B92B6989
:102720000BB96B693BB1A06A01F00DFE18B93146D7
:10273000A06A02F03FF83946A06A01F0F9FE01AA4A
:102740006A2105F11000FFF773F80027824657450C
:102750000ADB69692046FFF71BFC3146A06A01F0DD
:10276000E7FE02B0BDE8F087019B53F82780D8F858
:102770000800FEF73DFE024608BBD4F8109009F1B0
:1027800001032361D8F808104B462046FFF778FD77
:102790002046D8F80C10FFF7FBFBD8F80800FEF72E
:1027A00035FE0028D9D1A06A01F0CDFD18B9314617
:1027B000A06A01F0FFFF4946A06A01F0B9FE0137A7
:1027C000C5E770B54379CD68012B0446164606D19E
:1027D000436A0A465B7E3146FFF740FA6861002390
:1027E0001A4669692046FFF781FAE9682046FFF733
:1027F000CFFB062E03D10021A06A02F05EF8002371
:10280000A06A1A460121BDE8704002F05BB92DE9CB
:10281000F04F87B0044603910292972105AA03A8BE
:102820001F46FFF705F84FF0000B0190D946DA4636
:102830005E46D846019B9B4516DB5EB1BAF1000FA0
:1028400067D1A06A01F02CFFB9F1000F67D1A06A2F
:1028500001F026FF029B002B67D0334642463946E3
:10286000A06A02F03AF910E0059A52F82B50002DB8
:1028700040D0A8073ED12A79992A0FD1F10707D570
:102880002D4A29462046FFF7E7FA07B0BDE8F08F4A
:1028900046F00106AA460BF1010BCBE79A2A07D1B5
:1028A000B20701D5254AECE746F00206A946F2E751
:1028B0009B2A1FD1EA6822B1930702D112799F2A7D
:1028C00011D0A96801F00F02022A01D01C4AD8E7F2
:1028D0000909A06A01F0C6FEE9682046FFF758FB27
:1028E00008F10108D7E7062229462046FFF769FFCD
:1028F0000137D0E70EB1134AC3E7B8F1000F01D09A
:10290000114ABEE729462046FFF742FB01374646FB
:10291000C1E7DAF808102046FFF73AFB94E7D9F848
:1029200008102046FFF734FB94E733464246394609
:10293000A06A02F0C7F8A8E704E501081BE5010852
:1029400033E5010854E501086FE5010870B50D464F
:10295000417901290446134603D12A46FFF77EF93F
:102960006861A06A01F0BEFE6E6900231A46314616
:102970002046FFF7BBF9718AA06A01F073FEE9688F
:1029800029B18B0703D10B79962B08BF0021204674
:1029900002230022FFF73BFF708A70BD10B5436A27
:1029A0005A7E0446FFF7D2FF01462046BDE810409C
:1029B000FFF77CB900231A46896828E770B58C6850
:1029C00005462CB92146A86ABDE8704001F0FDBF5C
:1029D000A2072CD123798A2B29D1E668EEB1B3075F
:1029E0001BD133798D2B04D1A168FFF7D1FA0121D6
:1029F000E9E78E2B0AD1A168FFF7CAFA31462846CB
:102A0000FFF748FE7168090A0131DCE79F2B04D10A
:102A100021460322BDE87040D3E6A1682846FFF7AF
:102A2000B7FAE1682846FFF7B3FA0221CBE721465F
:102A30002846DAE72DE9F3418C68054634B921468A
:102A4000806A01F0CEFF02B0BDE8F08114F0030609
:102A5000F9D12379322B0BD10121806A01F0C1FF1A
:102A600028462146FFF794FAA86A01F0C5FFEAE775
:102A7000922BE8D1E3681A79942A2FD101AA03F1A5
:102A800008009521FEF7D4FE411C8046A86A01F09B
:102A9000A8FF2846A168FFF77BFAA86A01F0ACFFFF
:102AA0004645D0DA019B53F8261081B18A070ED132
:102AB0000F79A7F132035F425F412846FFF768FABA
:102AC0003FB9094A21462846FFF7C6F9BBE7002768
:102AD000F3E7A86A01F090FF0136E1E704222146FE
:102AE000FFF76FFEAFE700BF64E301082DE9F04197
:102AF000804615460C4611B1FFF74AFA012435B15C
:102B00006E680027360A0835B74207DB3444214691
:102B1000D8F82800BDE8F04101F04BBF55F8041B80
:102B20004046FFF735FA0137EEE70A460021DDE7B8
:102B30002DE9F04F044685B08A4602AA3B210AF1EE
:102B40000800FEF775FE636ADFF8BCB05F7E002602
:102B500080463546464515DBDAF80C100B79032B19
:102B60003A46204640D1FFF74FF907460026A8EB2A
:102B70000505AE423BDB39462046FFF797F805B026
:102B8000BDE8F08F029B53F82630009303AA66211C
:102B900003F10800FEF74CFE039B19680A09B02AEE
:102BA00081462CD1022805D05A462046FFF754F919
:102BB000013517E059680B09652BF5D10127F7E7B7
:102BC000039AA06A52F823100193090901F070FDDD
:102BD000019B01334B45F3DB009BD96811B12046C3
:102BE000FFF7D6F90136B5E7FFF7B0FEBDE70023E2
:102BF0001A460121A06A01F065FF0136B9E72046B7
:102C0000FFF7C6F90123E5E791E5010801F00F039D
:102C1000022B70B5044610D04B6803F0F702412A2E
:102C200002D10123837170BD422A39D0DBB2402B1F
:102C30000CBF0D69CD688E684DB9A37983BBE38A5B
:102C400073B32046174ABDE87040FFF705B9837992
:102C5000F3B1838A01339BB2012B838208D1C18AED
:102C6000806A91B101F0A5FE0021A06A01F0B9FED1
:102C700029462046FFF78CF9A06A310901F0F2FCE1
:102C8000A06ABDE8704001F0B7BE01F009FDEBE7B6
:102C9000C38A01332946C382BDE87040FFF778B983
:102CA00070BD00BFAFE501082DE9F8430C46896807
:102CB0000646FFF76DF9E568002D00F083806F6828
:102CC000FBB2862B736A1B7819BF04F10C05012730
:102CD0003F0A0835072B4AD1A36803F00F02022AE6
:102CE00045D11B09DA2B42D12B681A792D2A3ED106
:102CF0009B68002B3BD106213046FEF7C9FF726A64
:102D0000D36A128D32B929682F4A3046BDE8F8439C
:102D1000FFF7A2B85978C9070DD559683046FEF7B4
:102D2000B7FF022F0AD800231A460221B06A01F029
:102D3000C9FE012417E0013A0833E3E76B681A790A
:102D40002F2AF0D1AC6822792D2AECD19968B06A8B
:102D50000122090901F0B6FCA168002301223046D6
:102D6000FFF755FD0324A74203D8BDE8F8830024EC
:102D7000F9E704F1010847451DD955F824201179D8
:102D80002F294FEA840316D12B44D3F8049099F8E5
:102D900004302D2B0FD19168B06A0022090901F08F
:102DA00091FC00230122D9F808103046FFF72FFDCF
:102DB00008F10104D7E755F824103046FFF7E8F88A
:102DC000A046F5E7BDE8F883DDE501082DE9F0410F
:102DD0004D68114F0C4689680646FFF7D9F82D0A51
:102DE0004FF00208454501DCBDE8F081216930461D
:102DF000FFF7CEF8E368B06AC3F307132F3B082B45
:102E000096BFDB19192193F8D81001F0ADFD08F138
:102E100002080834E6E700BF74E301084B682DE9B7
:102E2000F0410C468968074690461D0AFFF7B0F846
:102E30000C340126AE4201DBBDE8F08154F8041BDE
:102E40003846FFF7A5F84146B86A01F08DFD013616
:102E5000F0E71722E2E71622E0E71522DEE72DE988
:102E6000F041CD6804460F4645BB0379A3B1436AE0
:102E70001D788DB92021FEF70BFFB9682046FFF7BA
:102E800087F82B462A460121A06A01F01BFEA06AA2
:102E9000BDE8F04101F05BBCB968880707D001F0DC
:102EA0000F03022B08D12046FFF772F8EFE7002945
:102EB000F9D00B79352BF6D1BDE8F081A90740F0A8
:102EC000BC806B68DAB2512A17D10122B968FFF7CA
:102ED000ABF8E9682046FFF75BF8AB68A06A1B090E
:102EE0004E3B0A2B9BBF584A9B18142193F8E110C4
:102EF00001F03AFD0222B96858E0522A25D11B0A96
:102F000003F1FF38013355F82310FFF741F8B8F10A
:102F1000000F02DDA06A01F00AFC0022B968204619
:102F2000FFF782F808350026464501DBBDE8F08151
:102F30000136B04502DDA06A01F0F9FB002255F828
:102F4000041B2046FFF770F8EEE7062A75D1BE682D
:102F5000002E72D0B2072ED17268D1B206292AD1C2
:102F6000190A022927D1120A022A24D1B36823B1EF
:102F7000980702D11B79202B5FD0F36823B1990702
:102F800002D11B79202B58D0A9682046FFF700F802
:102F9000E9682046FEF7FCFFA06A01F0E1FB002291
:102FA000B1682046FFF740F8F16800222046BDE8EE
:102FB000F041FFF739B8002E3FD0B2073DD172681B
:102FC000D1B2062939D11B0A032B36D1120A032AA2
:102FD00033D1B36823B1980702D11B79202B2CD0B1
:102FE000F36823B1990702D11B79202B25D03369CF
:102FF00023B19A0702D11B79202B1ED0A968204645
:10300000FEF7C6FFE9682046FEF7C2FF29692046A1
:10301000FEF7BEFFA06A01F0B9FBA06A01F0A0FBB9
:103020000022B1682046FEF7FFFF0022F16820462B
:10303000FEF7FAFF00223169B8E729462046FEF77D
:10304000A7FF002257E700BF74E3010838B50C461C
:10305000C9680546FEF79CFFA368C3F307132F2B2F
:1030600008D0302B0CBF01210221A86ABDE83840EE
:1030700001F06EBC0021F8E710B504468968FEF740
:1030800087FFA06A0321BDE8104001F061BC2DE973
:10309000F843D0F8108008F1010303614E6804463C
:1030A0009146360A01F108050027B74205DB414683
:1030B000A06ABDE8F84301F03BBA55F8041B20466E
:1030C0000137FEF765FFBE42EFDD42464946A06A82
:1030D00001F08BFBE9E70022D9E70122D7E72DE9D0
:1030E000F8434E68DFF8C89004460D46360A8968F2
:1030F000FEF74EFF032E83BFD4F8108008F10103C2
:1031000023614FF0000801277B1C9E421CDC032E2C
:103110004BDD2569A06A6B1C2361294601F04AFB3F
:103120004146A06A01F004FA0121A06A01F00DF9FC
:10313000A06A01F015FBA06A01F009FB2946A06A0C
:10314000BDE8F84301F0F4B9296920460237FEF7DB
:103150001FFFBE4205DDA06A01F0E9FAA06A01F096
:1031600015FBEB6803F00F020E2A13D11B09363B47
:103170000B2B96BF4B44062193F8EC10A06A01F08C
:10318000F3FBBE4204DD42460021A06A01F02DFBA4
:103190000835B9E71A797D2A01D12321EEE79B682A
:1031A0000BB90721EAE72421E8E7BDE8F88300BF6F
:1031B00074E301082DE9F0410569CF68AB1C036198
:1031C000884604462B460022B968FFF759F86E1C62
:1031D000D8F808102046FEF7DBFE3146A06A01F061
:1031E000E9FA2946A06A01F0A3F9A06A4FF0FF317D
:1031F00001F0ABF8F9682046FEF7CAFE3146A06A36
:10320000BDE8F04101F094B92DE9F04F8B6803F06F
:103210000F03022B8BB004460D4640F0EE80CB68C6
:10322000002B00F0EA80980740F0E7801A79292AFD
:1032300040F0E3809A6802F00F01022940F0DD803F
:103240001209BE2A40F0D980DB681A792D2A40F095
:10325000D4809B68089309AA972108A8FEF7E8FA8A
:10326000431E022B00F2C9800128099940F0B78063
:10327000D1F8009003260246930704D111799939B9
:10328000022940F2BA80B9F1000F08D019F0030FFB
:1032900005D199F804109939022940F2AE80AB6843
:1032A00001932B690293238B6F6903932569638BC9
:1032B0000493E38B05936B1C0693BDF81830A18B28
:1032C0006383E1836FEA0903291D19F0010805F101
:1032D000020A258305F1030B2161069305D14946B6
:1032E00020460792FEF754FE079A11462046FEF745
:1032F0004FFE5946A06A01F05DFA5146A06A01F0FE
:1033000017F9A06A01F013FA002201992046FEF78E
:103310008BFE02992046FEF73BFE691CA06A01F075
:1033200007F931462046FEF733FE0E21A06A01F070
:103330001BFBA06A594601F0FBF8A06AB8F1000F28
:1033400040F0A28001F0FBF9A06A01F009FA002E1A
:10335000ACBF00210121A06A01F006FB5246012109
:10336000A06A01F031FABDF80C302383BDF81030AB
:103370006383BDF81430E383002F00F08C80A06AD3
:1033800001F0E5F9B8F1000F02D1A06A01F0DFF910
:1033900039462046FEF7FCFD2669A06A731C2361AE
:1033A000314601F007FA069BA06A03F001010131E2
:1033B00000F0CBFFA06A294601F0BAF8A06A01F03C
:1033C000C6F9B8F1000F02D1A06A01F0C0F91FB12F
:1033D0003146A06A01F0ACF80BB0BDE8F08F0228CE
:1033E00091E8040204D10326002A3FF44CAF43E7DE
:1033F0008E68F10701D57308F6D12669A38BB4F85E
:103400001E90E3836FEA46436FEA5343B4F818B063
:103410002383F31C2361771CB4F81AA0E96867833F
:103420002046FEF7B5FD0121A06A01F046FA06F13B
:1034300002083946A06A01F07BF84146A06A01F013
:103440004BFA0022A9682046FEF7EEFD20462969C6
:10345000FEF79EFDA06A00F076FF18B93946A06A13
:1034600001F0A8F94146A06A01F062F8A06A01F0F3
:103470003DFAA4F818B0A4F81AA0A4F81E9069693F
:103480002046FEF785FDA3E701F051F949462046A5
:10349000FEF77EFD5BE73E468CE72DE9F0470446EC
:1034A000904699460F4621B91946BDE8F047FEF708
:1034B0006FBD0669731C036115683DB315F0030AFF
:1034C00024D12B79742B21D1A968FEF761FD3146F7
:1034D000A06A01F0CBF95246E9682046FEF7A4FD48
:1034E0002046FEF785FB4B4608F10402791E204674
:1034F000FFF7D3FFA06A314601F005FAA38BA06A5B
:10350000013BA383BDE8F04701F0CEB92946204630
:10351000FEF73EFDA06A314601F0A8F9A06A01F06D
:1035200016F9DDE737B50C46054601AA732104F10B
:103530000800FEF77DF9E368019A01462846FFF787
:10354000ACFF03B030BD2DE9F04F85B005691E46D4
:103550000E9B0393AB1C044603610F46806A294609
:10356000934601F08DF92046FEF742FB394620468E
:10357000FEF70EFD05F1010AA06A01F0BBF9514604
:10358000A06A01F017F92946A06A00F0D1FFA06AED
:1035900001F0E4FAD4F8108008F10103236100235C
:1035A0005B4517DBA38BA06A013BA38301F07CF989
:1035B000A06A01F0D6FA5146A06A00F0B9FF03995B
:1035C0002046FEF7E5FCA06A414605B0BDE8F04F95
:1035D00000F0AEBF3146D4F810900A68019209F1AC
:1035E00001022261019A9768013304360293002F89
:1035F00046D15B4539D1A06A01F0A9F800252F46D4
:10360000019B2046D968FEF7C3FC15B1A06A01F002
:1036100071F9A06A01F093F9CDB10E21A06A00F012
:10362000B4FF3946A06A00F083FF0E21A06A00F0C3
:10363000ACFF29462046FEF739FB20462946FEF717
:1036400043FBA38BA06A013BA38301F02DF9414604
:10365000A06A01F0AFF84946A06A00F069FF0121B5
:10366000A06A00F072FE029B9AE71C4A0968204695
:10367000FEF7F2FBA38B013BA38305B0BDE8F08FFF
:1036800017F0030527D13A796F2A3B4602D1DD684E
:10369000BF682D09A06A01F04AF839462046FEF7B6
:1036A00077FC0821A06A01F05FF94A460021A06A70
:1036B00001F08AF8002D9ED029462046FEF7F6FA42
:1036C0002769A06A7B1C2361394601F0E3F8204694
:1036D000FEF78EFA94E70025DCE700BFF5E5010868
:1036E0002DE9F3470569DDF828A0DDF82C8099461F
:1036F0006B1C044603610E46806A2946174601F09A
:10370000C9F82046FEF774FA27BB0321A06A00F02F
:103710001CFE31462046FEF73BFC6FF00201A06A1A
:1037200000F013FEA06A01F0E5F8A06A0E2100F097
:103730002CFF2946A06A00F0FBFE20464146FEF71A
:1037400027FCA38BA06A013BA38302B0BDE8F0472E
:1037500001F0AAB8CDF800A04B463A4631462046C3
:10376000FFF7F1FEDEE77FB5CD682B79712B0646BA
:103770000C4609D1AB6801930023009389681A466F
:10378000FFF7AEFF04B070BD6D2B03AA4FF07001C0
:1037900016D105F10800FEF74BF82B6902463BB93C
:1037A000EB680093039BA1683046FFF7CCFEE9E786
:1037B0009B680193EB680093A168039B3046DFE7A9
:1037C00004F10C00FEF734F8002300930246039B3B
:1037D000E9E72DE9F04705460C4604F00F03022BFC
:1037E00005D121092846BDE8F047FEF76DBA002C47
:1037F00064D0A20762D12379292B35D1A16828464C
:10380000FEF7C6FBE668002E58D016F0030855D127
:103810007768FAB2862A334609D13F0A06F10809C9
:1038200007F1FF3AD0450EDB013756F827301A79F9
:103830002E2A10D128469968FEF7AAFBA86ABDE88F
:10384000F04700F0ABBF59F8041B2846FEF7A0FB79
:1038500008F10108E6E72F2A30D19968A86A09091A
:10386000BDE8F04700F084BF2A2B27D1A4682CB311
:10387000E668EEB1B3071BD17768FAB28D2A01D1A1
:10388000A468AAE78E2A11D1A1682846FFF7A1FFF4
:103890003F0A08360024BC4201DBBDE8F08756F839
:1038A000041B2846FFF795FF0134F4E79F2A05D053
:1038B000A1682846FFF78DFFE4688EE72146284679
:1038C000024ABDE8F047FEF7C7BA00BF13E6010899
:1038D000426A1278072A10B5044604D0094ABDE8A6
:1038E0001040FEF7B9BA896841B90E21806A00F02C
:1038F0004CFEA06ABDE8104001F0FBB8FEF748FBA3
:10390000F7E700BF2BE6010838B5436A1B78072BA1
:1039100004460A4606D0022B04D0154ABDE83840BA
:10392000FEF79ABA916841B90E21A06A00F02DFE07
:10393000A06ABDE8384001F0F4B811F0030513D1D6
:103940000B79A22B10D120468968FEF721FB29466E
:10395000A06A00F0B2FFA06A0E2100F016FEA06A75
:10396000BDE8384001F0EBB82046FEF711FBDFE779
:1039700045E60108896830B4054619B9806A30BC4B
:1039800001F017B8CB689BB113F0030210D11C797A
:103990008D2C03D1896830BCFFF7A8B88E2C01D1DB
:1039A0001A46F7E79F2C03D1062230BCFEF709BF69
:1039B0000A4628460021EEE7F8B5134B5E6F044631
:1039C0000F4606BB05696B1C036101222B46896803
:1039D000FEF756FC3E21A06A00F0EBFCF96841B10D
:1039E0002046FEF7D5FA334632460121A06A01F09F
:1039F00069F8A06A012101F088F82946A06ABDE8AB
:103A0000F84000F095BDF8BD3C21002038B58C6829
:103A100005462CB92146A86ABDE8384001F075B8C2
:103A2000A3070BD12379582B08D1A168FEF7B0FA70
:103A3000E1682846FEF7ACFA0221ECE72146284669
:103A4000FEF7A6FA0121E6E72DE9F74F4379012BAE
:103A500004460F4605D1436A1B782BB91A4AFEF774
:103A6000FBF903B0BDE8F08F01AA672107F1080058
:103A7000FDF7DEFEDFF85490DFF854A08046002505
:103A8000A845EEDD019B606A53F8256036090DF10B
:103A9000030231460CF0D0F89DF80330834673B131
:103AA00001463246606A0CF0F2F89BF8003023B908
:103AB000524639462046FEF7CFF90135E0E7037854
:103AC000042BFAD04A46F4E75EE60108A1E60108B5
:103AD00083E601082DE9F3474479012C0646884620
:103AE0000BD101AA672108F10800FDF7A1FEDFF85C
:103AF00050A081460025A94502DC02B0BDE8F08750
:103B0000019B706A53F825703F090DF10302394695
:103B10000CF092F89DF803304BB90378012B06D0D6
:103B2000524641463046FEF797F90135E3E7047007
:103B30003946706A0CF0A5F80028F6D00470F4E756
:103B4000C2E601082DE9F74F80460C4611B9012164
:103B5000116013E011F0030517D10B79622B06D128
:103B6000CB681B0913608C68002CF0D0012504F091
:103B70000F03022B0BD12109002DE9D0D8F800004A
:103B800000F0E5FC03B0BDE8F08F0025EFE715B9C4
:103B9000A3681B091360666804F1080A360A771ED9
:103BA000D3464FF000094E4521DC384669460AF0FD
:103BB00057FC4FF0000907464FF02E0B4E451FDC17
:103BC00000980AF058FC0146D8F8000000F0BFFC4D
:103BD000002DD7D00C340125AE42D3DD54F8041BA0
:103BE000D8F80000090900F063FD0135F4E75BF83F
:103BF000040B00090AF05EFC09F101090744D2E751
:103C0000B9F1000F02D087F800B001375AF8040B61
:103C100001A900090AF058FC019A014638460CF047
:103C20009CFE019B09F101091F44C7E72DE9F341FF
:103C30008D6805F00F030E2B04460E4606D0002DAE
:103C40003DD0AB073BD12B795F2B2AD100950025C6
:103C500001AA5F216846FDF7EBFD0023019A194692
:103C600040F2AE4E834222DBF268A06A40F21E337D
:103C70009A4226D1264600F0AFFC2621A06A00F029
:103C8000F1FC56F8280F012100F093FE304601AAFE
:103C90002946FFF757FFA06A00F06EFC02B0BDE8AE
:103CA000F0815C2B0BD1AB680093ED68D0E752F844
:103CB000237077450CBF013103310133D2E7002176
:103CC000D2E700F089FC06F10C006A466421FDF79A
:103CD000AFFD00260746BE4211DB2646394656F8A0
:103CE000280F00F066FE294601AA3046FFF72AFF9A
:103CF0000025BD420DDBA06A00F029FDCEE7009B48
:103D0000A06A53F826309968090900F0ABFC013627
:103D1000E1E7009BA06A53F82580D8F808603609CF
:103D2000314600F01FFCD8F80C1029B93146204666
:103D3000FDF7BCFF0135DCE70909F8E773B5044678
:103D400025460E46806A002100F046FC55F8280FF3
:103D50000E2100F01AFC01AA31462846FFF7F2FEB8
:103D600001992046FDF7A2FF02B070BD2DE9F04F8A
:103D70008FB00F46144606462C22002103A81D468C
:103D80000CF00EFE4FF6FF73ADF82430ADF8263080
:103D9000326803972346002103A88DF81050FDF7E1
:103DA0005DFF044600F0FEF90B9F0D9005464FF0B5
:103DB0000008002F2FD10B9B13B1059A002A38D091
:103DC0004146284600F0F1F90B9F059B17B1002BE7
:103DD00000F0E1805BB10C9B06A8D968FEF734F8CF
:103DE0000C9B069A5B8A0399059803F023FE2846EC
:103DF00000F0E3F93046FDF7F1FE6569A66820465C
:103E00000BF000FF3446002EF8D10598002800F092
:103E1000D880FCF7BFFA059B002BCCD13946012294
:103E200003A8FEF703FB079BBF68984538BF984679
:103E3000BFE7197ECF071FD5188D411EC900D8B125
:103E4000DF6A0F4497F801E01EF0020F39D09AB1F3
:103E500097E8030092F800A092F80190B2F802C02F
:103E6000D2F804E082E8030087F800A087F8019008
:103E7000A7F802C0C7F804E04FF00002B3F828C06A
:103E80001A840021614524DB0022944541DCD3F8EB
:103E90000490B9F1000F12D0B9F828200192002146
:103EA0000A460198814244DB4AB100218C4563DC1B
:103EB000598B92B211445983198C0A441A849B6815
:103EC0007AE71AB9BEF1010F08BF3A46013808393E
:103ED000B5E71A78DF6AC800012A07EB000E05D1A2
:103EE000DEF80420062A07D10131CBE704D93A5C79
:103EF00012B94FF001023A543A5C022A03D09EF8FC
:103F00000120D007F0D51A8C501C1884AEF802207E
:103F1000EAE7D96A01EBC20011F83210032906D191
:103F20004178C9075FBF198C418001311984013282
:103F3000ABE7D9F82C0000EBC10B10F831000338C7
:103F4000012803D84FF0000EF44501DC0131A8E749
:103F5000D86A00EBCE0A10F83E00042809D1DAF83E
:103F600004000746DBF80400B84204BFAAF80220A8
:103F700001320EF1010EE7E7DF6A07EBC10017F827
:103F80003170042F02D14778FF0702D547881744C4
:103F9000478001318AE70222394603A80D95FEF7D2
:103FA00045FA059B23B90322394603A8FEF73EFADA
:103FB000059B23B90422394603A8FEF737FABF68E8
:103FC00003E732463146284601F0C8F90FB0BDE894
:103FD000F08F00BF37B50DF107020D4604460BF018
:103FE0002BFE9DF8073001461BB12A4620460BF0F8
:103FF0004EFE03B030BD13B50DF1070204460BF0C1
:104000001BFE9DF80720237832B1012B01D9022332
:1040100000E00023037004E0012B02D90378002B99
:10402000F5D002B010BD70B505460E4610461946D3
:104030001C460BF0F1FD03782BB9B36821462846E6
:10404000BDE870401847012B01D1F368F6E7022B59
:1040500042880CBF3368736821462846BDE870402B
:104060001847000037B50DF105040B46214602F054
:104070007F05D20904F8015DF9D1091B984701AD0C
:10408000411E2346AB4205D19DF804201B1BC254A0
:1040900003B030BD13F8012B62F07F0201F8012F4D
:1040A000F0E742790346032A026A89BF186B521867
:1040B0008018521894BF02621A62704710B50C46FD
:1040C0000121FFF7EEFF047010BD4279032A10B5FD
:1040D0000346826A02D80A44826210BD406A1418FC
:1040E000186B0A4420449A6210BD10B50C46012199
:1040F000FFF7EBFF047010BD38B504461546FFF717
:10410000F4FF2A4620460249BDE83840AAE700BF2E
:10411000CB4000082821EFE72921EDE738B5044618
:104120001546FFF7E2FFA36A033323F00303A362FC
:1041300004212046FFF7C9FF056038BD38B5437933
:10414000032B81BF846AC369C4F1FF2404F57F0493
:1041500084BF53F82230FD340D464FF003018CBF6D
:10416000E4180024FFF7B1FF4470240A057084703E
:1041700038BD38B54379032B81BF846AC369C4F560
:10418000FF4453F8223088BF7D340D464FF00301C1
:104190008CBFE4180024FFF798FF447024120570C8
:1041A000847038BD38200AF04FB810B504468161DC
:1041B00088000AF03DF8E06110BD10B50446C06902
:1041C0000AF062F82046BDE810400AF05DB8F8B584
:1041D000044600236171032983608371E2600361F7
:1041E0004FF001030F461546436106D88269C06946
:1041F00092004FF0FF310CF0D3FB0023A362236247
:104200002A8C6B8C3749D21808BF01222046FFF751
:1042100029FFAA8C33492046FFF724FFE368204694
:10422000197EFFF74BFFE3682046997EFFF746FFB4
:10423000E3682046197FFFF741FFE3682046997F36
:10424000FFF73CFF042F23D1626A236A2549D21A63
:104250002046FFF707FF6A8A22492046FFF702FF40
:104260002A8A20492046FFF7FDFE00262B8D9E421C
:1042700013DBFF212046FFF738FF042F31D1688B75
:10428000AB8B0022184482422BD02E8D002124E0DB
:1042900002212046FFF705FFDDE7EB6A03EBC602CC
:1042A00013F83630032B03D191782046FFF71DFF1A
:1042B0000136DBE7EB6A03EBC1035F78FF070BD541
:1042C0005F88BA4208D15B68616B9B0043F00203D0
:1042D00041F822300132D6E70131B142EADB262330
:1042E000F2E7F8BDA34000084379012B13B504465B
:1042F00019D00021FFF7E2FE6379032B15D1236A61
:10430000A06AE062033323F003032362636218446C
:1043100009F09AFFE3682063588B9B8B1844800058
:1043200009F092FF606302B010BD042BFBD1E0687E
:10433000616A037EE26A00930A44636B216B406901
:1043400000F0FEFFEFE7807970474379012B09D039
:1043500083681944C36881605A8C9142C8BF5984EC
:1043600000238371704738B501211446FFF7EDFF34
:104370000F2C05D8A4F15001C9B2BDE83840B4E60D
:1043800022461921BDE83840B6E638B50121154668
:10439000FFF7DBFF2A461A21BDE83840ACE638B506
:1043A0000D460121FFF7D1FF2A461B21BDE8384009
:1043B000A2E638B50D460121FFF7C7FF2A461C21AA
:1043C000BDE8384098E638B54FF0FF311446FFF7A6
:1043D000BCFF0F2C05D8A4F14001C9B2BDE838409C
:1043E00083E622462221BDE8384085E638B54FF005
:1043F000FF311546FFF7A9FF2A462321BDE83840C3
:104400007AE638B50D464FF0FF31FFF79EFF2A469A
:104410002421BDE838406FE638B50D464FF0FF3136
:10442000FFF793FF2A462521BDE8384064E638B5FA
:104430000D460021FFF789FF2A462A21BDE83840B2
:104440005AE638B50D460021FFF77FFF2A462B219B
:10445000BDE8384050E6F8B5069C1E46079B154659
:10446000891B620007462402891A53B10239FFF7FB
:104470006CFF691C44EA0602C9B23846BDE8F84040
:104480003AE6FFF762FF44EA0602E9B2F5E7274B96
:104490005B6F022B2DE9F04706468A4643D84569F3
:1044A0008D4240D2846A03694D1BE41A40F2FF79C1
:1044B00034B91DBBB36A3361C6F814A0BDE8F087F8
:1044C000062D01D90F2C1BD91F2CA04628BF4FF059
:1044D0001F08444510D8032D2F4628BF032701216C
:1044E0003046FFF7DEFD48EA47130370A4EB0804EB
:1044F000ED1BDDE7A046EEE70027F0E7062DF9D932
:104500004D452F464FF0020128BF4F463046FFF77A
:10451000C8FD3B0903F0700364F07F02134303708E
:104520004770A046E2E7BDE8F08700BF3C210020CD
:1045300038B50D460021FFF708FF4379012B05D060
:10454000032B9EBFC369826A43F8252038BD38B566
:104550000D464FF0FF31FFF7F8FE2A466821BDE80F
:104560003840C9E538B50D460121FFF7EEFE2A4671
:104570006921BDE83840BFE510B54FF0FF31FFF7C6
:10458000E4FE6A21BDE81040AFE538B50D460121D3
:104590000446FFF7DAFE0E2D08D00F2D08D00D2DA2
:1045A00008D110212046BDE838409EE51121F9E7E9
:1045B0001221F7E71721FFF798FDA36A033323F0D1
:1045C0000303A36204212046FFF77FFD014B036034
:1045D00038BD00BF8CFA010873B50C4601210646B0
:1045E000FFF7B3FE04F110033F2B06D8A4F18001BE
:1045F000C9B2FFF77AFD02B070BD1421FFF775FD57
:104600000DF105031946E2B202F07F00E41103F850
:10461000010C601C012803F1FF3516D8013402F0AB
:10462000400214D11AB97F2205F8012C9D1E491BA6
:104630003046FFF74AFD01AC411E2B46A3420AD18A
:104640005D1B9DF804204255D5E72B46DBE7002A89
:10465000EDD00022E8E713F8012B62F07F0201F8A9
:10466000012FEBE738B50D460121FFF76EFE2A4614
:104670001621BDE838403FE538B504460D46012116
:10468000FFF763FE1721FFF730FDA36A033323F022
:104690000303A36204212046FFF717FD056038BD20
:1046A00010B50121FFF751FE1821BDE810401CE5AF
:1046B00038B50D460021FFF748FE2A461D21BDE80A
:1046C000384019E570B50E4651001446C1F101019C
:1046D000FFF73BFE002C324614BF1F211E21BDE810
:1046E000704009E510B50121FFF72FFE2021BDE83C
:1046F0001040FAE410B54FF0FF31FFF726FE2121FC
:10470000BDE81040F1E438B50D466FF00101FFF748
:104710001CFE2A462621BDE83840EDE410B56FF0B6
:104720000201FFF712FE2721BDE81040DDE410B5BD
:104730000121FFF70AFE3021BDE81040D5E410B595
:104740000221FFF702FE3121BDE81040CDE410B593
:104750004FF0FF31FFF7F9FD3221BDE81040C4E40E
:1047600010B50021FFF7F1FD3321BDE81040BCE496
:1047700038B504460D46FFF793FF2046FFF7F0FFDC
:1047800029462046BDE83840FFF7BDBF10B50021DF
:10479000FFF7DBFD3421BDE81040A6E410B5044668
:1047A000FFF77EFF2046FFF7F1FF2046BDE81040EF
:1047B000FFF7B4BF38B50D460021FFF7C6FD2A4606
:1047C0003521BDE83840D4E470B515460E464FF0AB
:1047D000FF310446FFF7B9FD2A4626B136212046AF
:1047E000BDE87040C5E43721F9E770B515460E46BF
:1047F0004FF0FF310446FFF7A8FD2A4626B13821C5
:104800002046BDE87040B4E43921F9E7F8B5044624
:10481000164601F4004721F40045CAB91146FFF7D6
:1048200094FD2FB92A4620463521BDE8F840A0E482
:104830003221FFF75AFC20463221FFF756FC204672
:104840003221FFF752FC32212046FFF74EFCE9E708
:1048500046212A46FFF78DFC002F14BF802100213E
:1048600031432046C9B2BDE8F8403EE438B50D46B4
:104870000221FFF76AFD2A463D21BDE838405DE48C
:1048800038B50D460021FFF760FD2A463F21BDE8FF
:10489000384053E438B50D460021FFF756FD2A464F
:1048A0004021BDE8384049E410B54FF0FF31FFF733
:1048B0004CFD4121BDE8104017E438B50D460029F4
:1048C00014BF03210021FFF740FD002D14BF472135
:1048D0004221BDE8384008E438B50D460121FFF714
:1048E00034FD2A464321BDE8384027E46FF0030138
:1048F000FFF72BBD10B50021FFF727FD4421BDE8D0
:104900001040FFF7F2BB38B504460D46FFF7F2FF43
:1049100020460E21FFF739FE29462046FFF708FE04
:1049200020460221FFF711FD20463E21FFF7DDFB67
:1049300020466FF00301BDE83840FFF706BD10B513
:104940000021FFF702FD4521BDE81040FFF7CDBB78
:1049500038B50C460021FFF7F8FCA4F13001C9B2CC
:10496000BDE83840FFF7C1BB232970B505460C46AA
:1049700019D024291AD1012607244FF0FF312846E7
:10498000FFF7E3FCA4F12901C9B22846FFF7ADFB0C
:1049900076B128460021FFF7D8FC2846D321BDE890
:1049A0007040FFF7A2BB01260624E6E70026E4E7F5
:1049B00070BD38B50C46C1F10101FFF7C6FC2246B7
:1049C0005021BDE83840FFF797BB38B50C46C1F120
:1049D0000101FFF7BAFC22465121BDE83840FFF73C
:1049E0008BBB38B50D460121FFF7AFFC2A4653219A
:1049F000BDE83840FFF780BB10B56FF00101FFF74D
:104A0000A4FC5421BDE81040FFF76FBB70B5CC1E6D
:104A100018BF01241546E143FFF797FC621944EAE9
:104A200082025721BDE87040FFF766BB38B50C46DF
:104A30000139FFF78AFC22465921BDE83840FFF7CB
:104A40005BBB70B50C4615461144FFF77EFC44EA8B
:104A500005225A21BDE87040FFF74EBB38B5044629
:104A60000D4652B94BB90121FFF76FFC6A6960210D
:104A70002046BDE83840FFF751BB4FF0FF312046DC
:104A8000FFF763FC6A696121F2E770B50E460446E0
:104A90000499D5B27BB971B9C2F10101FFF755FC98
:104AA000726962212046FFF739FB29462046BDE89E
:104AB0007040FFF71ABBD1432046FFF746FC7269EE
:104AC0006321EFE707B58DE80C000B466422002157
:104AD000FFF7C1FC03B05DF804FB07B58DE80C00DF
:104AE0000B4666224FF0FF31FFF7B5FC03B05DF8CF
:104AF00004FB10B54FF0FF31FFF727FC0123837152
:104B00005B21BDE81040FFF7F0BA38B50C464942CA
:104B1000FFF71BFC0221FFF7D8FA5C2303704470F7
:104B200038BD10B50021FFF710FCC268137E43F0BA
:104B3000040313765D21BDE81040FFF7D6BA10B527
:104B40004FF0FF31FFF701FCC268137E43F004030E
:104B500013765E21BDE81040FFF7C7BA0421FFF7C6
:104B6000F4BB6FF00201FFF7F0BB00BF2DE9F04F7F
:104B70002DED028B85B006291D46B0EE408A824697
:104B80000E4617469DF8403014D8012907D93F2317
:104B9000037000F1010A00238AF8003001E00029C7
:104BA000F9D1012E94BF0020012005B0BDEC028B8D
:104BB000BDE8F08F10EE102A002A3DDAB4EE400A6C
:104BC000F1EE10FA38D12D23441C0370B1EE408A67
:104BD00007F0200318EE100A0293CDF80CA018F08D
:104BE000BDF90022CDE9000100230020BC499DF859
:104BF00008B018F031FB8046894602460B46DDE9D5
:104C0000000118F067FC38B9424609F10043DDE9BC
:104C1000000118F05FFCB8B18BF0490323708BF0F2
:104C20004E038BF0460B6370E01C84F802B0002347
:104C30000370A0EB0A00B8E723B10AF101048AF877
:104C40000030C5E75446C3E7B4EE488AF1EE10FAE7
:104C500009D04BF04E038BF0410B237084F801B068
:104C6000E01CA370E3E7002D47F02007B8BF06253E
:104C7000672F02D1002D08BF012518EE103A013E22
:104C8000A4EB0A00002BA6EB000641D1662F31D120
:104C90006B1C9E42D8BFB51E00216A1C66200E46C2
:104CA0000B4625EAE575652840F010816A1C4FF037
:104CB000000E4FF02E08F2EE047A724577DDBDEE5D
:104CC000C80AB64510EE109A09F1300904F1010C3A
:104CD00084F8009004D11DB104F1020C84F8018025
:104CE000B8EEC00A0EF1010E38EE408A644628EE96
:104CF000278AE2E76B1D9E42D8BFB51F652F384655
:104D00004FF0000240F0D2802B2116461346C8E730
:104D1000B3F17E5F7BD2DFED737A7348B4EEE78A3E
:104D2000F1EE10FA4FF00002ACBF4FF0310E4FF031
:104D3000300E2021134600F1180CB0EC017AB4EECD
:104D4000C87AF1EE10FAC4BF0CEB020898ED007AB5
:104D500002F10402C4BF5B1828EE078A182A4FEA42
:104D60006101EAD118EE102AB2F17E5F33D2B4EEBF
:104D7000E78AF1EE10FA29DB002B14BF2D212B213D
:104D8000B7EE008A662F03D0672F36D1042B34DCB0
:104D9000672F04BF03F1FF32AD186A1C9642D8BFDB
:104DA000B51E84F800E0C5B9013466202946662F97
:104DB00040F0A080012B00F3D780F1EE047AB4EE2E
:104DC000E78AF1EE10FAC0F2CF809AE0F2EE047AB0
:104DD00028EE278A01332D21D4E72E22627030215C
:104DE0002A460234013B63D01AB911464FF0FF3610
:104DF00044E004F8011B013AF4E7721F954261DBBD
:104E0000672F57D0B51F38460022164649E7374866
:104E1000002220211346A0F1180EF0EC017AF4EEE6
:104E2000C87AF1EE10FA9CBF0EEB020CDCED007AB2
:104E300002F104029CBF5B1828EE278A182A4FEA69
:104E40006101EAD1F2EE047AB4EEE78AF1EE10FAEB
:104E5000A2BFDFED277A013328EE278A662F0FD114
:104E6000B3420FDAEA180132964203DCF61AB51E95
:104E700000D5751E5A1901321E460021662010E722
:104E8000652F08D1721F954200DBB51F00222B2130
:104E90001646652005E7672F0ED12A1D9642D8BF1A
:104EA000751FAB420CDA5A1CAD1AE3E711462CE72A
:104EB00019469BE71546A6E7384600222B21A4E7B2
:104EC0006720FAE7002238461646ECE667287FF4AA
:104ED000EEAE15B901221546E9E62A46E7E600BF1F
:104EE0000000F03FF8FF7F3F14E701082CE70108BE
:104EF000CDCCCC3DF1EE047AB4EEE78AF1EE10FAB7
:104F000025DB621E4FF0300E16782E2E4FD0A6F104
:104F1000300CBCF1090F40D902F1010A9AF80020C7
:104F2000302A14D19AF801602E2E44D1662842D03E
:104F30002D298AF800608AF801203AD1013B08BF88
:104F40002B212246924538D331228AF80020672F40
:104F50000AD14DB122461446013A14F8010C30280A
:104F6000F9D02E2808BF144691B1029A61700A2028
:104F700042F04502227093FBF0F292FBF0F100FB4D
:104F8000123300FB112130313033A170E37004344F
:104F900000232370039BE01A07E6392E03D0013665
:104FA00016709246BAE7524582F800E0B6D0013A50
:104FB000AAE70133C5E70134C3E712F8010C02F890
:104FC0000109BFE708B5044631B1054B03608A6BA0
:104FD0000968002302F02EFD2046FBF7DBF900BF35
:104FE0005CEF01082DE9FF471F460192461882B980
:104FF0000546B5422C4609D22078013509F0DBFB85
:105000000028F6D123782B2B09D12C464FF000082D
:105010000CE0023A222AEBD92D4800F095FB2D2B0B
:105020000ABF2C464FF000084FF00108311B204604
:1050300001AA0AF05BFE0444A1460025B1454B4697
:1050400019D3B8F1000F00D06D426D0045F0010595
:10505000A34209D01C46B442234633D21878013407
:1050600009F0A9FB0028F6D11A491B4802F0A4FC5C
:105070003946FFF7A7FF19F8012BA2F1300ABAF160
:10508000090F07D942F02002A2F161011929D8D8ED
:10509000A2F1570A01998A45D3D2284609F034F87B
:1050A00028B9019B03FB05A595EA4503C6D504A8CD
:1050B000019B40F8044D4246311B03F095FC039BD5
:1050C0000546C5E7D0D1284604B0BDE8F08700BF4B
:1050D00044E7010867E70108A8EE01082DE9F84F49
:1050E0002DED028B0C9F1646984600EB01090546F4
:1050F0004D452C466AD22078013509F05CFB00282A
:10510000F6D123782B2B08D12C4682464D450BD364
:1051100000239E469FED818A56E02D2B03D12C461D
:105120004FF0010AF2E78246237843F02003692B0F
:1051300037D1A31C994540F2E880637843F02003FF
:105140006E2B40F0E280A37843F02003662B40F002
:10515000DC80DFED727AE21DB7EE007A914504F152
:10516000030387EE278A1AD9E27842F02002692ADF
:1051700015D1227942F020026E2A10D1627942F0D4
:105180002002692A0BD1A27942F02002742A06D1AA
:10519000E27942F02002792A01D104F108030026C5
:1051A0007FE06E2B15D025469FED5D7A9FED5B8AE3
:1051B00000232C469E461A46F0EE476AB2EE046A79
:1051C0004FF00A0B4C451AD300265AE04FF0000A64
:1051D000EAE7A31C994540F29880637843F02003E6
:1051E000612B40F09280A37843F020036E2B40F0B7
:1051F0008C80DFED4A7AE31C87EEA78ACFE7207820
:10520000A0F1300CBCF1090F04F1010116D8022AFB
:1052100003D10BFB03C30C46D4E707EE90CA012A67
:10522000F8EEE77A1BBF48EE067A002207EE878A7F
:10523000B0EE678A08BF27EE267AECE71AB92E2867
:1052400003D10122E7E7022A13D040F02002652AA9
:105250000FD1894503D962782B2A04D1A11C494575
:1052600030D00222D7E72D2AFBD1A11C4FF0010E2E
:10527000F5E736B140F020006A280ABF0C46002648
:105280000126BEF1000F00D05B4207EE903AB2EE6D
:10529000040AF8EEE70A0BF0C3FB20EE088A234667
:1052A0002C46BAF1000F01D0B1EE488A9C4209D0D9
:1052B0001C464C4523460CD21878013409F07BFA81
:1052C0000028F6D11749184802F076FB3946FFF757
:1052D00079FEF7D14EB19FED110AF0EE480ABDEC10
:1052E000028BBDE8F84F01F077BDB8F1000F04D094
:1052F000DFED0A0AB0EE480AF1E7B0EE480ABDEC6D
:10530000028BBDE8F84F02F073BCBAF1000FD9D0A0
:10531000234600269FED018AC6E700BF000000007B
:10532000CDCCCC3D82E70108A8EE010808B51020DD
:1053300008F08AFF0278012161F30202027008BDC1
:105340000278416010B5022464F302020270028800
:10535000029C836064F3C902028010BD10B504464C
:105360000846A3681146626802F0DDFE23889B06AA
:1053700003D5BDE8104002F03FBF10BD38B515465B
:1053800011F480720C4614BF95E806001146FFF731
:10539000E5FF620902F008022A44E1B2BDE83840A4
:1053A00001F0A4BC38B50C4C08F0BEFF04F1380580
:1053B0000023032104F124006363636702F00EF904
:1053C0000121284602F00AF966226E21284602F0E1
:1053D00086F92560656038BD3C2100207047014892
:1053E000704700BFF0060208034B80000A4640F0F9
:1053F0000201186802F073B93C210020034B8100C0
:1054000041F00201186802F074B900BF3C2100208D
:10541000034B80000A4640F00201586802F05FB971
:105420003C210020034B810041F00201586802F04A
:1054300060B900BF3C21002070B51C4693070646AA
:10544000154614D11368104A934202D16B68236049
:1054500070BD0E4A934207D110B101F09EF801468B
:105460006B682360616070BD094A934201D1256079
:1054700070BD5B68A3F18902012A01D96D2BF6D1B9
:1054800084E8600070BD00BFE0FF0108580002081A
:10549000A4FF010800232DE9F041136053600D467D
:1054A0000746144601F079F81D2D064606D1836A99
:1054B00023B1104B84E88800BDE8F081F3692BB17B
:1054C000224629463846BDE8F0411847B06B78B10E
:1054D000A9001A4641F00201043000F016FF38B16D
:1054E0002346426831463846BDE8F041FFF7A4BF85
:1054F000BDE8F0818C0602087FB5800040F0020014
:10550000064B01900491052001A902930393059293
:1055100006F05EFF07B05DF804FB00BF4CFA01081F
:105520002DE9F04389B000AF3A1D04460E46FFF75F
:10553000B1FFBB6833B132462B492C4802F0ECF97D
:10554000FAF728FF7868002849D1204607F07CF850
:105550000028F0D03A1D20461B21FFF79BFF39465B
:10556000786804F01DFE8146304608F0A3FF3A68D3
:10557000551C054405F10E0323F00703ADEB030DA5
:105580006B46DC084FEAC408494640460BF0E5F993
:1055900038682E2300F83430013008EB0004304620
:1055A00008F08DFF8146304608F084FF49460246E8
:1055B00020460BF0D2F92946404608F0EFFE0C4B8E
:1055C0003B61800040F002007B610A4BF860BB61E8
:1055D00007F10C0101230520FB6106F0F9FE2437D9
:1055E000BD46BDE8F08300BFA4E7010878F10108DB
:1055F0004CFA010898EA0108F8B503F0BFFE02F082
:10560000A1F80025064673689D4200D3F8BDB36833
:1056100053F83540EF0074B1042C0CD0A408204698
:1056200008F04DFF03785F2B05D0B3683B4420465C
:105630005968FFF7D9FE0135E5E7024608B5034989
:10564000034802F069F9FAF7A5FE00BFBAE70108BE
:1056500088F0010808B519B902F050F9FAF79AFE76
:1056600002F0AAF9FAE70C4B800010B540F00204F2
:10567000586800222146043000F047FE48B902462F
:105680002146064800F041FE18B905490548FFF7D4
:10569000E1FF406810BD00BF3C21002078030208F4
:1056A000E8E701084CF001080A4B10B5044609CBA5
:1056B000984207D0A100002241F00201043000F01E
:1056C00024FE20B92046BDE81040FFF7CCBF40685B
:1056D00010BD00BF3C21002010B51446FFF7DAFED4
:1056E00023681BB902490348FFF7B4FF10BD00BF90
:1056F000F9E70108F0F1010807B56A46FFF7ECFF8A
:105700009DE8030011B903B05DF804FB01F09AFABB
:10571000F9E773B504460D46164600F03EFFC3692F
:1057200043B104228DE8440029466A462046984742
:10573000009B1BB102490348FFF78CFF02B070BD0C
:10574000F9E70108F0F10108014608B50148FFF743
:1057500081FF00BFA8EE0108014608B50148FFF728
:1057600079FF00BFE4EE0108032837B505460C4673
:1057700007D1084601F078F9F0B1324C204603B069
:1057800030BDCB072CD54910072827D801A353F8E3
:1057900020F000BF7D570008C1570008DD57000802
:1057A000DD570008B5570008DD5700087D57000891
:1057B000BD5700080029E0D0234CDFE70029DDDADF
:1057C000B1F1404F05D14FF0804003F0E9F80446B5
:1057D000D4E74C42640044F00104CFE7CC43F9E73E
:1057E000062820D101F00303022B0BD0DBB90B6894
:1057F0009A69164B9A4216D1486840B98B68019352
:10580000C8680CE08C08204608F04FFE18B1400034
:1058100040F00104B2E701A9204608F055FE0199C5
:1058200008F072FDF3E7204600F0B7FE436913B9B4
:105830000748FFF791FF214628469847044600286D
:105840009CD1F5E7A0EA010898EA0108D9A100086F
:105850000BE801082DE9F04105460E46174698462B
:1058600000F09BFE04693CB143463A463146284667
:10587000A446BDE8F04160470148FFF76DFF00BF57
:1058800029E8010800231A461946FFF7E3BF2DE96E
:10589000F041174C90B08846616800910646216837
:1058A000019104A862602360FAF750FD054630B10B
:1058B000009B63600598019B2360FAF76BFD3768D6
:1058C0004246314602A8FBF7C6FF2B462A46394618
:1058D00002A8FEF74BFAFFF7D5FF0546FAF752FD8F
:1058E000009B6360019B2360284610B0BDE8F081F7
:1058F0003C21002007B502AB002243F8041D012122
:10590000FFF7A8FF03B05DF804FB07B58DE80600BC
:105910006B4600220221FFF79DFF03B05DF804FBF8
:1059200030B454680034154618BF0124A2EB840338
:1059300008330A462118286830BCFFF78BBFF0B542
:1059400091B01D4606460C46174600F026FE2F4B2A
:10595000984207D12B463A462146304602F058FC81
:1059600011B0F0BD826A2A4B42B19C422CD1304624
:10597000904728600028F3D00120F1E79C4223D112
:1059800001AA1D213046FFF785FD019B63B901AADD
:10599000C9213046FFF7A0FE039401AA002101208F
:1059A000FFF7BEFF2860E7E704A8FAF7CFFC01463F
:1059B00030B901AAFFF7B4FF2860FAF7E3FCDBE790
:1059C000059B2B600220CBE7002CE0D1384600F08D
:1059D000E4FD104906F0E6F801AA68B16C213046F2
:1059E000FFF758FD019B7BB101AA21462046FFF736
:1059F00097FF28602046B3E7DC213046FFF74AFDD9
:105A0000019B0BB10397C8E72F60DBE708F601089D
:105A10004CFA010858F3010810B5044601F0CEFF16
:105A200038B1002320461A461946BDE81040FFF75A
:105A300011BF204601F0D8FF28B904490448BDE849
:105A4000104001F0B9BF204610BD00BF3DE801087D
:105A5000E4EE010873B505460C4600F09EFD124BBE
:105A6000426A9A4206461CD01CB9102008F0E0FB9E
:105A70000446736A4BB96A460E212846FFF70AFDB1
:105A8000009B4BB90948FFF767FE21462846984717
:105A90000028F0D002B070BD2146684602F0AAFC92
:105AA000F8E72846F6E700BF196B000867E8010829
:105AB00037B5054600F071FD846A1CB12846A04741
:105AC00003B030BD6A461D212846FFF7E3FC009B6A
:105AD0002BB16A4621462046FFF722FFF0E7014836
:105AE000FFF73AFE7BE8010830B58FB0054600F0BD
:105AF00054FD846A2CB12846A047044620460FB0C6
:105B000030BD6A461D212846FFF7C4FC009BABB19F
:105B100002A8FAF71BFC014630B96A46FFF700FFFE
:105B20000446FAF72FFCE9E7039B0649186806F0DC
:105B300039F80028E2D10398FAF72CFC0248FFF765
:105B40000BFE00BF30EE01087BE801082DE9F04FA5
:105B50008BB013680293002864D102F10409044653
:105B6000C1F307235FFA81F800935B0008EB03029F
:105B7000019359F822A009EB82025768002F55D0F3
:105B800017F0030552D139688B4A914250D13846FB
:105B900001F0A2FD009B4FEA880B1D18BAF1000F1F
:105BA00048D108F1010000EB4505A80008F040FBD2
:105BB00006460CB10460012406EB84005A464946AF
:105BC0000AF0CBFE4444009B09EB0B01DA0006EB24
:105BD00084000AF0C2FE019B2344984697B117F057
:105BE000030940F0A2803A68734B9A4240F09D80CE
:105BF000384601F0A7FD4D46DFF8C89107467B689F
:105C00009D4276D3A8EB04022146334652080298FF
:105C1000FFF720FE0446304608F036FB20460BB066
:105C2000BDE8F08F02F10809546899E70020B1E758
:105C30002846AFE71AF0030F2BD1DAF800205F49AE
:105C40008A4202D05E498A4223D106AA05A950465B
:105C500000F07AFE059B0133434403EB4505A800A1
:105C600008F0E6FA06460CB1046001245A4649469B
:105C700006EB84000AF071FE059A069908EB040011
:105C8000920006EB80000AF068FE059B43441C442A
:105C900099E708F1040000EB4505A80008F0C8FAF0
:105CA00006460CB1046001245A46494606EB8400BE
:105CB0000AF053FE504606A9FFF7CCFE4444824644
:105CC0004FEA84085046FFF70FFF024600283FF4D2
:105CD0007AAFA54207D8E9003046039208F0C5FA2A
:105CE000039A06466D0046F80820013408F10408BE
:105CF000E8E7BB6853F835004FEAC50A98B10428B5
:105D000011D0830704D103684B4501D104F0B4F9E5
:105D100046F82800BA684FEA880352443344526870
:105D20005A6008F10208013569E706AAA52138463C
:105D3000FFF7D2FC002106AA0846FFF7F1FD00217B
:105D4000FFF788FE4FEA880982465046FFF7CCFEEF
:105D5000834600283FF456AF08F10102954208D867
:105D60006D00042D38BF04253046A90008F07DFAE7
:105D700006461BF0030F08D1DBF80020114B9A42B6
:105D800003D1584604F078F9834606AA0E21384616
:105D9000FFF7A2FC06AA00210120CDF820B0FFF7F2
:105DA000BFFD06EB090346F809B008F10208586088
:105DB00009F10809C9E700BF8CEC010804FF0108DC
:105DC00070F8010824FB0108F0B5830787B00C4682
:105DD00015461BD103681D4A934202D01C4A9342C8
:105DE00014D102AA01A900F0AFFD019B9C421DD86D
:105DF0001CD3029B043D03EB84049C4201D107B0F9
:105E0000F0BD54F8042D45F8042FF6E702A9FFF77A
:105E100021FE0023064601936FF04047019BA342F9
:105E2000304606D3FFF760FE0028E8D00948FFF7A8
:105E30008BFCFFF759FE0028F8D0019BFA1A224488
:105E4000013345F822000193E8E700BF04FF010891
:105E500070F8010892E8010883072DE9F34115461F
:105E6000CFB2C1F3072431D10368364A934202D03E
:105E7000354A93422AD101AA694600F065FD00988F
:105E80003B1983425AD80199002601EB8003A642B0
:105E900011D1BC00C01B2144801B03F0CCF9019937
:105EA00045F8260005EB86080B194246994208D1B1
:105EB00002B0BDE8F08153F8042D45F826200136E4
:105EC000E5E753F8040D42F8040FEFE70021FFF770
:105ED000C1FD002380460093009B9F4218D80021FB
:105EE000084603F0A8F906464046FFF7FDFD0146C7
:105EF000C8B9B1688C4221D845F8246005EB840309
:105F00008800AB4213D1091B304603F0AFF9CFE74D
:105F10004046FFF7E9FD88B1009BFA1A224401339D
:105F200045F82200D7E7304602F020FFDCE7F268B0
:105F3000C71A2A44D25943F8042DE2E70348FFF771
:105F400003FC00BF04FF010870F8010892E8010893
:105F50002DE9F043072885B080460C46164603D14C
:105F6000914210D0A548B4E0022801D005280CD1F8
:105F70003146204600F0A8FB10B1B8F1020FF0E75F
:105F8000B8F1020FEED09E48A3E0082828D11046B1
:105F900001F014FD30B13146204601F02CFD0028FF
:105FA000F1D1DFE716F0030540F003813268954B2D
:105FB0009A4240F0FE8006F1080773689D42D1D2F4
:105FC00057F8048B404601F0F9FC002800F0F180FE
:105FD0004146204601F00FFD0028D4D10135ECE701
:105FE000E10740F1F58012F001074FEA640500F087
:105FF000D1805410212800F2DC80DFE800F0BBBF24
:10600000DAC3C7DADADADA111B1E213A4244465201
:106010005B6D75111B1E213A424446525B6D75A2A1
:1060200045EA0407780090EA070F37D5384602F0B2
:10603000B7FC4EE085EA0407F4E705EA0407F1E758
:10604000002C02DA7048FFF77FFB1F2C09DC6FF091
:10605000404323419D4204DC4FF0404323419D4295
:1060600004DA2846E91702F08BFC5EE005FA04F733
:10607000D8E7002CE6DB1F2CA8BF1F2445FA04F745
:10608000D0E72F19CEE72F1BCCE72146284608F092
:106090003BF80028E5D104FB05F0400040F001008A
:1060A00017E0002C00F0CD802146284608F05DF86E
:1060B0000746B7E7002C00F0C48007EE905AB8EE10
:1060C000E70A07EE904AF8EEE77A80EE270A01F039
:1060D0008FFD05B0BDE8F083002C00F0B2802146B2
:1060E000284608F034F8E3E7002C18DBA946002C1A
:1060F00098D0E20707D54946384608F005F8002849
:10610000AFD109FB07F7012C8CD0494648466410F3
:1061100007F0FAFF0028A4D109FB09F9E7E707EE29
:10612000905AB8EEE70A01F063FD0446204600F0FD
:1061300034FA8369002B3CD03246214640469847CA
:1061400035E0002C7DD00021022004F0A8FF21467C
:106150000646284608F009F8400040F00100B0600B
:106160002146284607F0F3FF400040F00100F060B0
:106170003046AEE7A542FFF606AFF3E6A5423FF78D
:1061800002AFEFE6A5427FF7FEAEEBE6A542BFF613
:10619000FAAEE7E693071BD113681C4A93420AD173
:1061A00007EE905A3146B8EEE70A01F094FD002858
:1061B0008FD1174818E0174A934209D107EE905A39
:1061C0003146DFED150AB8EEE70A00F0DAFEEEE739
:1061D000B8F1060FAAD1304600F0DFF98369054611
:1061E00023B96B6AE3B90D48FFF7B6FA2246314688
:1061F0004046984700287FF46CAFF2E7A0EA010818
:1062000098EA010804FF0108B3E8010850F4010806
:106210000BE801085CEB01080000000067E80108DA
:1062200069463046FFF716FC05462846FFF75CFC3A
:1062300000283FF497AE214600F046FA0028F4D03B
:10624000A1E602490248FFF705FA00BFDFEB0108AB
:1062500068F20108410008B541F00101024801F06F
:1062600051FBFAF797F800BF10F00108014608B596
:106270000148FFF7EFF900BF98EF010810B5044699
:10628000416069B9816023686FF3DF032360DBB28B
:1062900043F0010303F0FD036FF38203237010BD8D
:1062A000C80007F0D1FFA060EDE70368416061F32B
:1062B000DF030360DBB243F00703037082607047C3
:1062C00003789B0710B5044602D4806807F0DCFF12
:1062D0002368002262F3DF036260236010BD03784D
:1062E0009B0710B5044602D4806807F0CDFF2368F1
:1062F000002262F3DF032360DBB243F0010362F3A9
:10630000410362602370A26010BD03782DE9F74F4E
:1063100013F0010804460E4692460ED001F0030227
:10632000022A08D01AB908687E4988423FD0BAF1DB
:10633000010F40F0F5804FF001085B0764D5276836
:10634000A56827F007072F44BD4232D3BAF1010FE9
:1063500040F0E68021686368C1F3DC01994211D105
:1063600004316160A068C90007F07FFF236862689C
:10637000A060C3F3DC03D21AD200002100EBC300FB
:106380000AF00EFB2368A168C3F3DC02501C60F323
:10639000DF03236041F8326006F00306022E01EBB2
:1063A000C20523D023786FF3000323701EE09046CC
:1063B000C3E7286886421DD1BAF1020F16D12368BF
:1063C0006E687A1B083B22F0070205F10801236082
:1063D000083A28460AF0CCFA2368A268C3F3DC0323
:1063E00002EBC305002142F833106E60284603B06B
:1063F000BDE8F08FB8F1000F04D1314600F064F928
:106400000028D9D108359FE7636833B9BAF1010F85
:1064100040F08680204600F087F806F0030BBBF1C1
:10642000020F28D1B00808F040F802466368B2FBBA
:10643000F3F103FB11231F464FF00009A16851F847
:10644000370001EBC705E0B9BAF1010F68D1236845
:10645000C3F3DC02B9F1000F18BF4D46013262F3FD
:10646000DF03BBF1020F23602E606860BED023788B
:1064700060F3000399E731460620FFF775F94210F3
:10648000D4E7042822D1B9F1000F08BFA9466168FA
:106490000137B7FBF1F001FB1077BB42CED1BAF167
:1064A000010F3DD1B9F1000F33D02368002208332A
:1064B000BBF1020F2360C9F80060C9F8042003D0C3
:1064C000237862F3000323704D468FE7864211D193
:1064D000BAF1020F8AD123686268083B0137236052
:1064E000B7FBF2F302FB1377A36853F8373073B9A5
:1064F0002B607BE7B8F1000FC9D131468DE80C0065
:1065000000F0E2F89DE80C000028C0D0E0E704238A
:10651000EEE72046009200F007F86368009A86E7ED
:10652000002563E724FB0108F8B5466819490446CD
:10653000731C002231F81250AB4206D90132222AD4
:10654000F8D103EB530343F00105E800A76807F017
:106550007BFE236865606FF3DF032360DBB243F0EB
:1065600001032370A0600025B54204D13846BDE880
:10657000F84007F089BE57F8351049B1042907D013
:1065800001222046FFF7C1FE07EBC5035B684360AD
:106590000135E9E7C8E801087047C30706D400F0F1
:1065A0000303022B04D000681BB9704701487047F1
:1065B0000148704774F7010824FB010808B5FFF78C
:1065C000ECFFBDE80840406807F079BF10B504460D
:1065D0000846FFF7E2FF83681BB12046BDE8104084
:1065E0001847426802492046BDE81040FAF760BAF1
:1065F00020E901080A4601460148FFF7E7BF00BF4E
:1066000030DA01082DE9F347054608460E4601F049
:10661000EBF9C0B101AA6946304601F047FA009B88
:106620008BB11B49DFF87080DFF87090DFF864A051
:106630002846F9F7D3FE009CE71E04F18044033C92
:10664000A400002F0BDA022231462846FFF7BEFFD6
:1066500010492846F9F7C2FE02B0BDE8F087019A5A
:10666000131941465B6812592846FAF721FA019B33
:1066700023449A6832B951462846F9F7AFFE033FE2
:106680000C3CDEE749462846FAF712FAF7E700BF66
:1066900025E901087111020849E901085EE90108CC
:1066A00008B50246FFF779FF064B0069984204D10E
:1066B0001046BDE8084005F0ADB9003018BF012014
:1066C00008BD00BFB9B90008884210B5044608D11A
:1066D000830744D10368234A934202D0224A93425B
:1066E0003DD1224B9C4201D1002010BD9942FBD0EC
:1066F000E00704D5CA07F7D423460C46194604F030
:106700000302022A01F0030304D082B92068184A68
:1067100090420CD1022B05D0002BE5D10A68144B16
:106720009A42E1D12046BDE8104003F0C3BC022BE1
:10673000DAD01BB90A680E4B9A42D5D02046FFF733
:106740002CFF8369002BCFD00A46022021469847B0
:106750000028C9D0074BC31A5842584110BD012028
:1067600010BD00BF50F401085CEB01084CFA0108B1
:1067700024FB010898EA01080D4A904208B513D09D
:106780000C4A904212D0C10701D5401008BD8207C3
:1067900007D10268084B9A4203D1BDE8084002F0D5
:1067A00042B90648FEF7D8FF002008BD012008BD09
:1067B000A0EA010898EA010874F7010867E90108EE
:1067C000C20705D4830705D10268034B9A4201D161
:1067D00002F022B9FFF7D0BF74F70108114B9842BD
:1067E00010B50C4603D100230B60012010BD0E4BE9
:1067F000984202D10120086010BD10F0010102D0C2
:1068000042102260F1E710F0030307D10168074A44
:10681000914205D102F007F92060E6E7084610BD75
:10682000184610BDA0EA010898EA010874F70108AB
:10683000164A904210B50C461ED0154A90421ED002
:1068400010F0010108D0431000EE103AB8EEC00A73
:1068500084ED000A012010BD10F0030212D103687C
:106860000C498B4202D102F02FFAF1E70A498B4220
:106870000AD101F02DFAEBE79FED080AE8E7B7EE41
:10688000000AE5E7084610BD104610BDA0EA010861
:1068900098EA010874F7010850F4010800000000AC
:1068A00007B501A9FFF7C4FF10B90448FEF754FF6C
:1068B0009DED010A03B05DF804FB00BF7CE901080F
:1068C00070B51B4EB0420D46144603D100230B6039
:1068D000236070BD174EB04204D14FF07E530B6061
:1068E0000023F5E7C60707D5431007EE903AF8EE08
:1068F000E77AC1ED007AF3E7860715D103680E4EFB
:10690000B34204D102F0E0F985ED000AE8E70B4E4E
:10691000B34202D101F0DCF9F6E7094CA34203D1FE
:10692000BDE8704000F028BB0648FEF715FF00BF29
:10693000A0EA010898EA010874F7010850F4010878
:106940005CEB010893E9010810B584070ED10368D8
:10695000084CA34203D1BDE8104004F07FBC064CB4
:10696000A34203D1BDE8104002F07BBC0348FEF710
:10697000F3FE00BF04FF010870F80108ACE901084C
:1069800013B50C4601A9FFF7DFFF019BA34202D01C
:106990000248FEF7D9FE02B010BD00BFC0E90108F1
:1069A00037B51D46D3070C460ED552100192019AF9
:1069B000002A16DA22440192ADB1002A0DDA002332
:1069C0000193019803B030BD01A91046FFF706FFFF
:1069D0000028ECD10848FEF7BFFE9442F1D20194A2
:1069E000EFE7002DF9D1019B002B01DB9C42E8D899
:1069F00002490348FEF72EFEDCE90108B6FE010855
:106A000000F10108820701D001F0CABF002801DAB5
:106A100001F0E0BF400040F00100704700F00303C8
:106A2000022B10B5014609D07BB903680C4A93428A
:106A300002D00C4A934208D1886802E0800807F02F
:106A400039FD400040F0010010BD0846FFF7A5FDEC
:106A500043691BB10520BDE810401847184610BD1A
:106A600024FB0108D0FA010838B5154B98420446BA
:106A700024D0144DA84201D1012038BD124B9842B8
:106A80001CD0C20704D5430814BF0120002038BD24
:106A9000FFF783FD43693BB121460420984718B1B5
:106AA000431B5842584138BD2046FFF7B7FF002826
:106AB000E2D010F1FF3018BF012038BD002038BDF2
:106AC000A0EA010898EA01084CFA010808B5FFF7A6
:106AD000A5FF10B90148FEF73FFE08BDF5E9010822
:106AE00038B505461446FFF758FD036A13B128462A
:106AF000984748B914B90548FEF72EFE042C01D179
:106B00000348F9E70348F7E738BD00BF07EA010883
:106B10002DEA010849EA0108704710B50446FFF75D
:106B20003CFDC36A2BB120469847B0FA80F040097B
:106B300010BD184610BD08B5FFF7EFFF10B90248A9
:106B4000FEF70AFE08BD00BF71EA0108062806BF6D
:106B5000480040F001000020704700BF097949005B
:106B600041F00101FFF7F4B9052805D00979490082
:106B700041F00101FEF7F8BD002070470B7913B119
:106B80000249F9F72BBC0249FBE700BF52DB0108C1
:106B90004CDB010837B50C46114600221D46009219
:106BA0000123204609F0E0F81CB12868FFF75CFFDC
:106BB00010B9024803B030BD0148FBE7A0EA010864
:106BC00098EA01082DE9F84F02EB430BBBF1040FE3
:106BD00000AF8046894615461E460BF101041ED8BB
:106BE000A4000E3424F00704ADEB040DEA460024A3
:106BF00050464FEA8B02B96A40F8049B09F0ADFE9B
:106C0000691C534632464046FEF724FE054614B141
:106C1000204607F039FB2846BD46BDE8F88FA000A6
:106C200007F010FB82460028DAD00446E0E707B5FB
:106C3000009313460A4681684068FFF7C3FF03B01C
:106C40005DF804FB38B505460C200C4607F0F0FA59
:106C5000024A846080E8240038BD00BFE4EA0108ED
:106C60002DE9F0479046826801EB4805044650192B
:106C7000052886B00F46994604F10C0A4FEA8505AF
:106C800018D89200514601A809F067FEA06801AB30
:106C90002A46494603EB800009F05FFEA168606860
:106CA00001AB42463944FEF7D5FD0446204606B006
:106CB000BDE8F087800007F0BBFAA2685146920059
:106CC000064609F04AFEA0682A46494606EB8000BF
:106CD00009F043FEA1686068334642463944FEF736
:106CE000B9FD0446304607F0CFFADFE72DE9F04161
:106CF000CD1CAD00804628460E46174607F098FA90
:106D0000064B8660044680E80801A5F10C0239466E
:106D10000C3009F022FE2046BDE8F08120EB01088E
:106D2000136810B5144633B9BF2905D190ED010A97
:106D300000F05EFF206010BD9229FCD190ED020AA8
:106D4000F6E730B591ED010A87B0B5EE400A0023B1
:106D5000F1EE10FA04460D4600934FF067024FF033
:106D600007034FF0100102A80AD195ED020AFDF7C2
:106D7000FDFE154902AA2046F9F79AFE07B030BD7C
:106D8000FDF7F4FE02AA11492046F9F791FED5ED70
:106D9000027AF5EEC07AF1EE10FA04DAF4EE677AD0
:106DA000F1EE10FA03D00A492046F9F717FB002349
:106DB000009367221021072302A895ED020AFDF730
:106DC000D5FE02AA0349D6E798EB01089CEB01081F
:106DD000A0EB0108A2EB010808B50C202DED028BF9
:106DE000F0EE408AB0EE608A07F022FAC0ED018A28
:106DF00080ED028ABDEC028B014A026008BD00BF33
:106E00005CEB010808B5072805D8DFE800F0052A83
:106E10000404070419360021084608BDD1ED017AA3
:106E2000F5EE407AF1EE10FA35D1D1ED027A1B4B36
:106E30001B49F5EE407AF1EE10FA08BF1946EBE770
:106E4000D1ED017A91ED027AFDEEE77ABDEEC77AD7
:106E500017EE903A17EE101A4B40590041F001011D
:106E6000DAE7D1ED020A91ED010AF1EE600AB1EE26
:106E7000400ABDE80840FFF7AFBF91ED020AD1ED2F
:106E8000017A20EE000A07EEA70A09F091FEBDE89C
:106E9000084000F0ADBE0249BEE700BFA0EA01080D
:106EA00098EA010830B52DED028B85B00C461146ED
:106EB00000221D4600920223204608F055FFF4B13F
:106EC000012C2B6822D09A0742D11968274A914297
:106ED0003ED1D3ED018A93ED028A686883073FD1E2
:106EE0000268224B9A423BD1D0ED027AD0ED010AE2
:106EF00078EEE78A78EE200AB0EE680A03E0DFED6C
:106F00001C0AB0EE600AFFF767FF14E003F003020B
:106F1000022A184604D0AAB91A6816498A420ED124
:106F200003A9184603F03CF90023009301231A46F5
:106F30000399FEF7D3F805B0BDEC028B30BD0B49C9
:106F40008A42F8D01846FFF7ABFCDFED090ADAE712
:106F50001846FFF7A5FC9FED068AF0EE408ABCE7D5
:106F6000FFF79EFC70EE080AC6E700BF5CEB010865
:106F70000000000024FB010843680B608368136075
:106F8000704710B52DED048B82B0044601AA084667
:106F90006946B0EE409AB0EE608AFFF791FCA01E01
:106FA0001E2800F2CE80DFE800F0B7CCCCCCCCCCF1
:106FB000CCCCCCCCCCCC101F5A282BCC69CCCCCC94
:106FC000CCCC101F5A282BCC6900DDED008ADDEDFA
:106FD000017A79EE288A38EE278AF0EE480AB0EE78
:106FE000680AFFF7F9FEA8E0DDED008ADDED017A21
:106FF00079EE688A38EE678AEFE75448FEF7ACFB13
:10700000DDED016ADDED007AF5EE406AF1EE10FA91
:10701000F5EE407A0BD1F1EE10FA03D14C494D4810
:10702000FEF718FBC9EE278A88EE278AD5E7F1EE2E
:1070300010FA06D1B1EE499AC8EE268A89EE268A60
:10704000CBE726EEA67A07EEA77A87EE876AB1EE3F
:10705000477AC6EE877A8DED006ACDED017A9DED17
:10706000017ADDED007A68EE078A59EE278A29EE6B
:10707000079A08EE279AB0EE498AAEE728EE080A8A
:1070800009EE090A09F094FDB5EE400AF1EE10FA96
:107090001BD1DDED017AF5EE407AF1EE10FA12D156
:1070A000DDED007AF5EEC07AF1EE10FA0BDBF5EECD
:1070B000407ADFED297AF1EE10FAF7EE008A18BF78
:1070C000F0EE678A89E72549A9E709F0C1FBF0EEF0
:1070D000490AF0EE408AB0EE480A09F03BFADDEDCD
:1070E000007A9DED017A20EE279A20EE070A08EE3D
:1070F000879A18EEA70A09F0CDFAB0EE408AB0EEF2
:10710000490A09F0BFFA68EE008AB0EE490A09F0B0
:10711000D9FC28EE008A60E7DDED007AF4EE497ACA
:10712000F1EE10FA0FD1DDED017A0D4B0D48F4EEC2
:10713000487AF1EE10FA08BF184602B0BDEC048B95
:1071400010BD0020F9E70748F7E700BFA7EB0108EB
:10715000D7EB010868F2010800000000F0EB01081D
:1071600098EA0108A0EA01080B46D3ED020A93ED64
:10717000010A1146FFF705BF044B0B60044B4B603F
:1071800000238860CB600846704700BF10FA0108F2
:107190008D720008044B0B60037A0B7143688B609F
:1071A0000023CB600846704708EC010810B5044680
:1071B0000C2007F03DF8034A80E814000222027216
:1071C00010BD00BF44EC010808B50430FFF787F894
:1071D000004808BD4CFA0108042803D0052809D04E
:1071E000002070474B68074833F00703064B08BF81
:1071F000184670474868C0F3DC00400040F00100CA
:10720000704700BF98EA0108A0EA010870B5064679
:107210000C4603C904301546FFF777F808B14368F8
:107220008BB9022E07D1022D0BD16168084800F0FE
:1072300069FBF9F7AFF8A368012D00D14360184648
:1072400070BD044BF8E7022D04BF00224260F6E750
:10725000C4F001084CFA01080122D7E70222D5E761
:107260000022D3E70B6870B586680446DA00B342A3
:1072700001D3002070BDE568A818AD5801330DB1E9
:10728000042D01D10832F2E70B6070BD08B500F1A2
:107290000C018068FFF7E6FF00B1006808BD13B578
:1072A000044600F10C018068FFF7DCFF60B1237930
:1072B000012B0BD0022B0BD0036800934368019382
:1072C0006946022003F0EBFE02B010BD0068FBE748
:1072D0004068F9E7F0B50B7A164E174F06EB8303BB
:1072E00085B00D460446996FF9F778F813492046A2
:1072F000F9F774F82B7A8DF804306B680293002349
:107300000096039301266846FFF7C9FF054628B992
:107310000B492046F9F762F805B0F0BD1EB93946B1
:107320002046F9F75BF8012229462046FFF74EF97F
:107330000026E8E708EC0108BFED0108BCED0108F4
:10734000C2ED01082DE9F347884602AE1649DFF881
:107350006090DFF860A00446F9F740F8002346F893
:10736000043D012731464046FFF77CFF054630B912
:107370000E492046F9F732F802B0BDE8F0871FB990
:1073800049462046F9F72AF8012229682046FFF7E6
:107390001DF951462046F9F721F801226968204677
:1073A000FFF714F90027DDE7C5ED01086D110208AC
:1073B000BFED0108EC0002082DE9FF470D680C46FF
:1073C000116816460122074600920223C90808F0F8
:1073D000CBFC022F17D1606810F0030324D10268A0
:1073E000D1682D4A91421FD1226890420BD00DF1F5
:1073F000100805F1040948F8043D41466068FFF7AC
:1074000031FF074640B90024043573689C4231D3EC
:10741000224804B0BDE8F087012239684846FEF7EB
:1074200074FF7B684360E8E70021FEF713FB05F17A
:10743000040A81464846FEF757FB0028E3D00021A6
:10744000FEF708FB8046FEF74FFB07464046FEF777
:107450004BFB04464046FEF747FB0FB104B110B1A9
:107460000F48FEF771F9012239465046FEF74DFFED
:107470004460DFE7B36853F83410E70049B10429EA
:1074800007D001222846FEF740FFB3683B445B6803
:1074900043600134B9E700BF977600084CFA010851
:1074A000C7ED010830B585B004A9002441F80C4DA2
:1074B0000546FFF7D7FE18B909490A48FEF7CAF88A
:1074C0006B68083B6B600368029343680393042373
:1074D00080E8180002A9022003F0E1FD05B030BDEC
:1074E000EDED0108C4F001080228F7B50E4611467B
:1074F00009D006282DD10022301DFEF706FFC0B9A5
:10750000154803B0F0BD9307FAD11268134B9A42A5
:10751000F6D173684A68534033F00703F0D102AFE5
:107520000C1D47F8043D39463046FFF79BFE0546E3
:1075300008B90B48E5E7002229682046FEF7E5FE7A
:107540000028DDD041686868FFF7BEF80028EAD15E
:10755000D6E70020D5E700BFA0EA01088CEC0108BF
:1075600098EA010810B40C7A012C05D1062803D141
:1075700049685DF8044BB7E700205DF8044B70479D
:1075800010B504460C2006F053FE034A80E81400B0
:107590000022027210BD00BF44EC010810B5044681
:1075A0000C2006F045FE034A80E814000122027216
:1075B00010BD00BF44EC010810B5002204300C4699
:1075C000FEF7A3FE28B92146034800F09BF9F8F71F
:1075D000E1FE406810BD00BFC4F00108024B40F856
:1075E000043BFEF74BBE00BF8CEC010838B50546E6
:1075F000102006F01DFE29460446FFF7EFFF204647
:1076000038BDF8B50C46054600216068FEF722FA41
:10761000022D064660688CBFA5680B4DFFF7FEF98A
:1076200050B9FFF7E3FF0446071D3046FEF75CFA4A
:10763000014618B92046F8BD4010F2E7012238464D
:10764000FEF763FE4560F0E74CFA010838B50546E1
:107650008068FFF7CBFF2B6803606B684268C3F359
:10766000DC0363F3DF0242602A79037962F30003EB
:107670006FF3410303712B790279C3F3800363F342
:1076800082020271AA68E9680446D200C06809F063
:1076900064F9204638BD2DE9F041804686B00020CF
:1076A0000D4616461F46FFF7A1FF0446C0F80080AE
:1076B00005B96EB13B68019407EB8502314603A81A
:1076C0000293FEF7F2FD03AA01A9681CFFF774FEFE
:1076D000204606B0BDE8F0814068C008704738B564
:1076E0000446154604300122FEF70FFE4560204691
:1076F00038BD13B502220446009001911046694638
:10770000FFF784FD204602B010BD38B50C461AB90B
:10771000FFF7EFFF094838BD042A0CD100220430DE
:10772000FEF7F3FD28B92146054800F0EBF8F8F71D
:1077300031FE406838BDFFF7D2FFEBE74CFA010895
:10774000C4F00108043070472DE9F34100250F46CD
:107750000646114638462A46984600954FF6FF736E
:1077600008F002FB102006F06DFD0F4CA84218BF78
:1077700004462660A5602FB90C4DE560204602B096
:10778000BDE8F081BE1CB600304606F05BFD054644
:107790000028F1D0064BA6F1080280E88800414697
:1077A000083009F0DAF8E8E750210020FCFE010873
:1077B00004FF010810B5013851F8044B03F06FFCC9
:1077C000E060014810BD00BF4CFA0108F8B513068F
:1077D00004460D46164602F07F070AD47B1E012B95
:1077E00007D80B68586806F06AFE01462046F8F78D
:1077F000F5FD022F0DD110492046F8F7EFFDEB689B
:107800000BB15A6872B920460C49BDE8F840F8F748
:10781000E5BD002FF3D03246E9682046BDE8F840C8
:1078200003F0BEBB012AF6D1996820460022BDE8CC
:10783000F840FEF7CBBE00BFEC0002087211020850
:10784000F8B51546826843680F46511999420446B7
:107850000FD30178D9B105F110061E44012231463B
:10786000C06806F00CFD78B96568A3682070013D1A
:10787000ED1AA368E0682A461844394609F06DF805
:10788000A3681D44A560F8BD6660E060F1E75D1E79
:10789000AD1AEEE7C3685A680AB1986870470148A4
:1078A000704700BF4CFA010810B5144612684AB17F
:1078B000252915D161680B4A914211D10022C2805D
:1078C000226010BD5D2902D1C368236010BD02682B
:1078D000054B9A4204D1E32902D1FFF7DBFF206078
:1078E00010BD00BF4CFA010830EE010810B4C468A6
:1078F0001346A44600225DF8044B6047002211465F
:10790000FFF7F4BF07B502AA42F8041D0121FFF7F3
:10791000EDFF03B05DF804FB0EB42DE9F04388B031
:10792000064610200F9D06F08DFC0446284609F0FF
:10793000A3F900F101088146404606F083FC54B9E2
:107940002346224621463046FFF7FEFE08B0BDE83A
:10795000F04303B0704704AF70B9C4F80890E56015
:10796000134B2360A168E06806F0CEFC3B466060E4
:10797000002204940121E6E7012310AA8DF81030BB
:10798000CDF814800B4B07904FF00008294602A851
:1079900003930192CDF818800297F8F757FF069BE2
:1079A000079A02F80380069BA360079BE360D7E772
:1079B00024FB010841780008FFF7AEBF830707D119
:1079C0000268064B9A4203D1C268054B9A4202D024
:1079D000044904F0E7B80120704700BFA4FF010884
:1079E000497700086CEE010808B5FEF7D6FDBDE842
:1079F0000840FFF7E3BF38B504460D46FFF7F4FF34
:107A000018B12046FEF7C9FD044629462046BDE8C8
:107A1000384004F0C7B810B50446FEF7BEFD044B6D
:107A2000C2689A4218BF24690023A36010BD00BF3A
:107A3000497700082DE9F041044616461D460F46D9
:107A4000FEF7ABFD184BC2689A4218BF2469D4F800
:107A50000880B8F1000F14D10C2006F0F3FBA060F1
:107A600068B10323A380A4F80680E388A16801EB32
:107A70008302D81CE08041F8237056609560BDE811
:107A8000F081E388A18802338B42EEDB03310122CF
:107A90008900404606F0F3FB0028F0D0A388A060E0
:107AA0000333A380E1E700BF4977000870B50446BF
:107AB00015460E46FEF771FD064BC2689A4218BF86
:107AC0002469A36813B933602B6070BDE28832600B
:107AD000FAE700BF4977000830B587B00D460023AC
:107AE0000446009367220723102195ED010A02A89E
:107AF000FDF73CF802A92046F8F770FC2E2102A8F9
:107B000009F0A4F868B9652102A809F09FF840B906
:107B10006E2102A809F09AF818B903492046F8F72F
:107B20005DFC07B030BD00BF9CF4010838B5D1ED55
:107B3000000A90ED000A2DED028B05460C4608F078
:107B400011FED5ED007AD4ED000A77EEC07AB5EEDD
:107B5000400AF1EE10FAB0EE408AC7EEA08A1BD1BF
:107B60009FED220A08F081FDB0EE408AF5EE408AD2
:107B7000F1EE10FA27D1D5ED000AD4ED007A9FED91
:107B80001B0AC0EEA70A08F070FD85ED000A84ED1F
:107B9000008ABDEC028B38BDB5EEC00AF1EE10FADA
:107BA000F5EEC00A4CBF01220022F1EE10FA4CBFE4
:107BB000012300239A421EBFF7EE007A30EE208A9E
:107BC00078EEE78AD2E7B0EE680A08F0A9FD78EE11
:107BD000C08AF6EE007AF4EEE78AF1EE10FAC4BF3E
:107BE000F7EE007A30EE270ACFE700BF0000000072
:107BF00008B508202DED028BB0EE408A06F018FB88
:107C000080ED018ABDEC028B014A026008BD00BF15
:107C100050F4010830B585B00C46114600221D46CF
:107C200000920123204608F09FF824B99FED0F0A27
:107C3000FFF7DEFF12E0286800F00303022B04D0F8
:107C40008BB903680A4A93420AD103A902F0A8FA41
:107C5000002300931A460399FDF740FA05B030BDA2
:107C6000044A9342FAD0FEF71BFEE1E70000000051
:107C700024FB010850F4010891ED010A072805D8FA
:107C8000DFE800F0051D0404070410180021084671
:107C90007047B5EE400A0C4B0C49F1EE10FA08BFE4
:107CA0001946F4E7FDEEC07A17EE901A490041F04C
:107CB0000101ECE7B5EEC00AF1EE10FAE7D5B1EE3E
:107CC000400AFFF795BF00BFA0EA010898EA010843
:107CD00090ED010A704730B50C4687B0054603A900
:107CE00020468DED010AFEF7A3FD002800F0B680C6
:107CF000212D00F21781DFE815F0D400E100EE003D
:107D0000FB000801150115011501150115011501EB
:107D100015011501150122002F0036003D004D0010
:107D20005B008B00150115011501150115012200DD
:107D30002F0036003D004D005B008B00BA009DED2A
:107D4000037ADDED017A77EE877ACDED017A9DED4C
:107D5000010AFFF74DFF81E09DED037ADDED017A29
:107D600077EEC77AF1E79DED037ADDED017A67EEF4
:107D7000877AEAE7DDED037AF5EE407AF1EE10FA64
:107D800003D169496948FDF765FC03A901A8FFF71C
:107D9000CDFEDCE7DDED037AF5EE407AF1EE10FA88
:107DA000EFD0DDED016A86EEA77A8DED017ACEE7A0
:107DB000DDED030AF5EE400AF1EE10FAE1D09DED9B
:107DC000010A08F0CFFCB5EE400AF1EE10FA8DED95
:107DD000010A08D1DDED030A9FED550A08F045FCC4
:107DE0008DED010AB3E7DDED037AB5EEC00AF1EEE1
:107DF00010FAF5EEC07A4CBF01220022F1EE10FA23
:107E00004CBF012300239A42A1D030EE270AE7E7B6
:107E1000DDED017AF5EE407AF1EE10FA06D19DED36
:107E2000037AB5EEC07AF1EE10FAAAD4F5EEC07A74
:107E3000F1EE10FA14D59DED030A08F071FCDDEDAA
:107E4000037AB4EE670AF1EE10FA09D02146DFEDAD
:107E5000380A9DED010A2020FFF793F807B030BDE6
:107E6000DDED030A9DED010A08F0DAFDB8E7DDED6E
:107E7000037AF5EE407AF1EE10FA82D003A901A858
:107E8000FFF754FE9DED010AFFF7B2FE9DED030AD8
:107E90000490FFF7ADFE04A90590022003F0FFF85F
:107EA000DCE7DDED037A9DED017A224B2248B4EE4A
:107EB000E77AF1EE10FA58BF1846CFE7DDED037A06
:107EC0009DED017A1B4B1C48B4EEE77AF1EE10FAF7
:107ED000D8BF1846C2E7DDED037A9DED017A164B57
:107EE0001448B4EE677AF1EE10FA08BF1846B5E709
:107EF000DDED037A9DED017A0E4B0F48B4EEE77A83
:107F0000F1EE10FA88BF1846A8E7DDED037A9DED83
:107F1000017A084B0848B4EEE77AF1EE10FAB8BFE0
:107F200018469BE7002099E7DFEB010868F201089B
:107F300000000000A0EA010898EA010891ED010A9A
:107F4000910710B403460AD1146808498C4206D13F
:107F50001146DFED070A5DF8044BFFF712B8114632
:107F600018465DF8044BFFF7B6BE00BF5CEB010896
:107F70000000000013B50023044600930846114694
:107F80001A4607F0F1FE636802B0BDE810401847DA
:107F900037B51C46002300930123054608461146C9
:107FA0001A4607F0E1FE6B68206803B0BDE8304078
:107FB000184737B51C4600230093022305460846A0
:107FC00011461A4607F0D0FE94E803006B6803B030
:107FD000BDE83040184737B51C4600230093032303
:107FE0000546084611461A4607F0BEFE94E807000B
:107FF0006B6803B0BDE8304018472DE9F04F83B0FF
:1080000000AF80468068796092469B4605F01CFF71
:108010000646D8F8080005F021FF05F015FF00EB33
:1080200040008419A4002C2C32D8223424F00704F8
:10803000ADEB040D6D46002452464FF00009DFF809
:1080400070A0C5F800805B467968C5F804902846A2
:1080500005F009FFDAF804302B614946D8F80430FE
:10806000CAF80430284604F0D5FF2B69CAF804305A
:108070008046A8B9AB681E682CB1284606F004F902
:10808000B8F1000F11D130460C37BD46BDE8F08F76
:1080900004F1140006F0D6F805460028CCD1C4E758
:1080A00005EB86063669002CE7D13046F8F772F901
:1080B0003C210020F0B50D46017987B01746828833
:1080C000044601F001011E46C2F34E02C38800912E
:1080D0002846394607F048FE2379DB070CD506EB26
:1080E0008502394603A8FEF7E0F8A36803AA3146E3
:1080F0002846984707B0F0BDA36831462846984700
:10810000F8E708B505F0AAFEBDE8084005F09CBEFA
:1081100008B5806805F0A2FE05F0A0FEBDE80840A5
:108120000430FFF7EEBF2DE9F8430F46914698461D
:108130000646F0B14568F7B1681C0430800006F0CF
:1081400077F80E4B03600E4BC0F808905B684360F5
:108150000446C0F80C802EB1AA0006F108011030C8
:1081600008F0FBFB17B1043544F825702046BDE844
:10817000F8830546DFE72846DFE700BFA0F40108E3
:108180003C2100202DE9F0414568A86898460E463C
:10819000174605F059FE0446A86805F05FFE05F095
:1081A00053FE073400EB40002044800006F040F806
:1081B000084B03606B68436000238560C36004461E
:1081C00043463A463146083005F04DFE2046BDE8AC
:1081D000F08100BF08F6010870B5054688680C46B6
:1081E000FFF796FF2346024602492846BDE8704045
:1081F000F8F75EBCC4F6010810B50446082006F086
:1082000017F8024A80E8140010BD00BF44F60108C8
:108210002DE9F041C56804461F461DB91D6028467A
:10822000BDE8F08103691830834205D1174B9942AC
:1082300003D01748FDF790FA1960164E6368D6F818
:1082400004807360114604F1080004F0E3FE012885
:108250000546C6F8048007D002280CD00023E3604E
:1082600023691B683B60DAE723691A683A60002AD1
:10827000D5D1E260D3E7A368986805F0E5FD04EB8B
:1082800080000023E3608369ECE700BF4CFA01083B
:10829000E2F601083C21002013B501ABFFF7B8FF5F
:1082A00001280DD00228104C0DD0019BA34218D0FC
:1082B000BBB101AA01210D48FFF718FBF8F76AF8D6
:1082C000019802B010BD0198FEF767F9074903F065
:1082D00069FC08B90198F1E70198FFF7DBFA8442DD
:1082E000F8D10020EDE700BF4CFA010830EE01089C
:1082F00008B50B4602280CBF4A688A68186803490B
:10830000FFF7CAFF08B900F043F808BD4CFA0108AE
:1083100008B50022FFF7C0FF08B900F039F808BD22
:1083200000220149B8E700BF4CFA010807B5124A1C
:10833000124901ABFFF76CFF012805D0022807D0D6
:108340000E4803B05DF804FB0D490E48FDF782F9B5
:108350000198FEF722F90C4903F024FC0028EFD124
:108360000198FEF71AF9094903F01CFC0028E7D12F
:108370000198F8F70FF800BF30F401084CFA010833
:1083800018F70108D4EF010858F3010830EE01088E
:1083900008B50248FFF7B2FAF7F7FCFF30EE010824
:1083A00030B58DB005466846F7F7D0FF014680B975
:1083B0002A1D0120FDF7B4FAEB6823F00103023314
:1083C00043F00103EB600446F7F7DCFF20460DB0F5
:1083D00030BD0198054A0368934204D0044A934291
:1083E00001D0F7F7D7FF0024F0E700BF30EE010817
:1083F00000F10108044B0B6003684B6043688B601D
:108400000123CB600846704738F701082DE9F04397
:10841000486885B00E46FEF7AFF9041E02DA002068
:10842000FDF792F9D6F8089040F2A628B9EB0807B4
:108430002146684618BF012706F0D8F8029D22465B
:108440000021284608F0ACFA3068C3070BD42B464D
:108450002246394600F02FFA69460A4801F030FBFF
:1084600005B0BDE8F083042C4FEA6003204628BF26
:108470000420C14514BF221A00222A44394603F0C1
:108480005CFEE9E7D0FA0108F0B50C4685B06068FB
:10849000174F012201A9FEF74EFBA6680299019A27
:1084A00040F2A6239E4205BF01F1FF334FF0FF3596
:1084B00001259B1818BF13460C460020C5F1000E7D
:1084C00014B900F087FA0BE0B8422B4404F1FF34F2
:1084D00008D940F2A620301A18BF012000F0DCF9BC
:1084E00005B0F0BD13F80EC04CEA0020E8E700BF6D
:1084F000FFFF3F0010B52DED028BB0EE408AF7F77D
:108500005BFE012805D116491648FFF755FAF7F723
:1085100041FF10B91448FDF717F918EE103A002B77
:1085200011DA33F0004204D003F1FF43B3F19C4F62
:108530000CD8FDEEC87A17EE900A400040F001001A
:10854000BDEC028B10BDDB0DDB05EFE700F06EF933
:10855000B0EE480A0446043006F020FB2046EFE760
:1085600000F80108A4F2010819F80108F0B585B077
:108570000E46002411461D46009402232246304632
:1085800007F0F2FB002E38D0012E28D12868C3074F
:1085900006D410F0030305D10368194A93420CD1A5
:1085A00005B0F0BD022B14D103A901F0F9FD0023A1
:1085B00003991A46FCF716FDF2E79969114A9142B0
:1085C000F2D0114A934204D1FFF782FBFFF792FFEA
:1085D000E6E7FEF7D1F8400040F00100E0E703A92C
:1085E000286801F0DDFD06466868039FFEF7C4F8C1
:1085F0002346024639463046DCE70120D0E700BF7B
:1086000074F70108D9A1000850F4010838B50A4CE4
:10861000214491F83B40B0FBF4F45BB1631C0325AB
:10862000B3FBF5F510460AB108F026FB03342C44E1
:10863000204438BD1D46F5E774F701082DE9F04FD9
:1086400085B0DF0706468B460192DDF838800F9D26
:108650009DF840A09DF8449041D55C105CD4002763
:108660004B462A4641462020FFF7D0FFDBF800307A
:108670009842024606D9029005F0DAFD029A30606F
:10868000CBF8002033689918002001F8010C002C69
:1086900045D001390846AAF10A0AB4FBF8FE08FBE6
:1086A0001E44092C8CBF5444303400F1FF3B00F8C9
:1086B000014CB9F1000F4BD0BEF1000F34D05B4537
:1086C00032D2A1EB0B04032C06D1A0F1020B5B45C7
:1086D00000F8029C28D2594674465846DDE79F07A9
:1086E0000FD11F68264CA7420BD1CDF84490CDF88E
:1086F00040A00F95CDF8388005B0BDE8F04F00F0F0
:10870000A3B8326800231370019AD6F800B0136042
:10871000584605B0BDE8F08F64422D27A0E7302011
:10872000A1F1020B01F8020CDDB12846039302927D
:1087300008F0A2FA039B029AABEB0000834210D22E
:10874000013D014615F8013F43B9834667B90FE083
:108750005B45E9D2BEF1000FBED1E5E701F8013B70
:10876000F0E72FB19B4503D90BF8017C0BF1FF3BE0
:1087700033681A44A2EB0B02019B013A1A60C7E767
:1087800074F7010830B58DB01023069300230393CE
:10879000029301930A23054608AC009307AA0B46EF
:1087A00005A806A90594FFF749FF01462846F7F7F3
:1087B00015FE0598A04201D005F066FD0DB030BD54
:1087C0001346144A934230B40C4603D1012230BC04
:1087D000FDF7BEBB104A934201D10322F7E71C28E4
:1087E00015D103F00302022A0DD082B91A680B4991
:1087F0008A4208D00A498A4205D00A498A4202D0F0
:1088000009498A4203D1224619461C20DFE700208D
:1088100030BC7047A0EA010898EA010824FB01086F
:10882000D0FA010804FF010870F8010810B5102003
:1088300005F0FEFC034B044640F8043B06F039F912
:10884000204610BD74F701082DE9F74304469DF852
:10885000346098680F4691461D460B9A0A99334634
:108860000001FFF7D3FE3B689842804604D905F02B
:10887000DFFC2060C7F800802468019400969DF812
:1088800030300B9A0A99281D07F06CF8C9F80000DF
:10889000204603B0BDE8F083F8B50E4617460546FE
:1088A000FFF7C4FF3B46044632462946043006F033
:1088B00022FA2046F8BD2DE9F04105460E4617463E
:1088C0001C460021184608F06BF823463A4631460C
:1088D000281DBDE8F04106F0EABF034610F0010094
:1088E00006D05B10002B0DDB14BF01200020704769
:1088F0009A684AB11B7913F0010F14BF4FF0FF3093
:10890000012070474FF0FF30704738B50C460728FC
:1089100005D8DFE800F005151E0407040E26002424
:10892000204638BD89681448144C002908BF044605
:10893000F6E7081D06F077FF400040F00104EFE77E
:10894000FFF774FF211D0546043006F033FA2C466C
:10895000E6E7FFF76BFF211D0546043006F039FA04
:10896000F5E70B79DB07DBD5FFF760FF211D054637
:10897000043006F014FAEAE7A0EA010898EA0108D0
:10898000D3B50F460646FFF751FF01230446009377
:1089900032463B46043006F0D5F8204602B0D0BD42
:1089A000430093EA000F02D5C117FFF7E9BF43F078
:1089B00001007047D3B50F460646FFF737FF002387
:1089C0000446009332463B46043006F0BBF820468E
:1089D00002B0D0BD10F0404F02D00021FFF7EABF37
:1089E000400040F0010070472DE9F34104460E4677
:1089F00017469846FFF71AFF3B460546CDF800801C
:108A000032462168043006F026F9236818442060B5
:108A1000284602B0BDE8F081C30702D4043006F056
:108A200002BF40107047C30707B503D5401003B01D
:108A30005DF804FB01A9043006F008FF08B10198B5
:108A4000F5E702490248FCF705FE00BF32F80108CD
:108A5000A4F201082DE9F0412DED028B11F0010384
:108A600088B007460C46904625D04B10022201A93B
:108A700002A806F055F802AE18F0010F25D04FEA13
:108A80006803022201A902A806F04AF802AD1E2FCF
:108A900001D0122F46D16B68002B70D0304606F003
:108AA00042FF2846B0EE408A06F03DFF88EE000AFD
:108AB000FFF79EF82BE011F0030040F0F0800A6809
:108AC000784B9A4223D10E1DD6E718F0030F23D11D
:108AD000D8F80030734A934202D108F10405D6E772
:108AE000714A934207D1304606F01DFF4146384691
:108AF000FFF7F1F80BE06D4A93420DD1304606F0D6
:108B000012FF4146DFED6A0A3846FEF73AFA08B02E
:108B1000BDEC028BBDE8F081424621463846FFF7A6
:108B20004FFEF4E7082F40F28C80FFF77FFEA7F19D
:108B300009030446172B71D8DFE803F043493D4F82
:108B40004F0C13191F70326443493D4F4F0C1319DA
:108B50001F7032642A463146043006F02BFA204654
:108B6000D5E72A463146043006F05CFAF7E72A4694
:108B70003146043006F0F1FBF1E76B681BB94D4953
:108B80004D48FCF767FD05A805F093FF2B463246DC
:108B900005A9201D06F09EFC05A805F098FFDEE75C
:108BA0006B68002BEBD005A805F083FF2B463246FF
:108BB000211D05A8EEE72A463146043006F072FA78
:108BC000CDE72A463146043006F0E7FAC7E72A46E1
:108BD0003146043006F055FBC1E74046FFF723FF5E
:108BE000021E02DA3548FCF7AFFD182F314604F1BA
:108BF000040001D00C2F02D106F024F9AFE706F0F3
:108C000084F9ACE76B681BB12B78DB073FF56BAFE2
:108C10002A463146201D06F01EFCA0E76B68002B9B
:108C2000ADD0FFF703FE211D07462B463246043028
:108C300006F050FC05A902200597069402F02FFAD1
:108C400065E72946304606F08AF8042F27D8DFE882
:108C500007F0030A1F111800194B1A4A32EA2000C4
:108C600028BF184653E7164B164A0028D4BF1046B3
:108C700018464CE7124B134A0028CCBF1046184642
:108C800045E70F4B0F4A12EA200038BF18463EE76F
:108C90000B4B0C4A002814BF1046184637E700203B
:108CA00035E700BF74F7010850F401085CEB0108D8
:108CB00000000000DFEB010868F20108B3E80108DA
:108CC00098EA0108A0EA0108043006F02CBE00BFB3
:108CD000042803D0052808D0002070478A68054B77
:108CE0000548002A08BF184670478868400040F0D1
:108CF00001007047A0EA010898EA0108044B0B60E4
:108D0000044B4B6000238860CB600846704700BF6F
:108D100010FA0108518D0008F0B58268022192FB1B
:108D2000F1F102F180420023013A8B4201DB074856
:108D3000F0BDC468D51A54F8236054F8257044F87F
:108D40002370C468013344F82560EEE74CFA01084B
:108D50008168C3680246886883423FBFC96851F88A
:108D600023000133D36028BF0020704738B50D467B
:108D7000836841688B42044613D3C900C06805F07C
:108D800074FA6268A368E06052006260D21A02F16D
:108D90008042013A01339200002100EB830007F08A
:108DA000FFFDA368E2680348591CA16042F8235004
:108DB00038BD00BF4CFA0108F8B583684C1048BFB5
:108DC000E418054648BF24EAE4749C420C4928BFD5
:108DD0001C461746FFF7CAFFAB68581E03F18043D5
:108DE000013B9B008442A3F10406E96803DB41F8E0
:108DF00024700348F8BD8A59CA5001383346F1E758
:108E00004CFA010838B50025044685601021C06879
:108E100005F02BFA0423E06063601022294607F076
:108E2000BFFD014838BD00BF4CFA01082DE9F84FDD
:108E300080460E4617469946B04501D3BDE8F88FE7
:108E4000A8F1040AFFB9D6F800B035460AF10404C7
:108E5000A54207D92168E7B95A460020FDF778F8FE
:108E600081450ED0043DAC4228D2BFB92A6859468C
:108E70000020FDF76DF88145F4D023682A68226050
:108E80002B60A246E2E731683846FCF733FD8346A3
:108E9000DBE73846FCF72EFD0146DDE7296838465A
:108EA000FCF728FD0246E2E7294640464B463A4693
:108EB000FFF7BCFFD04635462E46BDE72368326833
:108EC00022603360331B9B10A5EB0802013BB3EB20
:108ED000A20F0AF1080AE7DC4B463A4631465046F3
:108EE000FFF7A4FFE8E730B585B002AB0C4601936D
:108EF000104B009304310223013806F046FF23682B
:108F00009968012913D9D8680B4C9DF80C500B4B6C
:108F1000029A01F18041002D08BF2346084C013917
:108F2000A24208BF002200EB8101FFF77FFF044847
:108F300005B030BD60F8010898EA0108A0EA010810
:108F40004CFA010810B40C680B460246A168E068B0
:108F50005DF8044B02F09EBF70B50C680B46A1682B
:108F6000024619B918491948FCF774FB012A18BFC1
:108F70005A68206808BF4FF0FF320023FDF710FD4C
:108F8000A268E3688600013A53F82050A260311DC0
:108F9000121A19449200981907F0EAFCA368E268D3
:108FA000002142F82310616804290BD9B1EB430F6B
:108FB00008D949088900E06805F057F96368E0605E
:108FC0005B086360284670BD78F9010800F101086C
:108FD00007B58DE8030069460220FFF7B3FF694635
:108FE00001900220FFF7B8FF014803B05DF804FBD1
:108FF0004CFA010838B5044608460021FCF72AFD62
:1090000005462846FCF770FD0146204601B938BDEB
:10901000FFF7ACFEF5E70A468168C06802F06EBF54
:10902000F8B50E460E490F4F0546F7F7D7F900245D
:10903000B3689C4205D328460B49BDE8F840F7F7D2
:10904000CDB91CB139462846F7F7C8F9F3680122B3
:1090500053F824102846FDF7B9FA0134E8E700BFB9
:10906000BDED0108BFED01088CF9010870B511F0E4
:10907000030604460D4629D10A68174B9A4225D1AA
:10908000AB68816819444368994210D9043189005A
:10909000C06805F0EAF8AA68A368E06013441A1DE6
:1090A00062603146102200EB830007F079FCE36830
:1090B000AA68A068E968920003EB800007F04DFC05
:1090C000A368AA681344A360044870BD29462046DB
:1090D000FFF790FFF8E700BF70F801084CFA0108AD
:1090E00038B5042904460B4B0360084638BF0420FA
:1090F0006060A16080000D4605F09AF86268E0604B
:10910000521B00EB850092000021BDE8384007F0BB
:1091100047BC00BF70F8010838B50546102005F0BF
:1091200087F829460446FFF7DBFF204638BD0E28A6
:109130007FB503460C46154643D003D8042845D9CD
:1091400000243BE01A281CD01C28F9D103A91046A2
:10915000FDF744FB0028F3D0039B002BBCBF00238A
:1091600003930398A3685843FFF7D6FFC36800939F
:109170000546A268E068039B042102F0DBFD2C4653
:109180001CE012F00303DBD111681B4A9142D7D1D6
:10919000AB68A0681844FFF7BFFFA268E168064605
:1091A0009200C06807F0D9FBA068AA68F368E96874
:1091B000920003EB800007F0D0FB3446204604B059
:1091C00070BD11462046FFF751FFF7E7AA0703D10C
:1091D0002968094A914203D0022BB1D1074CEDE72F
:1091E000AB680093EB68A268E16802F008FE002813
:1091F000F4D0034CE2E700BF70F80108A0EA0108D0
:1092000098EA010873B50D46002411461E460094E5
:1092100001232246284606F0A7FD25B9284602B0BC
:10922000BDE8704078E72046FFF776FF316802B06E
:10923000BDE87040DEE670B50C460546FFF76CFFF2
:1092400024B104EB85052346AB4200D170BD1A1B47
:10925000C16853F8046B8E50F6E7C1688068FFF769
:10926000EABF83680B60C368136070478160704712
:1092700038B50446154600230A4681680068FDF7A4
:109280008FFBE36843F8205038BD37B504460D46E0
:109290003AB9694602208DE83000FFF75DFE0948C3
:1092A0000AE0042A0AD100230A4681680068FDF713
:1092B00077FBE36853F8200003B030BDFFF7D8FF19
:1092C000EDE700BF4CFA010810B5044648680022DB
:1092D0006E210430FDF719F848B1406800F048FFEE
:1092E000024620460349BDE81040F7F7E1BB024AB9
:1092F000F7E700BF00FA01087211020810B5144622
:10930000126840684AB9890041F002010430FCF754
:10931000FCFF08B14368236010BD03799B07FBD4B1
:109320006268890041F002011AB9FEF7E2F90023F0
:10933000F1E7FEF7D4F9FAE7800070B540F00205D6
:10934000012229460B48FCF7E0FF0646406878B941
:10935000082004F06DFF084B036004460120FEF76F
:1093600045F92A4660606E21FEF7B9F9746020461F
:1093700070BD00BF6421002090F90108406870476B
:10938000800010B540F00204002221460548FCF799
:10939000BCFF28B9024621460348FCF7B6FF00B1DE
:1093A000406810BD64210020CCF9010810B50C46BE
:1093B0008100012241F002010248FCF7A6FF44604F
:1093C00010BD00BF64210020436818470149F7F72A
:1093D00005B800BFD40002084A680149F7F768BB26
:1093E000B7E7010810F00302034603D100680749FC
:1093F000884209D013F0010007D132B91868044B34
:10940000C31A58425841704701207047A8EA010822
:1094100074F7010810B50446FFF7E4FF38B9A20756
:1094200006D12068034BC31A5842584110BD012091
:1094300010BD00BF50F40108044B0B60044B4B609F
:1094400000238860CB600846704700BF10FA01080F
:10945000DD9F0008044B0B60044B4B6000238860C9
:10946000CB600846704700BF10FA010871940008ED
:1094700013B50446806800F00303022B11D101A943
:10948000800805F021F8E368019A93423FBFC05C71
:10949000400040F0010001332CBF0020E36002B027
:1094A00010BD83680193C068EDE708B50148FCF77B
:1094B0004BF900BF08FD010801F00303022BF7B5CB
:1094C0000646084609D101A9800804F0FDFF0446BC
:1094D000019B33B9174803B0F0BD8B680193CC688A
:1094E000F6E7154B9E420AD0144B9E4225460DD1FD
:1094F0000027019A2B1B9A420ED85FB9EAE725464E
:10950000F6E715F8010BB0470028E3D0019A2B1BB2
:109510009A42F6D80A48DEE715F8010B05F056F92D
:109520000028E6D015F8010CB0470028D2D001275A
:10953000DFE700BFA0EA01082DE8000841E80008C5
:1095400098EA010801460148B6E700BFB7E70008FE
:1095500001460148B0E700BFCDE7000801460148D9
:10956000AAE700BFE1E7000801460148A4E700BF01
:109570002DE80008014601489EE700BF41E80008C9
:10958000884230B513D20378303B092B0FD8002323
:1095900013600A2510F8014B1368303C05FB0343A8
:1095A0008142136003D00378303B092BF2D930BDE0
:1095B000012A13B50C4613D100F00303022B0BD183
:1095C00001A9800804F080FF019B636042232060B2
:1095D000A360002002B010BD83680193C068F3E768
:1095E00000230B604B604FF0FF338B600120F1E7ED
:1095F0002DE9F74F834608680E46FCF7CEFF8146FB
:109600007068FCF7CAFF814501D001F0A7FC306803
:1096100000F00303022B33D16946800804F054FFA5
:109620000446706800F00303022B2DD101A98008C5
:1096300004F04AFF82460099BBF1020F04EB0108D7
:1096400029D9B268224FBA4223D001234846FDF7F8
:10965000A7F92518BBF1030F09D0F268BA4206D06A
:10966000012300994846FDF79BF904EB0008019B94
:109670009BB10024019AAB1898451AD2600013E000
:1096800083680093C468CCE783680193D0F80CA08A
:10969000D1E72546DEE72546E9E7A8EB05012846A0
:1096A00005F087F80130400040F0010003B0BDE84C
:1096B000F08F5146284607F03DF918B9019B013457
:1096C0001D44D7E7284605F065F80546D2E700BFF8
:1096D0004CFA01082DE9F84F98468F1804460D46BC
:1096E0000B4600229F4217D8002A0CBF27262226AD
:1096F00032462349DFF89890DFF898A0DFF898B059
:109700002046F7F7D5F9AF4210D8324620461C491B
:10971000BDE8F84FF7F7CCB913F8011B272903D0A0
:109720002229DFD12726E3E70122DBE715F8012B09
:10973000964205D1134932462046F7F7B9F9E2E7D8
:109740005C2A04D110492046F6F748FEDBE71F2AC1
:1097500008D97F2A12D0B8F1000F01D0130609D41E
:109760000749E9E70A2A01D10849ECE70D2A01D1A6
:109770005946E8E7092A01D15146E4E74946DBE7C3
:109780003BFD01083AFD01083EFD010841FD0108CD
:109790004AFD010847FD010844FD010801F00303EB
:1097A000022BF7B505461746084606D101A98008E1
:1097B00004F08AFE0646002409E08A680192CE6819
:1097C000002BF8D10C680E4BE31A5C425C41042F6D
:1097D00001D047B944B93346019A0A492846F7F7F8
:1097E00067F903B0F0BD1CB107492846F6F7F6FD4E
:1097F0002346019A31462846FFF76CFFF1E700BF88
:10980000D0FA010851FD01080F1D02082DE9F047AB
:109810009942804691461E46089F14D3002FA1EB23
:109820000301CDBF8A464FF0000A0C46002408EB26
:10983000040532464946284607F07CF820B15445D5
:1098400001D03C44F3E700252846BDE8F0872DE928
:10985000F04F87B08246086802920D460393FCF7EA
:109860009CFE07466868FCF798FE874201D001F02D
:1098700075FB286800F00303022B3AD104A9800885
:1098800004F022FE0446686800F00303022B34D182
:1098900005A9800804F018FE81460499BAF1020F68
:1098A00004EB010830D91E4BAA689A429B4629D086
:1098B00001233846FDF774F82618BAF1030F09D0D2
:1098C000EA685A4506D0012304993846FDF768F83E
:1098D00004EB0008029B00934A46059BA8EB060197
:1098E0003046FFF793FF88B9039BB3B10D48FBF7F0
:1098F0002BFF83680493C468C5E783680593D0F899
:109900000C90CAE72646D8E72646E3E7001B40004E
:1099100040F0010007B0BDE8F08F4FF0FF30F9E7ED
:109920004CFA010856FD0108002301228FE70023AD
:109930004FF0FF328BE701231A4688E701234FF0EF
:10994000FF3284E710B50C4611461A469DF80830E0
:10995000FDF726F8204410BDF8B50746102015463F
:109960000E4604F065FC0446076085607EB129461A
:10997000304604F0C9FC6060681C04F059FC2A46BB
:109980000746E060314606F0E8FF00237B5520469D
:10999000F8BD2DE9F04F89B00C4603901068904651
:1099A000FCF7FBFD012C824642D0D8F80400FCF7FE
:1099B000F4FD824501D001F0D1FAD8F8040000F09E
:1099C0000303022B2FD107A9800804F07DFD02902C
:1099D000079B0493D8F8000000F00303022B2CD15E
:1099E00007A9800804F070FD8346039B079E012BA6
:1099F0004FF0000409BF4FF0FF33012306F1FF359C
:109A000005931CBF05930025A1462746D6B9B9F199
:109A1000000F28D1224BA3F110009A4508BF062061
:109A200009B0BDE8F08F83680793C3680293CFE75E
:109A3000062304931B4B0293CCE783680793D0F86B
:109A40000CB0D2E7012300930BEB050204990298B6
:109A5000FFF7DCFEB0B9B9F1000F17D1039B53B982
:109A6000079C2F46013C621C079BD21B9A4211D1D6
:109A7000D8F80000D4E7039B012B2C4608D02F46D2
:109A80004FF00109059B013E1D44BFE72C46F9E755
:109A90004F46E8E70BEB07015046FFF75DFFBFE7D6
:109AA00024FB01080CFB01080A460146022070E76E
:109AB0000A46014600206CE70A460146012068E795
:109AC000194B984270B506460D460ED14968A868F4
:109AD00004F034FC044640B1284604F0A3FDA40081
:109AE00000232B6044F0020070BD102004F0A0FBA6
:109AF0006968816004460660A86804F005FC69682E
:109B00002B6860600131994209D1AB68E360E1687C
:109B1000A26800238B542046AB602B6070BDA86800
:109B200004F0A3FBE060F2E724FB01082DE9F0411B
:109B30008AB004460191FCF730FD04F00303022BC8
:109B4000064630D102A9A00804F0BEFC0746019ADF
:109B5000364B12F0030F05D112689A4209D03449EE
:109B60008A4206D0DC68314801AB00220121A047BF
:109B7000019004AA03A90198FCF7E6FE00242546FB
:109B8000039B9C4213D3294606A804F02FFD089C92
:109B90000025039B9D4228D306A93046FFF790FF7E
:109BA0000AB0BDE8F081A3680293E768CFE7049BA1
:109BB00053F82400FCF7F1FC86424FEA840802D0F7
:109BC0001C48FBF7C9FD0CB1029B1D44049B53F8D4
:109BD000080000F00303022B05D1800804F06AFCA2
:109BE00005440134CCE78068FAE735B12046029A93
:109BF000394606F0B2FE029B1C44049B53F8250034
:109C000000F00303022B0CD105A9800804F05CFCD2
:109C100001462046059A06F0A0FE059B01351C442E
:109C2000B7E783680593C168F3E700BF70F80108E0
:109C300004FF01086AFD01082DE9F04F04288FB0E8
:109C40000E4615D1C868FCF797FD18B930680FB0FB
:109C5000BDE8F08F40EAE07330680393FCF79DFCA9
:109C600082467068FCF799FC824504D001F076F9D1
:109C70004FF0FF33F0E7B068FCF78FFC8245F5D179
:109C8000306800F00303022B4BD107A9800804F0D1
:109C90001BFC0290706800F00303022B46D108A958
:109CA000800804F011FC0490B06800F00303022B5C
:109CB00041D109A9800804F007FC8346079B089A54
:109CC0009A42C3D80024089B079F002B38D124B1A7
:109CD000099A5946204606F040FE099D4FF00109B9
:109CE000DDF80880039B99450AD04FB1012300930A
:109CF000049A089B39464046FFF788FD034618BB87
:109D000024B13A464146601906F027FEE919002CB5
:109D10003DD1B9F1000F99D00AA804F067FC0C9C62
:109D2000D1E783680793C3680293B3E78368089316
:109D3000C3680493B8E783680993D0F80CB0BDE713
:109D40004FF000094D46CBE7089A02B90133A3EB67
:109D5000080734B13A4641466019059306F0FDFD07
:109D6000059B3D4434B1099A05935946601906F0A4
:109D7000F4FD059B089A079F099903EB0208029BD3
:109D80001F440D44A7EB080709F10109AAE70AA936
:109D90005046FFF795FE5AE72DE9F04101F0030325
:109DA000022B86B080460C4618D101A9A00804F009
:109DB0008BFB0646019902A804F018FC049D374667
:109DC000013D019ABB1B9A420CD82046FCF7E5FBEB
:109DD00002A9FFF775FE06B0BDE8F0818B6801931C
:109DE000CE68E7E717F8010BC04705F8010FE8E771
:109DF00001460148D0E700BF55E800080146014888
:109E0000CAE700BF65E8000870B51C468CB00029A1
:109E100077D0186800F00303022B04D06BBB0568F1
:109E2000394A954229D10239012967D8022B1ED11E
:109E300008A9800804F048FB0546206800F00303E9
:109E4000022B18D1800804F030FB044624B908998D
:109E5000284604F059FA04461020089E04F0E8F958
:109E60002A4B03608660C56044600CB070BD836897
:109E70000893C568E1E74468E8E701293ED8C307CD
:109E80000ED54410214608A804F0B0FB002122465C
:109E90000A9806F085FD08A91C48FFF711FEE4E7C3
:109EA000012201A9FCF739FE28B1029A019917484D
:109EB000FFF752FDD9E72068FCF7B0FD78B9102113
:109EC0000DEB010004F081FB206808A9FBF7C2FD3F
:109ED00004462046FBF708FE20B904A9DCE7411040
:109EE00004A8EFE7FCF748FCFF2802D90848FBF775
:109EF0002BFCC1B204A804F0ECFBEAE70548FBF731
:109F00002BFC0548B1E700BF24FB0108D0FA01088B
:109F1000AFFD0108C8FD010814FB010838B504466F
:109F20000D462AB104F03AFA800040F0020038BD34
:109F300004F004FA0028F7D12A4621460248BDE879
:109F40003840FFF709BD00BF24FB0108F0B589B018
:109F50000D460024074611461E4600940323224660
:109F6000284605F001FF002D34D0012D10D110211D
:109F70000DEB010002AA04F04AFB316802A8224658
:109F8000FCF724FB04A93846FFF79AFD09B0F0BDA1
:109F90003068830714D102680F4B9A4210D144688D
:109FA0008668C56824B93146284604F0ADF90446F0
:109FB000102004F03DF907608660C5604460E5E765
:109FC00004A90122FCF7B7FD002205990498FFF7C8
:109FD000A5FFDBE70620D9E7D0FA010813B5044650
:109FE000806800F00303022B11D101A9800804F05E
:109FF0006BFAE368019A93420DD20122184411468C
:10A00000FFF78CFFE3680133E36002B010BD8368A3
:10A010000193C068EDE70020F7E7F7B504460E4668
:10A020001746FCF7BAFA04F00303022B054615D1D4
:10A03000A00801A904F048FA0446042F18D100230F
:10A04000324601992846FCF7ABFC0A4B9D4209D1E8
:10A05000205C400040F0010003B0F0BDA368019314
:10A06000E468EAE7012211462044FFF757FFF3E7CF
:10A070000020F1E7D0FA010800F00303022B07B536
:10A080000CD101A9800804F01FFA019904F086F9A7
:10A09000800040F0020003B05DF804FB8368019388
:10A0A000C068F2E70A4601460148FFF755BC00BF09
:10A0B000D0FA01082DE9F34100F00308B8F1020FCE
:10A0C00004460D4601F0030616D1022E05D1431AAF
:10A0D0005842584102B0BDE8F081800804F0E5F92B
:10A0E0000746022E0AD1A80804F0DFF947B138B1BB
:10A0F000874205D00020EDE74768F2E76868F5E79A
:10A10000B8F1020F16D1A008694604F0DDF9044643
:10A11000022E13D101A9A80804F0D6F901469DE842
:10A120000C009A42E6D1204606F004FCB0FA80F01A
:10A130004009CFE7A3680093E468E9E7AB680193BF
:10A14000E968ECE708B500F00303022B0CD04BB92B
:10A150000268064B9A4205D18168C068BDE8084094
:10A1600004F01CB900F0FAFE800808BD24FB0108C9
:10A1700000F00303022B07B507D023B903689A69DF
:10A18000064B9A4208D000F0E9FE01A9800804F0CD
:10A190009BF903B05DF804FBC068FAE7D9A1000899
:10A1A00000F00303022B13B50C4607D023B9036854
:10A1B0009A69084B9A4209D000F0D0FE01A98008A4
:10A1C00004F082F9019B236002B010BD8368019303
:10A1D000C068F7E7D9A100082DE9F04F9DB01F280E
:10A1E00004460D46099201F0030640F0C48109AB14
:10A1F0000B9312F003044FF001030C93914608D126
:10A200001368AD4A934207D10BAA0CA9484601F046
:10A2100025F84FF0000904E0A84A934218BF4FF018
:10A2200000090C9B0593022E0B9B079306D10DA9E9
:10A23000A80804F049F90446002309E0AB680D932F
:10A24000EC68002EF8D19E4B2A68D11A4B424B4144
:10A2500010AA102114A8069304F0D9F90D9B002729
:10A2600004EB0308A04505D8059BBB4200F07881AC
:10A2700094481AE02178252904D014A804F029FA7A
:10A280000134EFE7661CB04501D8FFF70EF961789D
:10A29000252904D114A804F01CFA3446F0E7282933
:10A2A0002AD1B9F1000F02D18748FBF755FAA01C5B
:10A2B00001460E4616F8013B292B19D10122091A35
:10A2C000FFF72CFE01464846FDF776F901270546C3
:10A2D0004FF0000B33464FF0200A5E4698451C466F
:10A2E0001AD913F8012B2D2A08D146F00106F5E7FB
:10A2F0008845CAD93146DCE70025E9E72B2A02D197
:10A3000046F00206EAE7202A02D146F00406E5E715
:10A31000232A48D0302A42D00023A0450E9345D8A6
:10A320004FF0FF33A0450F93AFD923782E2B15D1D3
:10A33000601C8045A9D963782A2B52D1059BBB426A
:10A340003AD97B1C0893079B53F82700FCF714FAB3
:10A35000089B0F9002341F46A04596D935B9059B3E
:10A36000BB4229D9079B53F8275001372378672B25
:10A370005ED8652B05D2582B76D03BD8453B022BB7
:10A3800083D82846FCF78CFA0F9B217801930E9B0B
:10A3900000933246534610A8F6F70AFA70E746F0E3
:10A3A000400692469AE74FF0100B97E723782A2B46
:10A3B00010D1059BBB4201D8444876E77B1C08932B
:10A3C000079B53F82700FCF7D7F9089B0E90013440
:10A3D0001F46A5E720460EAA4146FFF7D1F80446DE
:10A3E0009EE71CAA002342F8343D4146FFF7C8F817
:10A3F0000446B1E7632B43D0642B7FF446AFAA0732
:10A4000009D12B68324A934205D12846FDF760FCFA
:10A41000FEF770F805460F9B03938DE840040E9BF2
:10A4200002930A226123294610A8F6F7A4F827E729
:10A43000732B14D8722B64D2692BE0D06F2B7FF46E
:10A4400024AFBBF1000F01D046F404760F9B0393B9
:10A450000E9B02938DE8400461230822E3E7752BED
:10A46000CDD0782B7FF411AF0F9A039246EA0B06FA
:10A470000E9A0292CDF804A00096173B1022D2E764
:10A4800005F00303022B04D043BB2B68114A93420F
:10A4900024D118A92846FFF783FE189A012A0146FD
:10A4A00001D00D4801E70E9B019320230093334612
:10A4B00010A8F5F7A2FFE3E604FF01088CEC010801
:10A4C000D0FA01084AFE0108E2FD0108F9FD010881
:10A4D00050F4010824FB010820FE01082846FEF77D
:10A4E00081FF60B12846FCF747F90E9B01932023BA
:10A4F00000938DF860003346012218A9D8E76B4815
:10A50000D3E612AA102118A804F081F82378722B40
:10A510000CBF0122002208D0069B33B1AB0704D147
:10A520002B6863498B4208BF0422294612A8FCF716
:10A530004DF80F9B199A002BB8BF0F920F990E9BE5
:10A5400001938A424FF02003009328BF0A46334606
:10A550001A9910A8F5F751FF18A804F063F88FE6D0
:10A56000534B069A03F1540014A9002A18BF184649
:10A57000FFF7A6FA1AE00846FCF70FF8022E074686
:10A5800017D112A9A80803F09FFF80461C2C25D1E3
:10A5900014A90998FCF722F940B1149B002B0DDC9B
:10A5A000444DA5F11000AF4208BF06201DB0BDE824
:10A5B000F08FAB681293D5F80C80E7E7129918A8D2
:10A5C000594304F013F81A9B009301214046149B51
:10A5D000129A01F0AFFB18A93846C9E70998FBF7B2
:10A5E000DCFF874216D1099800F00303022B0CD13F
:10A5F00018A9800803F068FF8146189E062C40D0F9
:10A6000018D8042C4AD90020D0E783681893D0F8D2
:10A610000C90F2E7264B9F420AD1012218A9099813
:10A62000FCF77BFA0028C1D0DDF86090199EE5E7C1
:10A6300000F094FC0E2C01D01A2CE4D1129B3BB9F3
:10A640000998FBF7AAFF874202D1099D2846ADE78A
:10A65000002EFBD0129918A8314403F0C7FF129ABC
:10A660001A98414606F079F9129B1A9832464946E3
:10A67000184406F072F918A93846FFF721FA054682
:10A68000E4E7012300934A46334612994046FFF718
:10A69000BDF808B1084889E7084887E700964B46A7
:10A6A000129A4146204601F07BFBF2E739FE010891
:10A6B000D0FA010824FB010898EA0108A0EA010881
:10A6C0002DE9F34705460868DFF838A10C46FBF78B
:10A6D00064FF012D814628D9022D666826D0A06826
:10A6E000FCF74AF8074600210846FEF7A4FD80461D
:10A6F000206800F00303022B1BD16946800803F099
:10A70000E3FE0446009D564525443AD1AC42264618
:10A7100071D23078013404F04EF80028F6D1AE4200
:10A7200069D2002F5ED0B2460AE056464FF0FF379E
:10A73000D9E783680093C468E4E7AA45544607D084
:10A7400054460AF1010A207804F035F80028F4D0C4
:10A75000A21B31464846FFF7FFF801464046FEF788
:10A7600005FBA54247D926460134307804F023F88A
:10A7700010B1AC422646F6D1002FC8BF07F1FF3713
:10A78000CDE73046FBF709FF814501D000F0E6FB3D
:10A7900001A93046FFF704FD019B82469BB918488A
:10A7A000FAF7D2FF2E46321B21464846FFF7D4F86F
:10A7B00001464046FEF7DAFAAE421CD2019C002F59
:10A7C000344400DD013F2646002FEBD0019AB31838
:10A7D0009D42E7D35146304606F0ACF80028E2D05F
:10A7E0000136F1E73146AA1B4846FFF7B5F80146A6
:10A7F0004046FEF7BBFA404602B0BDE8F08700BF16
:10A800007FFE01084CFA01082DE9F04F022885B0BF
:10A8100007460D4604D8FFF753FF05B0BDE8F08F9B
:10A820000868FBF7BAFE814695E8410000F0030393
:10A83000022B0CD102A9800803F046FE8046A868CE
:10A84000FBF79AFF041E07DA29463846E3E78368D8
:10A850000293D0F80C80F2E704F1010A002150467F
:10A86000FEF7E9FC294B9E42054602D12848FBF73A
:10A87000FDFC03A93046FFF793FC039B009013B93E
:10A880002448FAF761FF029F4FEA840B4744039E76
:10A89000BE1B4CB1B04507D8039A0099304606F06C
:10A8A00049F808B3013EF4E7A7EB080241464846E1
:10A8B000EE68FFF751F84FEA840B46F824008CB19C
:10A8C000AAEB0404E868A600324600EB0B0106F090
:10A8D0004FF86A68E868121B92000021304406F0C5
:10A8E0005FF8AC60284698E70399EB680193BA1BC0
:10A8F000521A48463144FFF72FF8019B013C43F8B8
:10A900000B003746ABF1040BC1E700BF4CFA01085E
:10A910008FFE01087FFE01082DE9F341804608689B
:10A920000D46FBF73AFE0746286800F00303022BAA
:10A9300021D16946800803F0C7FD044601A9686873
:10A94000FFF72EFCB8F1020F064618D90123AA68BA
:10A9500000993846FCF724F82044019A009B041B18
:10A9600014449C4203D8314605F0E4FF48B1064840
:10A9700002B0BDE8F08183680093C468DEE720463A
:10A98000EBE70248F4E700BFA0EA010898EA0108F3
:10A9900073B50646086800F00303022B0D460ED17E
:10A9A0006946800803F090FD044601A96868FFF736
:10A9B000F7FB022E014606D90A48FBF757FC8368CD
:10A9C0000093C468F1E7019A009B9A4204D89B1A4D
:10A9D000E01805F0AFFF10B1034802B070BD0348A6
:10A9E000FBE700BF9EFE0108A0EA010898EA010803
:10A9F0002DE9F04F2DED028B95B00C460590914658
:10AA0000102108AA0CA89A4603F001FE9FED778A50
:10AA10004C450AD30CAB0FCB059C84E80F002046B5
:10AA200015B0BDEC028BBDE8F08F21787D290CD1EB
:10AA300004F10108C1453DD961787D293AD10CA8BE
:10AA400003F047FE08F10104E2E77B2904D00CA8DB
:10AA500003F03FFEA046F5E7671CB9452AD96178A7
:10AA60007B2904D10CA803F034FEB846EAE77D291F
:10AA700003D0212901D03A291ED1394600273D466D
:10AA80000B78212B25D0002606E04A45114614D12B
:10AA90004D46002649450DD20B783A2B40F03182C5
:10AAA0004B787D2B01F101082AD0424601234A450B
:10AAB000114618D3FEF7F9FC3A4613787D2B114660
:10AAC00002F1010203D0212B01D03A2BDDD10D463A
:10AAD000D6E74B1C9945EDD94E78A6F17203012BB0
:10AAE000E8D80231D6E712F8010B7B2801D10133F7
:10AAF000DDE77D28DBD1013BD9D14446884602E021
:10AB0000C145D7D9002498F800307D2BD2D1002F31
:10AB100046D000233878069303F062FEE0B9394648
:10AB2000A9428B4606D20B4613F8012B2E2A01D0E0
:10AB30005B2A31D1C91B01223846FFF7EFF9002209
:10AB4000074601462298FBF7E0FB38BB3946284808
:10AB5000FCF7D8FEF5F71EFCDAF80030002BA9DC74
:10AB600006AA29463846FEF70BFD209A069B013AB5
:10AB70009A42834603D81F491F48FAF76BFD0133F9
:10AB8000219A52F823704FF0FF33CAF80030AB45DA
:10AB900014D21A48FBF76AFB1946C1E74768F6E783
:10ABA000DAF80030002B85DB209A013A9342E2D29A
:10ABB0000133219A52F82370CAF8003014BB002EDA
:10ABC00008BF73260AAA102110A803F020FDB6F1D1
:10ABD0007302394618BF01220AA8FBF7F7FC10A937
:10ABE0000748FEF76DFF07460EE000BF0000C842B1
:10ABF000C4F00108B0FE010800F10108C9FE010817
:10AC000024FB0108002EDDD14FF0FF3307930A9398
:10AC1000002C00F0E480229B0293219B0193209B57
:10AC2000009342465346214610A8FFF7E1FE10A8C4
:10AC300003F040FD119A017883188346049300299C
:10AC400000F0B080B04806F001F8002800F0AA80BB
:10AC50009BF8005000260BF1010B9BF800202B2ADB
:10AC600000F0B5802D2A00F0B480202A40F0B38097
:10AC700004240BF1010B9BF80020232A04BF0BF1E5
:10AC8000010B44F010049BF80020302A05D1002D60
:10AC900008BF3D25002E08BF302607AA0499584654
:10ACA000FEF76EFC027803462C2A04BF013344F001
:10ACB00020041A782E2A05D1581C0AAA0499FEF7F6
:10ACC0005FFC034693F800B0BBF1000F0AD0594671
:10ACD0008E48049305F0BAFF049B00287DD093F8BA
:10ACE00000B001331B78002B7FF4E4AE10A803F012
:10ACF00099FC35B93846FEF78DFB00280CBF3C2582
:10AD00003E25002E08BF202614F0060F04D00BF0BD
:10AD1000EF03632B3FF4CEAE3D2D63D05E2D64D0A8
:10AD20003C2D01D144F001043846FEF75BFB88B1AD
:10AD3000BBF1630F00F08A806ED8BBF1470F57D884
:10AD4000BBF1450F06D2BBF1000F6BD0BBF1250F55
:10AD50007FF4B0AE3846FEF75DFB002800F0B3800C
:10AD6000BBF1000F00F0AC80BBF16E0F00F0A880CB
:10AD7000BBF1470F00F29180BBF1450F80F092804C
:10AD8000BBF1250F7FF496AE3846FBF789FD0A9B91
:10AD90000193079B009344F480723346662120EEB2
:10ADA000080A89E09BF800507DB19BF8015065B11D
:10ADB0002946554805F04AFF30B15A469BF80150E4
:10ADC00012F8026B934648E705462E4645E70224F3
:10ADD0004FE700244DE700244DE7834682E7A34672
:10ADE000264687E744F040049EE744F080049BE752
:10ADF000BBF1580F47D0BBF1620F7FF45BAE00236D
:10AE00008DE850000393079B029302226123394689
:10AE100008A8F5F7B0FB15E6BBF1670F0BD8BBF13F
:10AE2000650F97D200230393079B02938DE8500090
:10AE300061230A22EBE7BBF16F0F16D0BBF1780F4D
:10AE400021D0BBF16E0F7FF435AEEBE73846FBF750
:10AE500093FC14A9079B01F8100D012201930096A1
:10AE6000234608A8F5F7C9FAECE5E3064FF000031E
:10AE700048BF44F400740393079B02938DE850008D
:10AE800061230822C3E700230393079B02938DE805
:10AE90005000ABF117031022B9E7ABF16503022BA9
:10AEA0003FF608AE3846FBF7FBFC0A9B0193079B75
:10AEB000009322463346594608A8F5F779FCC1E5C8
:10AEC0004FF0670BEEE73D2D3FF4F4ADBBF1000F03
:10AED00003D0BBF1730F7FF4EDAD10A93846FFF737
:10AEE0005FF90A9B109A0096002BB8BF0A920A9B42
:10AEF0009A4288BF1093079B019301462346109AFC
:10AF0000AFE74FF00008F8E5E6FE0108EBFE0108A8
:10AF100070B50546086800F00303022B8AB00C46A2
:10AF2000164615D104A9800803F0CEFA0146049A0A
:10AF3000029600230A44059306A805AB01940095E8
:10AF4000FFF756FD06A90448FEF7BAFD0AB070BD2A
:10AF500083680493C168EAE724FB010808B5014847
:10AF6000FAF7FAFB1AFD01088168C36802464868CF
:10AF700083423FBF981C013351F82000D36028BFA3
:10AF800000207047044B0B60044B4B60002388602B
:10AF9000CB600846704700BF10FA010869AF00088F
:10AFA0002DE9F0410E461249DFF850800446F5F7CE
:10AFB00015FA06F10807002573689D420BD3012B93
:10AFC00003D10C492046F5F709FA20460A49BDE8A5
:10AFD000F041F5F703BA1DB141462046F5F7FEF9F9
:10AFE000012257F8041B2046FBF7F0FA0135E3E78E
:10AFF00074FF010876FF010816070208BFED01087B
:10B0000010B40C680B460246616804F108005DF854
:10B01000044B00F03FBF0A46083050F8041C00F013
:10B020006DBF0528F8B50D461ED0062808D00428A7
:10B030001DD14A680F4B1048002A08BF1846F8BDBA
:10B040000E4C01F1080700266B689E4203D3600096
:10B0500040F00100F8BD57F8041B0620FAF784FB06
:10B06000013604EB6004EFE748684000F0E7002099
:10B07000F8BD00BFA0EA010898EA0108FCFE01083B
:10B08000042A10B5044608D10A46002303C8FBF77A
:10B0900087FC023054F8200010BD002010BD38B5E8
:10B0A0000D46044690B10230800003F0C1F8084B11
:10B0B00080E818005DB100F10802002355F8231064
:10B0C00042F8041B01339C42F8D138BD014838BD19
:10B0D00004FF0108FCFE0108F0B51C2885B00446F9
:10B0E0000E46154609D80123344F83401F402AD10C
:10B0F000334A1A401AB9DB0641D1002021E0284624
:10B10000FBF74BFA2F4900F04DFD0028F5D06B6896
:10B11000706839461844FFF7C2FF726800F10807EB
:10B12000920006F108010446384605F016FC6A68EC
:10B130007068920005F1080107EB800005F00DFC36
:10B14000204605B0F0BD03A91046FBF747FB0028D9
:10B15000F7D0039B002B10DD706800215843FFF7E8
:10B160009EFF00F10803044600937268039B0421CC
:10B1700006F1080000F0DEFDE2E71348E1E72846AB
:10B18000FBF70BFA114B426A9A4209D028460D4947
:10B1900000F092FD054618B9022CAED10C48D0E75C
:10B1A0006B680093726805F1080306F108012046F8
:10B1B00000F025FE0028F1D00648C2E7000001108B
:10B1C0000040000404FF0108FCFE010885AF0008F0
:10B1D000A0EA010898EA01082DE9F3410C4611465E
:10B1E00000221E4600920123204604F0BDFD74B3E8
:10B1F0003468A30703D12268164B9A4217D0102057
:10B2000003F016F8002105463068FAF723FC002405
:10B21000804604264046FAF767FC074658B92046A0
:10B220002946FFF73CFF0446284603F02DF8204648
:10B2300002B0BDE8F081A64205D8F100284603F02F
:10B2400014F87600054645F824700134E2E7024C14
:10B25000EDE700BF04FF0108FCFE010843680B6036
:10B2600008301060704703F00FB800BFF8B50F4604
:10B27000114C1249124B88421AD0C268A24203D024
:10B28000386001242046F8BD406B98B102689A42AC
:10B29000F1D1466800F1080505EB86060024B542A9
:10B2A000F0D2394655F8040BFFF7E0FF0444F6E707
:10B2B0000024E7E70446E5E7C9B30008701902086F
:10B2C00004FF010810B5C46814B90348FAF744FA3A
:10B2D000A446BDE810406047A40002082DE9F047ED
:10B2E000364F374EDFF8DC8005460C46AB684BB175
:10B2F000E268BA4206D0E35823B1EB6804221A6030
:10B30000BDE8F087A06B08B369688900002241F0AE
:10B3100002010430FAF7F9FF0246B8B12B7C3BB1C9
:10B32000EB68296842680020BDE8F047FAF784B866
:10B33000286838B1E36821498B4203D020498C4208
:10B3400018BF0069EB6852682146EDE72B681BB90E
:10B35000646BA4B9BDE8F0872A7C002AF8D1E268C2
:10B36000BA42F5D0B442F3D01869EA686968FAF7CE
:10B3700091F8EB681B68002BEAD0BDE8F0872368E2
:10B3800043450BD1626802F1804204F10803013A9F
:10B3900003EB82091C464C4503D32468B442A5D173
:10B3A0000AE054F8041BB142F5D02846FFF796FF97
:10B3B000EB681B68002BEED0BDE8F087C9B300082E
:10B3C0007019020804FF01082DE9F0478AB00E4603
:10B3D00001A9154698460746FFF748FF04304FEA93
:10B3E0008009484602F024FF0021044640F8047B0F
:10B3F000FAF744FFA9F11002002104F1100005F052
:10B40000CFFA012E04D1D8F80030042B00F081804F
:10B410000DF10C091C220023069205A80C223946C6
:10B420000393C9F8043005930792CDF820908DF866
:10B430002430FFF753FF0398042828D1019843468E
:10B44000D0F80CA02A463146D04720612046FBF7B1
:10B45000A4F887425DD100231322394605A804933E
:10B460000393079305940692FFF738FF039B002B85
:10B470004FD096BB8DBB294628464A46FAF750FA6C
:10B480000546264B9D4244D02548FAF765F9002829
:10B49000DCD04EB945B90AAB2A4643F8207D0121DC
:10B4A000FAF7D8F90446D1E706EB45040134A400C5
:10B4B000204602F0BDFE221F8246414640F8047B32
:10B4C00005F04BFA53462A46711C0398FAF7C2F965
:10B4D0000446504602F0D8FEB8E706EB45070237AF
:10B4E000BF00384602F0A4FE039B0360049B436048
:10B4F0008146A7F108024146083005F02EFA294698
:10B500004A463046FAF70CFA0546484602F0BCFEB9
:10B51000B7E720460AB0BDE8F08700BF4CFA010843
:10B52000BB000208F0B5146887B016466CB94368D2
:10B530000291596B82680192039404968DF814402D
:10B5400029B9104901A8FFF7C9FE07B0F0BD0A6884
:10B550000D4B9A420ED14F6801F10805BC42F0D064
:10B5600055F8241001A8FFF7B9FE3368002BECD181
:10B570000134F3E701A8FFF7B1FE3368002BE4D1F3
:10B58000DFE700BF7019020804FF01082DE9F04150
:10B590001446126806460F4688B08900043052BB34
:10B5A00041F002052946FAF7B0FE10B14368236066
:10B5B0001EE005908DF81C003168039603A80497DF
:10B5C0000694FFF78BFED4F80080B8F1000F0FD17E
:10B5D0000D2F0DD06A460D213046F9F75BFF009B19
:10B5E00033B16A46414601200295FAF799F9206085
:10B5F00008B0BDE8F08165683DB902221143FAF751
:10B6000084FE0028F4D00023D1E7012241F002019A
:10B61000FAF77BFE4560F6E737B51D460023009339
:10B6200001230446084611461A4604F09DFB0820F3
:10B6300002F0FEFD2A684260046003B030BD37B5F9
:10B640001C460023009302230546084611461A466D
:10B6500004F08AFB0C2002F0EBFD94E80600056084
:10B660004160826003B030BD4A680149F5F720BAF5
:10B67000D900020870B515468AB0142204460E4659
:10B680000DEB020000210091019105F089F92023C2
:10B6900005940793CDF820D085B908232168069337
:10B6A00005A8FFF71BFE02210098042812D12A46A4
:10B6B00031462069FBF714FA0AB070BD042D01D1A0
:10B6C0000E23EBE722232168069305A8FFF706FE69
:10B6D0000321E9E70028EFD002AB00220294039691
:10B6E0000495FAF7B7F8024B042D18BF1846E3E7A4
:10B6F0004CFA01082DE9F041DFF8608088B004467B
:10B700000E461746002518F80430049303A81823A2
:10B71000316800950195029503960593CDF818D0F0
:10B720008DF81C50FFF7DAFD0098042807D13A463F
:10B7300031692046FAF70CFC08B0BDE8F08130B161
:10B740006A46002101200297FAF7EAF8F4E7A4F12B
:10B7500009030B2BF0D80C34E4B2D4E778FF0108CE
:10B7600030B51E4B034489B00C4693F82210049167
:10B770001421002301AA059105462168019303A81D
:10B780000293039406928DF81C30FFF7A7FD0198F1
:10B79000042807D121692846F9F7E6FF0446204628
:10B7A00009B030BD58B12146FAF7A4F8062D044679
:10B7B000F5D1FBF705F8440044F00104EFE7062D4E
:10B7C00001D00024EBE70A232168049303A8FFF7C4
:10B7D00085FD019B002BF4D16400EDE778FF0108A3
:10B7E00038B50D4604460B49F4F7F8FD00226968A8
:10B7F0002046FAF7EBFE08492046F4F7EFFDA9686A
:10B8000020460022FAF7E2FE20460449BDE838400F
:10B81000F4F7E4BDE6000208BFED0108E400020809
:10B8200070B588B00C46002A0CBF23212121049159
:10B83000082100230591064615462168019301AAB7
:10B8400003A802938DF81C3003940692FFF746FD7F
:10B85000019B3BB935B921232168049303A80595C1
:10B86000FFF73CFD0198042819D12069FAF795FEED
:10B87000134BC2689A4210D13DB12368586802F058
:10B880001EFE01463046F4F7A9FD45F0800221690D
:10B890003046FAF79BFE08B070BD2A46F7E728B19C
:10B8A0002146FAF727F800220146F1E72046FAF789
:10B8B00085FE2346024603493046F5F7F9F8EAE7E4
:10B8C00049770008EF00020830B5136887B01446C6
:10B8D00063B90190029103930146012301A80492E8
:10B8E0008DF81430FFF7FAFC07B030BD806B0028EC
:10B8F000FAD05568043089003DB902221143FAF7A5
:10B9000004FD0028F0D02560EEE7012241F002019D
:10B91000FAF7FBFC0028E7D063684360002323604C
:10B92000E2E7F0B589B00E462C2100230390059183
:10B930000546016801931746012401AA03A8029352
:10B940008DF81C3004940692FFF7C8FC019B042B71
:10B9500009D12869FAF721FE3A46C36A28693146B7
:10B96000984709B0F0BD2046FBE7F0B589B001AEBD
:10B970001523002403900493054624230F460168F1
:10B98000019403A87460059306968DF81C40FFF798
:10B99000A5FC019840B1042808D12869FAF7FDFDFB
:10B9A0003946436A2869984709B0F0BD32462146B6
:10B9B0002046F9F7B5FFF7E7F0B58BB01F46052332
:10B9C00006930D46102300210391049105900793DF
:10B9D0008DF8241003AB01680893044605A81646A9
:10B9E000FFF77CFC039810B90948F9F7B5FE042865
:10B9F00007D13B46324629462069F9F72BFF0BB0A9
:10BA0000F0BD009733462A460499FBF7DBF8F6E7CA
:10BA100029E8010800B589B005220492102200230C
:10BA2000039005920168019301AA03A8029306926C
:10BA30008DF81C30FFF752FC0198003018BF012030
:10BA400009B05DF804FBF0B50D4685B001A90746C5
:10BA50001646284602AAFFF701FC019A0299002324
:10BA600093422CD13C2002F0EFFB264B019A80E858
:10BA70008800254B8360254BC360254B0361254B14
:10BA80004361254B8361254BC361254B0362254BE5
:10BA90004362254BC362044642B1029B1968096B9D
:10BAA0000163012A96BF1B6845634363A66303A92C
:10BAB0002046FFF7DBFB01280AD91C4804E051F8B7
:10BAC0002300C06810B91A48F9F746FE0133C7E7EA
:10BAD000A06B002272210430FAF717FC054668B10A
:10BAE000436813F0030209D11B685B68892B05D1F9
:10BAF000031D01210F48FFF78FFD6860204605B048
:10BB0000F0BD00BFA4FF010821B80008C9B30008B8
:10BB1000B9B9000861B70008F5B600088DB500088E
:10BB200075B600086BB9000823B9000825010208A2
:10BB300001010208E0FF010837B50D461C4600234D
:10BB40001146009301220323284604F00DF9012D2C
:10BB500004D0032D08D00948F9F7FEFD206803B092
:10BB6000BDE83040FAF719BD2068FEF7EBFAA2688D
:10BB7000616803B0BDE83040FFF765BF53010208BC
:10BB80001FB5074B01934B6802930A468B680393DA
:10BB9000014601A8F9F7A0FD05B05DF804FB00BF60
:10BBA0001C0002082DE9F041154FDFF858800E46C1
:10BBB000B0421ED010F003031ED10268BA421BD15E
:10BBC000406BB8B103684345F2D1436803F1804349
:10BBD00000F10804013B04EB8305AC42234601D38A
:10BBE0002068E5E7314618680434FFF7DBFF0028DA
:10BBF000F3D00120BDE8F0810020BDE8F08100BF56
:10BC0000A4FF010804FF01082DE9FF418B07074647
:10BC1000019108461AD10B68144A93420ED10123B0
:10BC2000029301AB0393029D039EDFF8548000242E
:10BC3000AC420ED10E4804B0BDE8F0810D4A9342EB
:10BC400004D103AA02A9FFF709FBECE70A48F9F7B8
:10BC500083FD56F82410414505D03846FFF7A2FF72
:10BC600008B90134E4E70548E5E700BFA4FF01088F
:10BC7000A0EA010804FF01086F01020898EA010820
:10BC800070190208820708B503D10268044B9A4272
:10BC900002D00448F9F760FDBDE80840B4E700BFF2
:10BCA000A4FF0108A801020810B50C46FAF775FCBC
:10BCB0002146BDE81040A7E738B50D460446FAF71F
:10BCC0006CFC2946FFF76EFF00B1206938BD00BF4C
:10BCD00070B504460D46FAF760FC2946036A042253
:10BCE0002046BDE87040184770B504460D4616461C
:10BCF000FAF753FC3246036A29462046BDE87040F5
:10BD0000184770B504460D46FAF747FC2946036A02
:10BD100000222046BDE87040184770B50D46044625
:10BD2000FAF73BFC2A46836921460620BDE87040AD
:10BD3000184700002DE9F041069D80461F4602FB92
:10BD400001F60024BC4201D1BDE8F081284632460C
:10BD5000414604F002FE35440134F3E72DE9F04199
:10BD6000884600210846966892E89000FDF763FA3D
:10BD7000002E054611DABC4202DA2846BDE8F08101
:10BD800058F824102846FCF7F1FF3444F3E758F83C
:10BD900024102846FCF7EAFF3444BC42F7DBECE70A
:10BDA00070B5022804461546049E03D1B24207D05E
:10BDB000002070BDA0B1032814D032462E4615468F
:10BDC0001A460B461146AE423246184628BF2A464E
:10BDD00004F0B0FD022C07D1B0FA80F0400970BD2C
:10BDE0000124F0E70424EEE70028E1DB02D1AE42B3
:10BDF00002D0DDD3012070BD012CFBD1D8E72DE9A5
:10BE0000F74F022806461746DDF8308005D1424537
:10BE100009D0002003B0BDE8F08FB0B1032816D0E0
:10BE20004246B84617461A460B461146B845C34621
:10BE30001C4628BFBB460D464FF00009D94508D126
:10BE4000B84522D0E5D30120E4E70126EEE7042639
:10BE5000ECE72B46A2461968DAF800000193FAF7DE
:10BE600033FC04340435019B10B109F10109E5E705
:10BE7000022ECED01A68DAF80010F0B2FAF768F89D
:10BE8000034B1B1A58425841C4E7012EDBD1C0E7CF
:10BE900098EA01082DE9F0478146186817461E46C2
:10BEA0000D46FAF77AFB022F8246D6F8048013D9A2
:10BEB0000123B2682946FAF773FD032F044606D022
:10BEC00029460123F2685046FAF76AFD0546A54265
:10BED00004D80948F9F738FC0024F8E7414659F836
:10BEE0002400FAF7F1FB08B90134F0E7600040F0F4
:10BEF0000100BDE8F08700BFEC0102082DE9F04128
:10BF0000002507460E4690462C46B54204D16000F7
:10BF100040F00100BDE8F081414657F82500FAF7EE
:10BF2000D3FB00B101340135EFE700BF3E2808B56F
:10BF30000E4B03D040280BD03C2806D14239C9B261
:10BF40002F2902D8585C012360B90948F9F7FCFB96
:10BF50000139C9B27029F8D8194491F8300091F923
:10BF6000A130F1E702B1136008BD00BF030202086F
:10BF700015030208512808B540D011D849282FD000
:10BF800007D8422803D0482827D0012806D1885C4A
:10BF900010E04F284BD017D84C2821D0002009E0C2
:10BFA000682817D00AD8642838D066282ED062288E
:10BFB000F4D18856400040F0010008BD6C2803D041
:10BFC000712813D06928E9D151F82200BDE8084052
:10BFD000FCF7E6BC31F91200ECE731F81200E9E7B2
:10BFE00051F82200BDE80840FCF7F4BC01EBC201A7
:10BFF000D1E90001BDE80840FCF7C2BC01EBC20179
:10C00000D1E90001BDE80840FCF7D4BC01EB820196
:10C0100091ED000ABDE80840FBF7EABD01EBC20163
:10C02000D1E9000111F088FA00EE100AF2E751F8A8
:10C03000220008BD2DE9F0431C46C2B9431E1C4432
:10C040004FF0FF35A9B194F900804FEAE8794FEA43
:10C05000D9720023524263EB43030021C5F1000E65
:10C0600081422C4408D110461946BDE8F0830125D1
:10C07000E8E700220023F0E71F0247EA12671602F2
:10C0800014F80E20002332433B430131E8E7F7B5B3
:10C0900005461468174601AA0E46FFF747FF402DD4
:10C0A00005D1019A531E1C44524214403C252318CA
:10C0B0003B602346A5F13E04624262415A2E94BF82
:10C0C00000210121FFF7B6FF4F2E044601D103B036
:10C0D000F0BD532E07D104F0CFFD002201462046CB
:10C0E000FDF71CFFF3E7662E04D100EE100AFBF704
:10C0F0007FFDECE7642E04D111F01EFA00EE100A69
:10C10000F5E75A2E0ED910F1804241F10003002BC1
:10C1100008BFB2F1004F02D2FCF742FCD7E7FCF7B0
:10C120002FFCD4E7002908BFB0F1804F02D2FCF702
:10C1300051FCCCE7FCF73EFCC9E737B502AC05463D
:10C1400044F8043D104629B92A46214604F005FC6E
:10C1500003B030BD2C44501E2D1BEC42F8D014F817
:10C16000013D00F8013FF8E72DE9F04385B01446A2
:10C1700001AA0646884699461D68FFF7D7FE402E5D
:10C18000074605D1019A531E1D44524215403C26D4
:10C19000EB19B8F1640FC9F8003018D0B8F1660F88
:10C1A0000FD0B8F14F0F33D1A6F13E0041424141CB
:10C1B000042F384623462A4628BF0420FFF7BDFF38
:10C1C00035E02046FAF76CFB10EE104AECE720460B
:10C1D000FAF766FB10EE100A10F0C0FEA6F13E0260
:10C1E000CDE902015142514104AB03EB81032A46E0
:10C1F00053F8083C0420FFF7A0FFB6F13E0318BF38
:10C20000012304AA02EB8303043553F8084CCBE75F
:10C21000A3070FD12268134B9A420BD12B46A6F1EC
:10C220003E0569423A4669412046FCF744FB05B0A9
:10C23000BDE8F0832046FAF79FFA042F0446B3D9ED
:10C24000B8F15A0F0CD90028ACBF0021FF212846B5
:10C250003A4604F0A5FB3E2E04BF3B1FED18A3E7B2
:10C260000021F4E774F70108512810B525D010D843
:10C2700048281FD004D8012814D0422812D010BD5D
:10C280004C2803D0502801D0492801D141F8223050
:10C2900010BD68280ED007D864281ED0662813D099
:10C2A0006228F5D18B5410BD6C28EFD0712804D0D2
:10C2B0006928EAE721F8123010BD01EBC2011A46E5
:10C2C000DB17C1E9002310BD07EE903AF8EEE77ADC
:10C2D00001EB8201C1ED007A10BD184601EBC204EA
:10C2E00010F02AFEC4E9000110BD64282DE9F041D8
:10C2F00006460C4617461D4610D0662805D04F2826
:10C3000019D144F82730BDE8F081184601EB8204CA
:10C31000FAF7C6FA84ED000ABDE8F081184601EB91
:10C32000C204FAF7BDFA10EE100A10F017FEC4E9C5
:10C330000001BDE8F08113F0030811D11A680E4B1B
:10C340009A420DD1424601464020FFF7EFFD41469B
:10C3500000FB074302462846BDE8F041FCF7ABBAB4
:10C360002846FAF709FA3A46034621463046BDE820
:10C37000F041FFF779BF00BF74F7010870B50546BB
:10C38000084602F097F9F4F702FF04462846FCF746
:10C39000F5FF0121034602462046BDE87040F9F74B
:10C3A00076BA10B5044602F085F9F3F7B5FF012817
:10C3B0000BD00649204602F096F9204602F07AF9A1
:10C3C000F3F7AAFF022818BF002010BD6803020877
:10C3D0002DE9F04FCBB0032800AFD1F8009009D978
:10C3E000CB68FB60042834D00C69641005D50020AC
:10C3F000F9F7AAF98D4BFB60002407F114014846B8
:10C40000FDF7CEFE0546002C53D0894E6E21706894
:10C41000FBF7D2F88046706800227A210430F9F7E1
:10C4200074FF07F1280106464046FDF7B9FEBA6AD7
:10C43000013C014602442EB9914203D212F8013D5B
:10C440002E2BF9D114F1FF3409D291420AD1794847
:10C45000CEE70024D1E712F8013D2E2BF2D0914215
:10C46000F9D3EFE77E69541A002E3FD1264606F134
:10C470000E0323F00703ADEB030D6B464FEAD30920
:10C480004FEAC9082246404604F067FA7A693AB191
:10C490002E23601C04F839302946404404F05DFA2C
:10C4A0003146404601F07AFF800040F002097E618B
:10C4B00045464846FDF746FEFCF762FF0446C0B11C
:10C4C0002E21284604F0C2FB50B1584BFA689A421C
:10C4D00006D1411B284601F061FFFCF751FF0446DD
:10C4E000204607F59677BD46BDE8F08F0136264415
:10C4F000BDE707F128024FF4807107F1180002F040
:10C500007DF8A2464FF00108A1467B69984505D900
:10C51000464BFA689A4208BF5446E1E708F1010326
:10C520007B6003D015F808302E2B76D14146284683
:10C5300001F034FFFB69B8607BB94246294607F138
:10C54000180002F019F807F11800FFF72AFF8346D8
:10C5500068B939493948F9F77DF82F2107F11800F2
:10C5600002F0BEF8A8EB090205EB0901E7E7B8689D
:10C57000FCF706FF064600283CD1B868FCF7DCFE55
:10C580007A699045064612D1FB681A462C4B9A42AE
:10C590000DD1BBF1010F0DD066226E214068FBF773
:10C5A0009EF807F118013046FFF7E8FE22E0BBF1E4
:10C5B000010FF6D10022F969386AFDF7AFFC1E21A0
:10C5C00002463046F9F7A5F82F2107F11800D7F8F1
:10C5D0001CB002F085F81B4907F1180002F083F83F
:10C5E00007F1180002F066F8F3F796FE022817D05C
:10C5F000C7F81CB054B1A8EB090105EB090001F024
:10C60000CDFE324601462046F9F783F8D7F804906C
:10C61000BAF1000F08BFB2463446D7F8048074E779
:10C6200007F118013046FFF7A9FEE1E74CFA0108CF
:10C630003C210020300302084F03020878F1010872
:10C64000A0EA01086003020807B51E216A46F8F750
:10C6500021FF0098003018BF012003B05DF804FBF3
:10C66000014B5868704700BF3C210020014B1868FF
:10C67000704700BF3C2100202DE9F0431A4D85B0E2
:10C68000804600200C46D5F80090FAF7AFFF2860EE
:10C6900007462068F9F7F6F8B8F1020F0646C5F824
:10C6A00000901FD0A068F9F778FF054663680193F2
:10C6B00004F10801A8F10200FEF7F1FC01AB0290C1
:10C6C0000022032128460397F9F7C4F8074B9E423E
:10C6D000044603D00146304603F0B8FB204605B0BF
:10C6E000BDE8F083024DE1E73C2100204CFA01084F
:10C6F000A4FF010801460720F9F736B801460620D5
:10C70000F9F732B80021F9F7A5B91FB56946F9F76D
:10C71000A1F904462046F9F7E7F910B9044804B036
:10C7200010BDFAF7A1F90028F4D10248F7E700BFDD
:10C7300098EA0108A0EA01081FB56946F9F78AF9E5
:10C7400004462046F9F7D0F910B9044804B010BDEA
:10C75000FAF78AF90028F4D00148F7E7A0EA0108BF
:10C7600098EA010807B5AE2301900022694602202D
:10C770000093FEF7CDFB03B05DF804FB08B5F9F7B5
:10C780008FFF034B034A002814BF1046184608BD0C
:10C79000A0EA010898EA010807B5F9F7EDFFFF28BC
:10C7A0000AD802AB012203F8040D11461846FDF722
:10C7B000B5FB03B05DF804FB0148F8F7C5FF00BF07
:10C7C000FC0602080A4601462120F9F7C1BB0246D1
:10C7D000AA211F20F9F7BCBB0246A6211F20F9F7AA
:10C7E000B7BB30B50B46012885B014BF4C68044672
:10C7F00069461868F9F72EF905462846F9F774F9DD
:10C80000024610B9204605B030BD21461A20F9F77E
:10C810009FFB0446F1E707B501A9FDF7C1FC019BA9
:10C82000012B02D00448F8F797FF0078400040F051
:10C83000010003B05DF804FB180702082DE9FF476B
:10C8400014468146002220468A4640F22A31F9F7F2
:10C850005CFD002205464FF4F5712046F9F755FDC1
:10C86000012304460293039315B368681B4B984257
:10C870001ED002A9FDF794FC0646DCB16068174B98
:10C88000984217D003A9FDF78BFC05460024DFF87A
:10C89000508027464C450FD1002301930093039A03
:10C8A0000F482946F3F7A9FD0C4804B0BDE8F0870E
:10C8B0000C4EE2E70C4DE9E73CB1019700970023ED
:10C8C000029A31464046F3F798FD5AF824100022A8
:10C8D0004046F9F77BFE0134DCE700BF4CFA010863
:10C8E00030DA01087E2202087111020808B5074BF0
:10C8F0009842014607D006480122F9F767FE05492C
:10C900000348F3F76BFD014808BD00BF4CFA01086E
:10C9100030DA01087111020810B586B004466A4683
:10C9200002A8102101F073FE012221466846F9F7A2
:10C930004DFE02A90248FDF7C3F806B010BD00BFC6
:10C9400024FB010810B50C68E2072DED028B30D4F2
:10C95000A30703D12268194B9A422AD001281DD976
:10C960004868F9F709FF08EE100A2046F9F798FF22
:10C97000F8EEC80AF0EE408AB2EE040A04F050F86D
:10C98000B0EE408A28EE800AF3F729FC80EE080A10
:10C99000BDEC028BBDE81040FBF72AB92046F9F741
:10C9A0007FFFF3F71CFCBDEC028BBDE81040FBF7EA
:10C9B000A1BDBDEC028B204610BD00BF74F701087D
:10C9C000012837B50B46144602D90948F8F7C4FECA
:10C9D00008480022C5680121A84702A9224641F85B
:10C9E000040D0120FCF77FFA019803B030BD00BFB1
:10C9F0003007020870F8010813B504460846FDF731
:10CA0000A1FB6A4601462046F8F744FD044B054A5F
:10CA10000098002814BF1046184602B010BD00BF91
:10CA2000A0EA010898EA010837B50228486888BFDB
:10CA30008C680D6898BF0024FDF784FB094A0A4BF7
:10CA40000146002C18BF134628466A4698470098AE
:10CA500020B1019909B1FAF7F5F80446204603B070
:10CA600030BD00BF95540008D956000838B50446BB
:10CA700008461546FDF766FB2A4601462046F8F7AC
:10CA800048FE014838BD00BF4CFA010808B5F9F767
:10CA90000FF820B90248FAF731FFF3F77BFC08BD25
:10CAA00030EE0108022808B505D106C92020BDE8EE
:10CAB0000840F9F74DBA02490248F8F7CBFD00BF2C
:10CAC0005B07020898EF0108F8B50E4618B9264B27
:10CAD0001D68002412E00868830723D10368234AF5
:10CAE00093421CD1FCF74AFC05463068F9F755FD26
:10CAF0001F4BC2689A42ECD13468043400210846C6
:10CB0000FCF799FB07461DB10026AB689E4214D383
:10CB10001CB1002563689D421AD33846F8BD154AFA
:10CB2000934201D0F9F739FD856B002DDDD02A68DD
:10CB3000114B9A4218BF0025D7E7EB6853F836101F
:10CB400021B1042902D03846FCF710F90136DCE7A0
:10CB5000A36853F8351021B1042902D03846FCF7F8
:10CB600005F90135D6E700BF3C21002090F9010806
:10CB7000C9B30008A4FF01088CEC010810B52DED25
:10CB8000028B0446F9F78CFE2046B0EE408AF9F796
:10CB900087FEB4EE408ABDEC028B034B0348F1EEF6
:10CBA00010FA08BF184610BDA0EA010898EA01086B
:10CBB00073B50646F9F774FE0022002300201249DF
:10CBC0008DED010A10F048FB9DED010A04460D466B
:10CBD00010EE100A10F0C2F922462B4610F07AFC33
:10CBE00078B93046F9F75CFE10EE100A10F0B6F98D
:10CBF000224605F1004310F06DFC10B9034802B065
:10CC000070BD0348FBE700BF0000F03FA0EA010849
:10CC100098EA0108D0B52DED028B82B00446F9F7F1
:10CC20003FFE00220023002019498DED010A10F07B
:10CC300013FB9DED010A06460F4610EE100A10F098
:10CC40008DF932463B4610F045FCF0B92046F9F725
:10CC500027FE10EE100A10F081F9324607F100436A
:10CC600010F038FC88B92046F9F71AFE2046B0EEDD
:10CC7000408AF9F715FEB4EE408AF1EE10FA04D1BD
:10CC8000044802B0BDEC028BD0BD0348F9E700BFF9
:10CC90000000F03F98EA0108A0EA010808B5F9F79A
:10CCA000FFFDDFED047ABDE8084020EE270AFAF721
:10CCB0009FBF00BFE02E654208B5F9F7F1FDDFED3B
:10CCC000047ABDE8084020EE270AFAF791BF00BFBA
:10CCD00035FA8E3C08B5F9F7E3FD03F0E7FFBDE850
:10CCE0000840FBF707BC1FB504AC002344F80C3D1B
:10CCF000F9F7D6FD204603F05BFEFAF779FF9DEDCC
:10CD0000010A0290FAF774FF02A903900220FEF7CD
:10CD1000C6F904B010BD10B52DED028B0C46F9F725
:10CD2000BFFD2046B0EE408AF9F726FDB0EE480A76
:10CD300003F050FDBDEC028BBDE81040FAF758BF80
:10CD40001FB504AC002344F80C3DF9F7A9FD2046BB
:10CD500003F027FDFAF74CFF02900198FBF720FE45
:10CD600002A903900220FEF79AF904B010BD08B59D
:10CD7000F9F796FD03F0D4FCBDE80840FBF7BABB19
:10CD800003F0C6BC03F071BC08B5F9F789FD03F0E8
:10CD900042FCBDE80840FBF7ADBBF8B52DED028BBA
:10CDA0000C46F9F77DFDF0EE408AA047B4EE400A4C
:10CDB000F1EE10FAB0EE408A04D0F4EE688AF1EE9B
:10CDC00010FA31D018EE100A10F0C8F8002206460A
:10CDD0000F46002300201A4910F03EFA04460D4683
:10CDE00002460B463046394610F074FB38B92246ED
:10CDF00005F100433046394610F06CFBB8B118EE2F
:10CE0000900A10F0ABF806460F4602460B46204645
:10CE1000294610F05FFB50B9224605F10043304629
:10CE2000394610F057FB10B90648F8F78DFCB0EE04
:10CE3000480ABDEC028BBDE8F840FAF7D9BE00BF46
:10CE40000000F03F3C0902080049A6E781CD000838
:10CE50000049A2E7F105010800499EE7C104010865
:10CE600000499AE7F9030108004996E7890C01088F
:10CE7000004992E7C50A010800498EE785060108C6
:10CE800000498AE795060108004986E7B10B0108C9
:10CE9000F8B52DED048B0D461446F9F701FD284633
:10CEA000F0EE408AF9F7FCFCF0EE400AB0EE409A52
:10CEB000B0EE680AA047B4EE400AF1EE10FAB0EE08
:10CEC000408A09D0F4EE688AF1EE10FA04D1B4EE8B
:10CED000499AF1EE10FA31D018EE100A10F03EF82F
:10CEE000002206460F46002300201A4910F0B4F92C
:10CEF00004460D4602460B463046394610F0EAFA23
:10CF000038B9224605F100433046394610F0E2FABE
:10CF1000B8B118EE900A10F021F806460F46024606
:10CF20000B462046294610F0D5FA50B9224605F1A5
:10CF300000433046394610F0CDFA10B90648F8F7EC
:10CF400003FCB0EE480ABDEC048BBDE8F840FAF7EC
:10CF50004FBE00BF0000F03F3C090208004A97E7BF
:10CF600065070108004A93E785CD0008004A8FE76E
:10CF700055050108004A8BE7210A010838B5054626
:10CF80002DED028B08680C46F9F78AFCB5EEC00A55
:10CF9000F1EE10FA02D81348F8F7D6FB03F058FC6C
:10CFA000012DB0EE408A05D1BDEC028BBDE83840C2
:10CFB000FAF71EBE6068F9F773FCB5EEC00AF1EE31
:10CFC00010FAE8D9B7EE007AB4EE470AF1EE10FA9B
:10CFD00003D105490548F8F73DFB03F039FC88EE1D
:10CFE000000AE1E73C090208DFEB010868F20108EA
:10CFF00010B5064C20B9606F400040F0010010BD34
:10D000000868F9F7B9FB6067014810BD3C210020B2
:10D010004CFA01082DE9F04F0368DFF8F08295B073
:10D0200007469868039100F00FFFFB68021D92000D
:10D03000BC1803F00101013823F003038DF8171029
:10D04000019004F1040B0094069308A8F3F77EF90D
:10D05000002840F09680039B7C68BE68002B00F09F
:10D06000938023785E2B00F08F80039B03901846FB
:10D07000F8F7D2FC8146F3F785F9CDF82490D9F87A
:10D0800000009E49FEF78EFD40B17B6833B11A78EF
:10D09000432A00F08C855E2A00F0E185099B984ABE
:10D0A000934200F08185974A934200F07D853B686A
:10D0B000986800F0D3FE00F0D1FE7B68051D28467D
:10D0C0005C1B00F0C1FE0646284600F0C7FE054680
:10D0D00000F0BAFE8246284600F0C0FE054600F089
:10D0E000B3FE8146284600F0B9FEA31B0478012256
:10D0F00064B919E004F01F059D4200F101004FEAF8
:10D10000541111D804785B1B0A446CB12106F1D587
:10D110004678210104F00F0501F4E0619D4241EAE7
:10D12000060100F10200EDD9534649460998FAF785
:10D1300081FC099A08E0069B5B6803F001038DF807
:10D140001730069B0C3B06939DF81730002BF2D14D
:10D15000069B9B4500F2F98501238DF81730069850
:10D16000069B06995B680068786023F003038A6079
:10D1700043F8042F08A8BB60F3F7E8F800283FF451
:10D180006AAFDDF824907AE7DFF884A17C6022782A
:10D19000A2F11003651C5A2B00F2FA84DFE813F0A9
:10D1A00062020A039C02F804E802F8043D02EF045C
:10D1B000B804DF048F04CE04A704BE047E046D040B
:10D1C00059046004470433042404150404047A0356
:10D1D00049035F033C032F03F804F804F804F80440
:10D1E0002A03E2007800FC03EC03E503D703C9033C
:10D1F000BD03B403F804F804F8048403BA009200F1
:10D20000920073008B0017035B005B00F301E401E5
:10D21000F804F804F804F804F804F804F804F8042E
:10D220001902C401F8042D02D801F804F804AD0174
:10D23000F804980127010501EA007E005A01F8046C
:10D240004D0189013D01FA02CF0282026702B50257
:10D25000A10250020F03069B5B6803F001038DF8E7
:10D260001730069B0C3B2C460693D8F83430002B25
:10D270008CD00023D8F83490C8F83430F3F782F813
:10D28000CDF82490FBE633681F4A934240F099841E
:10D29000043E2C46E9E7079B33602546F3F772F816
:10D2A0009DF81720069B7D601343BE60FB60012044
:10D2B00015B0BDE8F08F00213068F8F7CBFB2C46A5
:10D2C0003060D2E7069AB4F801300C320692069A22
:10D2D0000698E11C0B44136022789DF81730069DD8
:10D2E000402A14BF0022022213433343002243602A
:10D2F0000C468DF81720AA60B7E700BF30EE010892
:10D3000030F4010840F401084CFA01083C210020E7
:10D3100058F301083368C94CA34200F0418513F06B
:10D32000010100F0A8845B10012B00F0FB84324661
:10D3300056F8083C56F8049C46F8084C46F8044C4D
:10D34000002142F8104903200293F8F7E9FA052278
:10D35000029B46F8103C46F80C9C46F8082C083E08
:10D360002C4682E7326856F8043CB26073602C4663
:10D3700008367AE76378022B00F06284002B40F0D5
:10D380006084069B9B4505D900F0BEBC0C3B9B45C9
:10D3900000F2BA8498680028F8D0F8F73DFB81467F
:10D3A000F2F7F0FFCDF8249069E69DF81730A3B1AD
:10D3B000069B5B6803F001038DF81730069B0C3B5E
:10D3C0000693069B9B450BD8069B5B6813F0020FE8
:10D3D000069B40F025840C3B0693069B9B45F3D9A6
:10D3E000F2F7D0FF0020BE6015B0BDE8F08F2C46EC
:10D3F000002514F8013B03F07F021B0602EBC51564
:10D40000F7D4324629463068F8F726FDC5F30723DE
:10D4100053FA85F506EB850627E7EB1C23F003039B
:10D420005C1D19791868C1EB817306EB830604361D
:10D430003246F7F7A3FF306017E7EC1C24F0030433
:10D44000002220681146F7F789FF331D706004340D
:10D450001E460AE7DDF80C90331F0293B9F1000F66
:10D4600000F03184DDF80C9056F8040C4FF0000EFB
:10D470004A46714607ABCDF80CE0F8F760FA012890
:10D480003FF409AF002840F02E84079B6B4A002B25
:10D4900008BF134646F8043CB9F1000F06D05146C8
:10D4A0004846FAF7A8FA00287FF4E8AE029E2C4618
:10D4B000DBE6EC1C24F003043268206856F8041CF8
:10D4C000F7F74CFF331F46F8040C04341E46CCE635
:10D4D0002C46002514F8013B03F07F0202EBC51532
:10D4E0001A06F7D4294605F1804532463068013DD9
:10D4F000F8F76AFC06EB8506B7E6002215F8013B53
:10D5000003F07F01180601EBC212F7D49308C3EBB6
:10D510008373910756F8230040F06D8356F8041981
:10D520002C46FBF723FCA0E62C46002014F8013B18
:10D5300003F07F021B0602EBC010F7D4C0EB807330
:10D5400006EB830604363146FBF775FE30608CE649
:10D55000A6F1080356F8042C316856F8080C2C463E
:10D560001E46FAF7BCF880E6B146314659F80C0B76
:10D57000F8F770FA864200F0AF83002370603360E2
:10D580002C464E4671E6B4F80130A3F5FF437D3BCF
:10D5900023447360E278B26006F108010FE0069B55
:10D5A0005B689C0702F1FF3200F12E83069B5B68EB
:10D5B00003F001038DF81730069B0C3B06935006D1
:10D5C000EDD151F8044C002A40F04583A1F1080642
:10D5D0004BE62C46002014F8013B03F07F0202EBDF
:10D5E000C0101A06F7D4C0EB807306EB830604362E
:10D5F0003146FDF754FD306037E62C46002014F824
:10D60000013B03F07F021D0602EBC010F7D4F9F7CF
:10D61000EDFF331D70601E4627E62C46002214F8ED
:10D62000013B03F07F01180601EBC212F7D493000F
:10D6300043F002037360043617E600BF4CFA01089A
:10D640002C46002114F8013B03F07F02180602EB80
:10D65000C111F7D4354655F8040BF7F761FF706038
:10D660002E4602E6C94B73602C460436FDE52C4677
:10D67000002114F8013B03F07F0202EBC1111A06EE
:10D68000F7D4C8B2CB09421C03F4FF731344C3EBB5
:10D69000837306EB8306C1F307213246F8F740F99E
:10D6A0003060E2E52C46002114F8013B03F07F02D4
:10D6B000180602EBC111F7D4CB0903F4FF7353FA38
:10D6C00081F3C3EB837306EB8306083E32460020EA
:10D6D000F8F73CFA3060C8E5AD4B73602C46043671
:10D6E000C3E52C46002014F8013B03F07F021D0621
:10D6F00002EBC010F7D456F8042C3168F7F7FCFEA3
:10D70000331F46F8040C1E46AFE52C46002114F8E2
:10D71000013B03F07F021B0602EBC111F7D4CB09DA
:10D7200003F4FF7353FA81F3C3EB837306EB8306B1
:10D730000C3E32460120F8F709FA306095E52C4698
:10D74000002214F8013B03F07F011D0601EBC21219
:10D75000F7D4D309D1B203F4FF730B44A6EB8306CD
:10D76000C2F30722331D3068F8F774F830607CE5A7
:10D7700062782C4642F3801214F8013B03F07F01DB
:10D780001D0641EAC212F7D4530043F0010373604F
:10D7900004366AE5EB1C23F003035C1D1979186855
:10D7A000CB4306EB830641F480713246F7F7E6FD82
:10D7B00030605AE5774B73602C46043655E5306887
:10D7C000A6F104092C46F7F717FF4E464DE5B4F8CD
:10D7D0000150BE6056F80C3C0334002B00F08082F0
:10D7E000A6F10C00F8F764F9002840F07C81103EA7
:10D7F0002C443AE5336873602C46043635E52C46F4
:10D80000002014F8013B03F07F021D0602EBC0105C
:10D81000F7D4F7F707FE28E52C46002014F8013B63
:10D8200003F07F021B0602EBC010F7D4F7F7E6FD0A
:10D830001BE5002215F8013B03F07F01180601EB00
:10D84000C212F7D4C2EB8272009951F82230002B39
:10D8500000F09B8200232C4641F8223005E500228F
:10D8600015F8013B03F07F0101EBC2121906F7D452
:10D87000C2EB8274009B53F8240002F0E5FA002802
:10D8800000F08382009B002153F824002C4602F014
:10D89000DDFAEAE456F8082C316856F8040C2C46F8
:10D8A000F9F71EF90C3EE0E4D6F80090324606F196
:10D8B000080548460B21F7F70FFF48462A4609217D
:10D8C000F7F70AFF00212A460846F8F729F8069BD1
:10D8D000B4F801200C330693DDF818C0DDF818E029
:10D8E0009DF81730069903342244CCF8002043F009
:10D8F0000203321D13430022CEF804308DF81720A6
:10D900008A60B0602E46B0E43068B4F80150033449
:10D91000F9F7AAF848B1043EA7E43068B4F801501A
:10D920000334F9F7A1F80028F5D0A5F500452C44FB
:10D930009BE43068B4F80150043E0334F9F794F8DE
:10D9400000287FF492ACA5F500452C448DE43068A6
:10D95000B4F80150043E0334F9F786F800283FF488
:10D9600084ACA5F500452C447FE4B4F80130A3F560
:10D97000FF437D3B1C4478E416E90C00316846F80F
:10D98000081C2C4646F8042C33606EE4A0EA01081B
:10D9900098EA01084CFA0108336856F8042C326002
:10D9A0002C4646F8043C60E42C46002114F8013B68
:10D9B00003F07F021D0602EBC111F7D456F8042CC8
:10D9C00056F80809F7F7A5FE4FE42C46002014F896
:10D9D000013B03F07F021B0602EBC010F7D4316855
:10D9E000043EF7F715FD40E42C46002014F8013BF7
:10D9F00003F07F0202EBC0101A06F7D43168043E30
:10DA0000F7F7F2FC31E42C46002214F8013B03F056
:10DA10007F0101EBC2121906F7D4C2EB8272009BA0
:10DA2000316853F82200043E02F010FA1DE42C463F
:10DA3000002214F8013B03F07F01180601EBC2122B
:10DA4000F7D4C2EB82720099336841F82230043E69
:10DA50000BE4F7F7C4FC331D70602C461E4604E44B
:10DA6000316856F8040C0422F9F73AF8331F46F8E7
:10DA7000040C2C461E46FFF7F8BB2C46002014F879
:10DA8000013B03F07F021D0602EBC010F7D4A6F1A4
:10DA90000801043EFEF774F8FFF7E7BB2C460021AF
:10DAA00014F8013B03F07F021B0602EBC111F7D40F
:10DAB00032463068F7F710FE0436FFF7D6BB2C4627
:10DAC000002214F8013B03F07F011B0601EBC21298
:10DAD000F7D4C2EB8272009B53F8220002F0B4F933
:10DAE000002800F0528170600436FFF7BEBB2C4660
:10DAF000002014F8013B03F07F02190602EBC0106E
:10DB0000F7D4F7F7B0FD331D70601E46FFF7ADBBCD
:10DB1000002373602C460436FFF7A7BB2C46002178
:10DB200014F8013B03F07F0202EBC1111A06F7D48F
:10DB30003068F7F7E1FD3060FFF797BB2C46002017
:10DB400014F8013B03F07F021D0602EBC010F7D46E
:10DB5000F7F7AAFD331D70601E46FFF786BB2C4603
:10DB6000002214F8013B03F07F0101EBC2121906F9
:10DB7000F7D4C2EB8272009B53F82200B0E7EC1C92
:10DB800024F00304043654F8043B3360FFF76DBB04
:10DB9000AF2A23D8A2F180035B0043F00103736036
:10DBA0002C460436FFF761BB1A46FFF7CDBAB3F82F
:10DBB0000110BA6803330B44103A7B60BA60FFF778
:10DBC00044BAD90740F10681C3F34703012BA6F1FC
:10DBD000040100F0A48056F8042CF0E4BF2A6BD9AD
:10DBE000CF2A00F2C080C2F1C0020099336841F828
:10DBF00022302C468FE656F8042C56F808192C468D
:10DC0000F9F76DFDFFF731BB0E460698069B46F807
:10DC1000042B05224A600C3B04680693FFF7B6BA52
:10DC20005B680699069A306823F00306A2F10C039C
:10DC300003227060B2600C6806930836FFF7A6BA3C
:10DC4000043E3068F7F7E8FE8146F2F79BFBCDF81B
:10DC50002490FFF714BAA1F11806FFF706BBBC68C1
:10DC60000998231DBB60F9F715FE60607B680133DE
:10DC70007B60FFF7EAB9736018460291F8F78DFCF4
:10DC8000A6F1080930600299B4604A460320F7F70C
:10DC900047FEF8F7E9FE00285ED0069B46F8084CE0
:10DCA0005B6803F001038DF81730069B0C3B4E4672
:10DCB0002C460693FFF7D9BAC2F1B002009B2C465E
:10DCC00053F822000CE707AB4A46316856F8040CBB
:10DCD000F7F735FEFFF7D3BB4E462C46FFF7C5BA24
:10DCE00056F8080C7EE54A490798F9F784FE0028A3
:10DCF00078D00798F9F7CEFD46F8040CB9F1000F7B
:10DD00007FF4CDABFFF7D2BB42494348F9F754FE4D
:10DD10008146F2F737FBCDF82490FFF7B0B90E46F5
:10DD2000FFF75BBB56F8049C3460746046F8044C03
:10DD3000A6F10C0200210320F7F7F2FD032346F8B9
:10DD40000C9C46F8083CFFF70ABB019B07EB8307D6
:10DD500002207A61FFF7ACBA736846F8083C2C469B
:10DD60004E46FFF782BAD62A2BD9FA2A42D8293250
:10DD7000D0B256F8041C3268F8F7EAF8331F46F8B8
:10DD8000040C2C461E46FFF770BA24492448F9F7C4
:10DD900013FE8146F2F7F6FACDF82490FFF76FB93B
:10DDA000A6F108097360B3604A460021032002937C
:10DDB000F7F7B6FD029B46F8083C2C464E46FFF7A7
:10DDC00054BA3032D0B23168F7F7CEFC2C4630600E
:10DDD000FFF74BBAF2F7D6FAD6F80090CDF82490B8
:10DDE000FFF74DB9F2F7CEFADDF81C90CDF824908C
:10DDF000FFF745B90B490C48F9F7DEFD0446F2F789
:10DE0000C1FA019B07EB830702207C61FFF750BA40
:10DE100030EE0108D4090208D4EF01088C09020889
:10DE20004CF00108B809020898EF010810B5026823
:10DE3000002312F8011B01F07F04090644EAC31312
:10DE4000F7D40260184610BD07B502AB43F8040DC5
:10DE50001846FFF7EBFF03B05DF804FB10F9013B38
:10DE6000002BFBDB70472DE9F04FD0F800A08DB000
:10DE7000984605924368DAF808201344044640F8AF
:10DE8000043F0D46FFF7D2FF83466068FFF7E6FFC9
:10DE9000431C63600346002113F8022B6360C31C1C
:10DEA0004778636083780293031D6360C3780192AF
:10DEB0000BF180420393033A04F11003A36004F1D1
:10DEC000140093000493C318E360049B03F10C0255
:10DED00002F066FD08EB8503029A0893ABEB07039B
:10DEE000A3EB02090693019B09F10406AF4204EB80
:10DEF000860603F0010363D20BB901F02FFFE81B84
:10DF000008EB8701FDF7CBF804EB8909043EC9F85B
:10DF100010003D46049B2033234408EB8505A845AB
:10DF200075D1019B059A03F002031AB9019A1207F1
:10DF300040F1C78003F0FF020792002B6CD00598D8
:10DF4000F9F754FB81463060029BDAF80C80089D9B
:10DF5000FB18089300260BF1FF33059A96425ED119
:10DF6000069D039E0535AD0062190AF10C001146AD
:10DF7000002E7CD1039B02EB8302049B20332344BD
:10DF80009A427CD3019A02F008020192039A043D5E
:10DF9000254408EB870302F10409029A964277D3DD
:10DFA0000CA8666840F8046DFFF740FF064416F8B9
:10DFB000015BFF2D40F0918066600DB0BDE8F08FF1
:10DFC0002BB104EB8909494BC9F81030043E059B7D
:10DFD000002B9FD1019B19079CD4039BFB1A9D42E8
:10DFE0008BD3039A2B1D1344C5F10402DB1B5A4447
:10DFF0000AEB830304EB8202043B04322946B94254
:10E0000088D253F8040F42F8040D0131F7E758F8AD
:10E01000042B43F8042D82E7DDF81C9094E729686F
:10E0200000220898824204D3079ACAB93048F7F709
:10E0300093FB58F82200814210D19A1A04EB820215
:10E04000506930B18A082B492B48F9F765FCF2F783
:10E05000A1F969685161013608357EE70132E0E7D0
:10E060006A6809934846F9F73AFB099BF3E70B689E
:10E0700013B950F826300B60013E043178E752F8AE
:10E08000041B00297FF47CAF9A1A92101B49DBE72E
:10E090002A686AB9019971B15AF8290053F8261013
:10E0A00003930430F8F731F928B14268039B2A60E2
:10E0B0000136043D71E73E44114958F82620920884
:10E0C000C2E7029A0AB10F48B1E7002B3FF468AFEC
:10E0D0000298F9F78BFA306062E7ED435D4404EB98
:10E0E0008505686901F0B4FE686160E7FCFE01081F
:10E0F000230A0208F4090208E4EE01083F0A0208B4
:10E10000710A0208A10A0208002810DD002908DDB2
:10E110006FF0404393FBF1F18842D4BF002001200F
:10E1200070474FF0404393FBF0F0814206E0002936
:10E1300008DD4FF0404393FBF1F18842ACBF002073
:10E14000012070470028FCD06FF04043EBE790FBC4
:10E15000F1F303FB1100002802DA002903DC704709
:10E1600002D0002900DA08447047002806DB0029A5
:10E1700001DACB43184490FBF1F070470029FADB39
:10E18000C1F10103F6E700004968014802F057BCFD
:10E19000940B020808B5024802F051FC014808BD82
:10E1A000A80B02084CFA010808B5024802F047FC27
:10E1B000014808BDB50B02084CFA010837B51C46EA
:10E1C000002300930123084611461A4601F0CCFDB6
:10E1D0002068F8F7D1FA04460146651E094802F0A6
:10E1E0002EFC032D06D9224607490848F9F794FB6F
:10E1F000F2F7D0F8012002F0BFFC054800EBC500A3
:10E2000003B030BDC50B0208D40B0208A8EE01080C
:10E21000C80A020808B5044802F011FC012002F007
:10E22000ABFC024808BD00BFEA0B02084CFA01082B
:10E2300010B5044602F090FD18B914B12046F7F766
:10E24000FCF910BD02F088BD38B50546FFF7F0FFB8
:10E25000044618B915B12846F7F7EFF92A46002108
:10E26000204602F09DFB204638BD10B50C4602F05A
:10E2700079FD18B914B12046F7F7DFF910BD0AB1DE
:10E2800002F070BD1046704702F058BD074B1B6985
:10E290000BB9184670475A68824204D8801A043075
:10E2A00053F8200070471B68F2E700BF3C210020B4
:10E2B00070B5144E336905469868DB68834234466E
:10E2C00015D30230C000FFF7BDFF20B9336998684D
:10E2D0004000F7F7B2F9336903605A68D9689B6860
:10E2E0005B0083600A4400234260C360306123699D
:10E2F000DA68501C0432D86043F822505B68013B56
:10E30000184470BD3C210020014441F2055388426D
:10E3100004D313F0FF0008BF0120704710F8012B51
:10E3200003EB43135340F2E7024B034A1A61002206
:10E330009A6670473C210020F80B02082DE9F84F3F
:10E3400082468946FFF7E0FF134B1C69834614B9E8
:10E350002046BDE8F88FE66804F1100707EB860653
:10E360003D46B54201D32468F1E7A84658F8040BAE
:10E3700003789B450ED1437899450BD14A465146C7
:10E38000023002F0D7FA28B96068ED1B00EBA50057
:10E39000BDE8F88F4546E4E73C2100202DE9F04731
:10E3A00081460E46FFF7CAFF0246002849D1264C97
:10E3B000A06EF51C78B1236FE16E2B448B420AD915
:10E3C0002944FFF75CFF0746C0B90246216FA06EE3
:10E3D000FFF755FFA766A36EC3B9802D2F4638BF40
:10E3E00080273846FFF72EFFA06660B92846FFF762
:10E3F00029FFA06630B92846F7F71FF9E36E2B44D2
:10E40000E366E8E72F460023E7662367D4F87080C9
:10E41000D4F868A03146454448462567FFF774FFA5
:10E420000AEB08070AF8080032467E704946B81C15
:10E430003E4402F092FA0023B3703846BDE8F0473C
:10E4400036E7BDE8F08700BF3C21002010B5044648
:10E4500002F012FC01462046BDE81040FFF79EBFC7
:10E4600038B5054603300C46FFF7E2FE20604570E4
:10E470002068023038BDF8B5871C4178044638461C
:10E48000FFF75CFF064658B9657838462946FFF71E
:10E490003BFF25442070AE702046BDE8F84007E7FA
:10E4A0002046FFF7F1FE3046F8BD08B5FFF7EEFE57
:10E4B000007808BD08B5FFF7E9FE407808BD08B54B
:10E4C000FFF7E4FE023008BD08B5FFF7DFFE437832
:10E4D0000B60023008BDF0B5002404600C601460CD
:10E4E0001C60154CDFF854E024690CB1744504D16C
:10E4F0001968126811441960F0BD0568013505609E
:10E50000E6680D6835440D60E66804F1100505EB1A
:10E510008606B54207D3A56824682E1D1D6805EB45
:10E5200086051D60E1E755F8047B97F801C0176880
:10E53000033767441760ECE73C210020F80B020822
:10E5400038B5446803680C449C42054610D9037BE7
:10E55000DB0703D500210748F7F77CF8103424F0D7
:10E560000704083421468068FFF77FFE2C60A8600E
:10E5700038BD00BFD4EF010870B504460E46114601
:10E580001546FFF7DDFFA06863682A463146184448
:10E5900002F0EEF962682A44626070BD70B54668A8
:10E5A00004468E42354628BF0D460121FFF7C8FFBD
:10E5B000A368681C5919721B184402F0D9F96368E2
:10E5C000A06801336360284470BD38B50446002557
:10E5D000002914BF0846012020606560FFF728FE6F
:10E5E000237BA06065F30003237338BD38B505466F
:10E5F0000C460131FFF7E9FF6C6038BD0023436032
:10E60000037B016043F0010382600373704738B5F8
:10E6100014460546FFF7D9FF014B2560636038BDFE
:10E6200079E50008037BDB0710B5044602D4806857
:10E63000FFF72AFE0023A36010BD38B50546102061
:10E64000FFF7F6FD29460446FFF7BFFF204638BD19
:10E6500010B5044650B1037BDB0702D48068FFF796
:10E6600013FE2046BDE81040FFF70EBE10BD38B5C2
:10E67000037BDB0704460D4603D500210648F6F769
:10E68000E9FF016880682944FFF7EFFD2368A06077
:10E690001D442560184438BDD4EF010850E738B553
:10E6A00004460D46FFF74CFF6368A0681D44656093
:10E6B000184438BD90E80C009A4210B5044602D1C7
:10E6C0000121FFF7D4FFA26863680021D154A0683C
:10E6D00010BD10B50C460121FFF7E1FF047010BD1D
:10E6E000C9B2FFF7F6BF38B5054608460C4602F03A
:10E6F000C3FA214602462846BDE83840FFF73CBF32
:10E7000010B51446FFF74AFF047010BD10B514464B
:10E71000FFF744FF047010BD43688B4234BF0023F1
:10E720005B1A4360704738B5154642688A42044612
:10E730000B460ED929448A4201D8436038BD80680F
:10E74000D21A521B0144184402F012F96268521B9B
:10E75000626038BD0A460021FFF7E5BF07B5044BEC
:10E76000009068460193F2F771F803B05DF804FB7E
:10E7700079E500080EB403B503AA52F8041B019210
:10E78000FFF7ECFF02B05DF804EB03B0704700BF89
:10E7900000787047013070470023814201D8184645
:10E7A000704711F8012D02F0C002802A18BF013312
:10E7B000F3E7084670477F289DBF034B185CC0F302
:10E7C00040000020704700BF531802087F289DBFFB
:10E7D000024B185CC0F3C0000020704753180208B9
:10E7E0007F289DBF024B185CC0F38000002070475B
:10E7F000531802087F289DBF024B185CC0F380109D
:10E8000000207047531802087F2809D8064B1B5C6C
:10E8100013F00C0F06D1A0F15F0358425841704726
:10E820000020704701207047531802087F289DBFC1
:10E83000024B185CC0F30010002070475318020808
:10E840007F289DBF024B185CC0F34010002070472A
:10E850005318020808B50246FFF7E8FF00B120325E
:10E86000104608BD08B50246FFF7EAFF00B1203A9E
:10E87000104608BD3038092884BF20F02000073832
:10E88000704710B501440246E5240020914203D8A8
:10E89000B0FA80F0400910BD12F8013B20B11B0610
:10E8A00011D50138C0B2F1E7BF2B09D9F72B09D830
:10E8B000DB0803F0060344FA03F303F00300E5E783
:10E8C0001B06E3D510BD0020FCE700BF02398142E2
:10E8D0000B4603D31A880239002AF8D00233181ADB
:10E8E0004010704770B51C09944215D2121B01EB01
:10E8F0004401154603F00F030E46012D31F8024B7B
:10E9000018BF3468DC40A4B2013D20F8024BF3D1BB
:10E9100004B9013A104670BD0022FBE7F0B5059C32
:10E920000025121B2E46AC420FD164000519023C93
:10E930000C442F46114699B905EB420316B125F850
:10E9400012600233181A4010F0BD31F8157033F818
:10E9500015E077443E4420F81560360C0135E2E7B7
:10E9600034F8023F1E4427F8026B0139360CE2E707
:10E97000F0B4049C0025121B2F46AC420AD164005F
:10E980000519023C0C441346294673B905EB4201B4
:10E99000F0BC9BE731F815603E4433F81570F61B68
:10E9A00020F8156037140135E7E734F8026F3E446C
:10E9B00021F8026B3714013BE7E710B5044638B184
:10E9C0008068FFF761FC2046BDE81040FFF75CBCA3
:10E9D00010BD38B502290446806838BF02210D46B3
:10E9E00018B12368B1EB930F07D96900FFF73DFC1D
:10E9F0002368A06065F39F03236038BD38B50546E2
:10EA00000C20FFF715FC2A78037862F300036FF3FC
:10EA100041030370044628682368C0F39D0060F337
:10EA20009F0323606B686360AB6813B9A3602046E3
:10EA300038BD4000FFF7FCFBA0602A68A968C2F35C
:10EA40009D02520001F089FFF1E710B54B00184418
:10EA50001A4409B9084610BD30F8023D32F8024D9B
:10EA60001B1B002B02DB04D10139F2E74FF0FF3012
:10EA700010BD012010BD38B505460C460221FFF738
:10EA8000A8FF2B78002CB5BF43F001036FF3000300
:10EA90002B702B704FF00003B8BF64426B6004B959
:10EAA00038BD6B68AA68581C686022F81340240CB3
:10EAB000F5E7037803F0FE036FF341030370036887
:10EAC0006FF39F030360002343608360704728B1A6
:10EAD00003789B0702D48068FFF7D6BB704738B530
:10EAE00005460C464968FFF774FF22782B78A86822
:10EAF00062F300032B7063686B606268A168520068
:10EB0000BDE8384001F029BF034609B95960704794
:10EB1000B1E708B5FFF7CDFFBDE80840FFF7F4BF48
:10EB200030B40578816005F0FE0545F002050570FA
:10EB3000056862F39F05002205604260194630BCFB
:10EB4000FFF7E2BFF8B504469DF8185004211F46B0
:10EB50001646FFF73EFF23787DB1002E77F10002C5
:10EB60000BDA43F001037642237067EB470700217D
:10EB7000616056EA070304D1F8BD6FF30003237008
:10EB8000F5E76168A0684D1C656020F81160310CE4
:10EB900041EA0741380C0E460746EAE710EE102A14
:10EBA0000378D10F61F300032DE9F0410370C2F344
:10EBB0000F4313F4FF43054603D100236B60BDE808
:10EBC000F081B3F5FF4FF8D0C2F3C754A4F17F032F
:10EBD000002BF2DB03D10121BDE8F0414BE7162BFE
:10EBE000C2F31602D8BF4FF00008A4F16F064FF031
:10EBF000100142F4000796FBF1F6D3BFC3F11703EF
:10EC00000933963C4446C8BF94FBF1F43146D4BF67
:10EC1000DF4003F00F08FFF7DCFE6E6024B16200F6
:10EC20000021A86801F0BCFEB8F1000F08D0AB6865
:10EC300007FA08F223F81420C8F11003DF4001346A
:10EC40006300B44201D1BDE8F081AA680134D75213
:10EC50003F0C0233F5E72DE9F84304468F18C2F361
:10EC60005B020D469846511C089EFFF7B2FE2278C3
:10EC7000B8F1000F0BD042F0010200232270636054
:10EC80002846B1B2B84205D3401BBDE8F88368F30B
:10EC90000002F2E70278A2F13003092B00F1010E25
:10ECA00005D9A2F14103192B15D8A2F13703B342BC
:10ECB000EAD2A068D4F804C09BB2624680468AB902
:10ECC00000EB4C0213B120F81C300232121A521021
:10ECD00062607046D6E7A2F16103192BD4D8A2F185
:10ECE0005703E4E7B8F8009009FB013328F8023B2A
:10ECF000013A1B0CE3E7F8B5044615461E46C1B1C0
:10ED0000531E1E444FF0FF37E9000F31090920461A
:10ED1000FFF75FFE237800216FF30003237061602B
:10ED20004DB9A068616800EB4101FFF7CFFD60605D
:10ED3000F8BD0127E8E700230F2908DC32788A4074
:10ED40001343013D9BB201F108013E44F4D16268D6
:10ED5000501C6060A068103920F81230E0E70A46C5
:10ED6000416838B5044609B9506890B113782578E0
:10ED700003F0010305F00100181A0AD15368994203
:10ED800008D30AD89268A068FFF75FFEEB0748BF78
:10ED9000404238BD4FF0FF30F8E70120F6E78842E7
:10EDA00010B5044601D0FFF79AFE23786FF30003F5
:10EDB000237010BD884210B5044601D0FFF78FFEC6
:10EDC0002378C3F30002C2F1010262F3000323704F
:10EDD00010BD88421FB5044601D0FFF780FE62686F
:10EDE00062B901212046FFF7F4FDA26801231380D8
:10EDF0006360237843F00103237010E02378D90780
:10EE00000FD56FF30003A16823700123ADF80E3016
:10EE1000009308460DF10E03FFF7AAFD606004B0F1
:10EE200010BD511C2046FFF7D4FDA1686268012384
:10EE3000ADF80E30009308460DF10E03FFF76EFD9E
:10EE40006060D6E72DE9F0470F464968064615464B
:10EE500001B12AB939463046BDE8F047FFF73FBE59
:10EE600002F10F0424092144FFF7B3FD7968B36868
:10EE7000B8686FF0004E04EB010815F00F026FF058
:10EE8000010C08EB0E054FEA45050CFB01FC8E4416
:10EE90000CEB4E0E08BF10222B44704499464FF0E5
:10EEA000000EC2F1100209BB2EFA02FE03EB0C09A0
:10EEB00023F80CE06300C3F1020304F1004299441B
:10EEC000013A4846520001F06BFD0235A944B8F101
:10EED000000F02D039F8023DA3B1C6F804803A7899
:10EEE000337862F300033370BDE8F08730F811A087
:10EEF0004AEA0E0E2EFA02FA29F802A94FEA0E4E3D
:10EF00000139D0E708F1FF38E1E7F0B50E4649686E
:10EF100085B00546144601B12AB931462846FFF7A7
:10EF2000DEFD05B0F0BDFFF754FD23467268B16801
:10EF3000A868FFF7D7FC686031782B7861F300038D
:10EF40002B70DB070246ECD500237068ADF80E305D
:10EF50002109834202D08B4213D103469942E0D269
:10EF6000B36804F00F0433F81110012303FA04F41A
:10EF7000013C214218BFADF80E30BDF80E304BB940
:10EF8000CFE7B76837F813707FB101238142ADF83E
:10EF90000E30E5D30123A9684AB1009308460DF16C
:10EFA0000E03FFF7BBFC6860BBE70133D1E70B80C2
:10EFB0006B60B6E773B553680C46496899420646DC
:10EFC000154606D308D89268A068FFF73EFD0028D2
:10EFD00002DA23462C461D4623782A78616853407E
:10EFE000DB0713D401313046FFF7F3FC6B68009365
:10EFF000AB686268A168B068FFF790FC7060227827
:10F00000337862F30003337002B070BD3046FFF70F
:10F01000E0FC6B680093AB686268A168B068FFF7BA
:10F02000A7FCEBE7F7B553680C46496899420646DA
:10F03000154606D328D89268A068FFF706FD002879
:10F0400022DA234601272C461D4623782A78616858
:10F050005340DB071AD501313046FFF7BAFC6B6825
:10F060000093AB686268A168B068FFF757FC7060F6
:10F07000227833781FB1C2F30002C2F1010262F3B9
:10F080000003337003B0F0BD0027DEE73046FFF722
:10F09000A0FC6B680093AB686268A168B068FFF77A
:10F0A00067FCE4E72DE9F04F15464A686B689A4221
:10F0B0000C463EBF2C460B461D462378616813F074
:10F0C000010308BF2B7803F0010385B019440646FD
:10F0D000FFF77FFCD4F804C0D4F80890D5F804B04A
:10F0E0002478D5F808E02D78B06884EA0503DF07B6
:10F0F00054BF04F00103002304F0010259421746F3
:10F1000089B205F001050191794289B2C5F1000883
:10F11000ABEB0C04009202912A461FFA88F80CF11E
:10F12000FF31A9F10209824603944C1C12D100EB75
:10F130004C011BB1012320F81C300231FFF7C6FB44
:10F14000009C337870602C4064F30003337005B08A
:10F15000BDE8F08F39F802BF029C8BEA040B039CD8
:10F160005F4404EB010B8B4598BFBEF800B0019CD7
:10F1700094BF88EA0B0BC3465A4407EA020B8BEA9A
:10F18000040B13FA8BF32AF8023B98BF0EF1020E20
:10F19000120C3F0C1B0C0139C7E72DE9F04F154647
:10F1A0004A686B689A420C463EBF2C460B461D4689
:10F1B0002378616813F0010308BF2B7803F0010383
:10F1C00085B019440746FFF704FC6168D4F808E0ED
:10F1D00024782E78D5F804A0B868AD68009514F0AE
:10F1E000010308BF334603F001035A4204F001044F
:10F1F00092B206F001060192624292B2C6F1000C90
:10F20000AAEB01050292A046B1461FFA8CFC4A1EE9
:10F21000AEF1020E83460395551C0CD100EB410163
:10F22000FFF754FB3B787860344364F300033B7092
:10F2300005B0BDE8F08F3EF802AF029D8AEA050AEC
:10F24000039DD04405EB020A524525BF009DB5F849
:10F2500000A0E2468CEA0A0A28BF0235D14428BF42
:10F260000095019D48EA090A8AEA050A13FA8AF319
:10F270002BF8023B4FEA19494FEA18481B0C013A98
:10F28000CAE72DE9F74F15464A686B689A420C4663
:10F290003EBF2C460B461D462378616813F00103E0
:10F2A00008BF2B7803F0010319440646FFF791FBD2
:10F2B00023782A78D4F804E0B068D5F808C083EA47
:10F2C0000207D24302F001020092A268A2F10209F1
:10F2D0006A68DB43A2EB0E0207F0010703F00103AB
:10F2E0000EF1FF3180464FF6FF7A01924A1C13D18E
:10F2F00000EB4E011FB1012320F81E300231FFF751
:10F30000E5FA706022782B785340327863F300027C
:10F31000327003B0BDE8F08F39F802BF019AD344D0
:10F320005B4402EB010B594528BFBCF800B0009AC2
:10F330002CBFD3444FF6FF7B5A4483EA020B17FAE3
:10F340008BF74FEA124228F8027B28BF0CF1020C1F
:10F3500000921B0C3F0C0139C8E72DE9F04F4B68B8
:10F3600085B004460E4615460BB1536823B90023F9
:10F37000636005B0BDE8F08F814207D1FFF73EFB27
:10F38000B542074600D105463E4605E082422DD1F2
:10F39000FFF734FB074605466B6871682046194441
:10F3A000FFF717FB2268A068C2F39D0252000021FC
:10F3B00001F0F6FAB368D6F804E0D4F808A0029396
:10F3C0006FF0010303FB0EF3D5F808806A6803931E
:10F3D0000AEB4E010020039B03EB010C42B3029B9E
:10F3E000CDF804E0A3F10209002310E00027D3E7E1
:10F3F00039F8020FB8F800B00BFB0033BCF800B0CE
:10F4000001985B4401382CF8023B01901B0C0198D9
:10F410000028EDD1084601F1020C0BB10B806046CB
:10F42000A0EB0A004010013A08F102086146D2E759
:10F430006060337829784B4013F0010F2378384609
:10F440000CBF62F3000343F00103237005B0BDE875
:10F45000F04FFFF7B2BA4B6870B50646144613B1C9
:10F460001378DA0702D50023736070BD636823B98F
:10F470000121BDE87040FFF7FEBA0846FFF7BEFA6B
:10F4800005462046FFF7BAFA012104463046FFF749
:10F49000F2FA636883B1A3681B88DB0704D52A46A8
:10F4A00031463046FFF759FFA168626801230846DC
:10F4B000FFF718FA606038B92846FFF77EFA204651
:10F4C000BDE87040FFF779BA2A4629462846FFF77B
:10F4D00044FFDEE72DE9F04F0C4651688FB09146AE
:10F4E000013105460293FFF774FAD9F80420A868A1
:10F4F00001325200002101F053FA00236B60D9F869
:10F50000041020460131FFF764FA49462046FFF710
:10F51000E6FA029B67689E685B680193AB68039399
:10F52000019BD4F808B0BB422CD82DD332463946C3
:10F530005846FFF78AFA002823D1039A6060012316
:10F5400013806B60029A99F8003012785340DB0701
:10F5500014D52B7843F001032B70636873B14FF01F
:10F56000FF310BA8FFF7D5FA0BAA29462846FFF76B
:10F5700021FD029A21462046FFF71CFD0FB0BDE891
:10F58000F08F01DA0023DCE7019B03F10040013832
:10F590004FEA400A36F81030002213F4004F02F10F
:10F5A000010156D07B0092B24FF0000C791C03F1A0
:10F5B00002080593C2F110032BF817C0D84461600C
:10F5C000DE4667460493C64547D336F8100000FA76
:10F5D00002F30493019B012B09D906EB0A00C2F147
:10F5E000100730F8020CF840049F07430497019875
:10F5F000059B091A6960039801F10041013900EB8C
:10F60000410106916FF00101A1EB0A010991B11EC0
:10F610005B440891D4F804A00199514529D30AF11B
:10F62000004A0AF1FF3A0BEB4A0A0020C2F1100629
:10F63000D34540F28D806FF000416B6833B15A18AA
:10F64000039830F81220002A00F08C806FF00041FF
:10F650008DE05B009BB20A469FE7BEF800C00CFA43
:10F6600002F31F43049B2EF8027B2CFA03F7BFB270
:10F67000A9E7198833F8026C46EA01460499B6FBFB
:10F68000F1F60999591805910F460899079100213B
:10F690008C46BB4212D81888814237D3091A484297
:10F6A000188088B2003018BF012000EB114179B3F7
:10F6B0000020DDF82080059F844640E0079837F859
:10F6C000028B30F802EF07900EFA02F040EA1C4C71
:10F6D0001FFA8CF07043404503D2A8EB000E8E4514
:10F6E0000ED80144A1EB0808C8F1000127F8021C5C
:10F6F0001FFA88F1003118BF012101EB1841C8E75A
:10F70000AEEB010127F8021C0021C2E7411A198063
:10F71000069921F8026906910AF1FF31023B616006
:10F7200078E738F802EF0EFA02FE4EEA1C4CB7F802
:10F7300000E010FA8CF0704427F8020B000CBB427A
:10F74000EFD81F8838441880A1EB1041013EAEE786
:10F75000BAF8003043FA02F10143B3402AF8021923
:10F7600098B265E7013B6B6067E7013B63606368E4
:10F77000002B3FF4E7AE5A183BF81220002AF4D0D1
:10F78000E0E6F0B51F464B6885B00646154613B156
:10F790001378DA0703D50023736005B0F0BD6B68FA
:10F7A0001BB90121FFF767F9F7E70846FFF726F9CC
:10F7B00004462846FFF722F9054601A8FFF779F924
:10F7C00001213046FFF757F96B68B3B1AB681B886E
:10F7D000DB070AD5224631463046FFF7BEFD3B46E1
:10F7E0003246314601A8FFF775FEA9686A68012311
:10F7F0000846FFF777F8686048B901A8FFF767F98E
:10F800002046FFF7DAF82846FFF7D7F8C5E7224683
:10F8100021462046FFF7A1FD3B462246214601A88E
:10F82000FFF758FED0E710B581684268002301EB6E
:10F830004202914205D30278D20748BF5B42184684
:10F8400010BD32F8024D44EA0343F2E730B5426896
:10F850008468002304EB4202944206D30278D20764
:10F8600048BF5B420B60012030BDB3F5004F04D2AE
:10F8700032F8025D45EA0343EEE7002030BD03782D
:10F8800013F0010310B510D18468426804EB420202
:10F89000944202D30B60012010BDB3F5803F04D227
:10F8A00032F8020D40EA0343F2E7002010BD2DE9D3
:10F8B000F043884661B19D18846841680026A4F130
:10F8C000020E4FF0010937461A4419B9BDE8F0831A
:10F8D0001D46F1E73EF8024F103744EA0646072F6F
:10F8E00001DC0139F1E790F800C0B4B21CF0010F5F
:10F8F0001FBFE44359FA84F4A4B24FEA1429B8F1C3
:10F90000000F07D005F1FF3C634505F8014C06D117
:10F91000BDE8F08305F1010C94452C70D6D0083F6A
:10F92000360A6546DBE7826843689FED0C0A9FED67
:10F930000C7A02EB43039A4205D30378DB0748BFF6
:10F94000B1EE400A704733F8021D07EE901AF8EE48
:10F95000E77A40EE077AB0EE670AECE700000000B5
:10F96000000080472DE9F84F0B9C9DF828A08046A9
:10F97000894616469B46002C00F085808B1E1E2B68
:10F9800003D900202070BDE8F88F456895B97AB199
:10F99000561E204616F8013F3BB930230370002362
:10F9A00000F8013F001BBDE8F88F00F8013BF1E7CC
:10F9B0002046F2E76D002846FEF73AFC2A46074645
:10F9C000D8F8081000F0C9FFABF13A0B20462246E8
:10F9D00007EB050EAEF1020300219F4210D9303132
:10F9E000392988BF5944551C11703B469E4519461C
:10F9F00010D8BAF1000F1ED0012313E02A46E9E720
:10FA00001D8845EA0141B1FBF9F523F8025909FBCC
:10FA10001511E2E7098802330029E7D0BAF1000F97
:10FA2000ECD00023291A032902BF951C82F801A0FB
:10FA30002846002BE2D03846FEF726FC3EB1304681
:10FA400001F01AF92B463044B0421D460FD898F801
:10FA50000030DB0742BF2D232B7001356B1E224681
:10FA60009A4209D300232B70281BBDE8F88F10F8A9
:10FA7000012D03F8012BE7E71178187802F8010B44
:10FA800003F80119ECE72046BDE8F88F8368C268E7
:10FA900093423DBF5A1C826018784FF0FF30704788
:10FAA000036810B5044613B14068FEF7EDFB20462D
:10FAB000BDE81040FEF7E8BB10B50378044613B16B
:10FAC000406801F0EFF92046BDE81040FEF7DCBBCE
:10FAD0008368C2689A4210B5044610D353B100F14E
:10FAE00010011422406801F0D9FB00284FF00003F8
:10FAF00003DCA3604FF0FF3010BDA060E360E3685B
:10FB00005A1CE2601C44207C10BDF8B5054610204C
:10FB10000C461F461646FEF78BFB054B446084607F
:10FB200034440760C4606B60024B2860AB60F8BD72
:10FB30008DFA0008A1FA0008F8B5054624200E4603
:10FB40001746FEF775FB14220770466000F110019E
:10FB50000446304601F0A2FB431C08D117B13046E1
:10FB600001F0A0F900F032FB0068F6F773FB002308
:10FB7000E360034BA0606B60024B2C60AB60F8BD90
:10FB8000D1FA0008B9FA000810B54FF4D272044651
:10FB90000846012101F0EDFA011E04DA00F016FB1F
:10FBA0000068F6F757FB20460122BDE81040FFF73A
:10FBB000C3BF00BF2DE9F041054630200E469046F8
:10FBC0001F46FEF741FB072D04460570C660A0F8EE
:10FBD000108001D0012D0FD1B3681B096382F5F7A6
:10FBE000A5FB042360616776E3842020FEF720FBF9
:10FBF000E0622046BDE8F081014B5B5DEEE700BFAF
:10FC0000D318020810B50446C06AFEF73DFB204633
:10FC1000BDE81040FEF738BB30B5048D0022A2428B
:10FC200002D30023184630BDC36A03EBC2035D68EC
:10FC30008D42F7D00132F2E770B504460E46154604
:10FC4000FFF7EAFF10B100232B7070BDE18C238D0C
:10FC50008B4208D30631C900E06AFEF706FBE38C4D
:10FC6000E0620633E384228DE16A531C01EBC2009B
:10FC70002385002301F8323043704380466001231E
:10FC8000E2E743680BB9FFF7C7BF1846F9E7F7B5D6
:10FC900044680D4616464CB900232B7004E00378E7
:10FCA000022B01D10323037003B0F0BD23465F682C
:10FCB000002FF1D018463146FFF7AEFF3B46002833
:10FCC000F5D00378023B022BE6D804232B701D46A7
:10FCD0000DF1070231462046FFF7AEFF9DF80730D1
:10FCE000002BDCD005706468F2E700BF012910B575
:10FCF00011682DD931F01004037815D1302B13D1B0
:10FD0000447844F02004782C00F1020303D1102140
:10FD10001160181A10BDF1B96F2C01D10821F7E755
:10FD2000622C16D10221F3E7082908D1302B12D119
:10FD3000437843F020036F2B0DD1831CE9E70229A0
:10FD400006D1302B07D1437843F02003622BF3E731
:10FD500009B90A2313600346DBE7000008B5014830
:10FD6000F5F7FAFCDA18020810B59DF8084011B151
:10FD70000CB9FFF7F3FF9A4202D18242F9D110BDCC
:10FD80008242F6D88342FAD2F3E72DE9F74F0C9D71
:10FD9000DDF834A00193002481468B469046264628
:10FDA0002746019B9C4209D14F4523D3D8F8003008
:10FDB000B6EBD30F1ED303B0BDE8F08F4C450DD288
:10FDC0006A88920516D45BF824000137AA78012AC4
:10FDD0001DD1F6F749FE8AF8000010E02988890055
:10FDE000002241F002014046F6F78FFA60B96A88B6
:10FDF000D30501D5FFF7B2FF6A68CAF800200134C5
:10FE000008350AF1040ACCE701364068DEE7022A29
:10FE100001D1F6F7B1FCCAF80000F0E770B586B082
:10FE20000446154602EB800203A81E46F6F73DFA8B
:10FE30000B9B01930A9B009303AA33462946204655
:10FE4000FFF7A3FF06B070BD406870474160704780
:10FE500010B504460820FEF7EBF9024A80E81400CA
:10FE600010BD00BFF81802082DE9F04104464068B3
:10FE70008000FEF7DDF904F10C08074600256168F3
:10FE80008D4206D33B46A0680022BDE8F041F5F75D
:10FE9000E1BC58F8040BF5F727FE064618B147F801
:10FEA00025000135EBE73846FEF7EEF93046BDE8B0
:10FEB000F0812DE9F3410D460024074611462846FE
:10FEC000984602224FF6FF730094FFF74DFFA81CDF
:10FED0008000FEF7ADF90760013DD8F800304560BD
:10FEE0000646836000F10C07AC42234603D330463C
:10FEF00002B0BDE8F0815C1C002158F82400F5F741
:10FF0000A9FD47F8040BEFE713B50023044600935F
:10FF1000084611461A46FFF727FF0420FEF788F926
:10FF2000046002B010BD0000C268002A034605DD6F
:10FF300040689968884206DB00207047FCD0406822
:10FF400099688842F8DD596848000A4440F0010089
:10FF50005A607047C26883684068181A1044002AC3
:10FF6000CCBF00F1FF30013090FBF2F020EAE070EE
:10FF7000704710B504460846FFF7ECFF042C03D089
:10FF8000052C08D0002010BD054B064A0028CCBF28
:10FF90001046184610BD400040F0010010BD00BFE3
:10FFA000A0EA010898EA010810B582684468C368AD
:10FFB00003488A6081E81100CB60084610BD00BF8D
:10FFC000AC1902082DE9F3410E4600271146804680
:10FFD0001D460122032330460097FFF7C5FE10207F
:10FFE000FEF726F90123C0F800809E4204464760D0
:10FFF000C360286806D1F6F7BFFBA060204602B0B8
:020000040801F1
:10000000BDE8F081F6F7B8FB60606868F6F7B4FB0E
:10001000032EA060F2D1A868F6F7AEFBE0600028DE
:10002000ECD10148F5F790FB241A020838B50C46CC
:100030004A688B6809490546F0F73AFDE268012AEB
:1000400005D128460649BDE83840F0F7C7B928462B
:100050000449BDE83840F0F72BBD00BF2E1A020856
:10006000160702083D1A0208042A10B504460FD1EB
:10007000FFF770FF00230A4601462068F6F790FC60
:10008000E368626803FB0020400040F0010010BDFF
:10009000002010BD136810B514462BB9D22904D125
:1000A0004068F8F77DFC206010BDD62901D180683A
:1000B000F7E7D529F8D1C068F3E700BF2DE9F84389
:1000C0000646406860B10021FAF7E9FF06F1080929
:1000D000044600F10808002573689D4202D32046BB
:1000E000BDE8F88359F8040BF5F7FEFC074628B97C
:1000F0002046FBF7B8F83846BDE8F88348F8040B0B
:100100000135E9E72DE9F3410E4600240746114683
:1001100030462246984600944FF6FF73FFF724FEC0
:10012000B01C8000FEF784F807600546466000F1C9
:100130000807B44203D1284602B0BDE8F08158F860
:1001400024000021F5F786FC013447F8040BF0E7A2
:10015000194B0128F7B50D46174693E850001AD9F8
:100160004968164A914207D08C0710D10C68144B8D
:100170009C420CD10C460E4602280CD0AB68934230
:1001800009D09A0703D119680D4A914202D0002084
:10019000F5F7E2FA1C4601A92868FAF701F8019A76
:1001A000014600233420F0F7E4FF23463246394667
:1001B000F5F76DFB03B0F0BD3C2100204CFA0108BF
:1001C0008CEC01080222C3E70122C1E708B500F068
:1001D00061FE38B9044B186820B1837E032B01D12E
:1001E0006C3008BD014808BDE4220020DC05002079
:1001F0004F4D504A504E01232B70002383B513609E
:1002000053604E4A136053604D4A136053604D4A29
:10021000136053604C4A136053604C4A1360536040
:100220004B4A136053604B4A136053604A4A338011
:100230001F464FF6FF7099189F500833802B888017
:10024000F9D13388454C318803F00F03204642F83A
:10025000334002EBC30291804FF4AC72002100F0F6
:100260009FFB3388A3813E4B236163610623A383F5
:100270003C4B3049C4F85831032604F5AC73204692
:10028000C4F85431A676C4F85C7100F0A9F8204691
:1002900000F0E0FD022301A968462B7000F076FD16
:1002A0009DE8030000F050FD2F4B2E700BB108F0BD
:1002B000CBF82E4B0BB101F0FBFC2D4B0BB107F033
:1002C0009BFF2C4B0BB1AFF300802B4B0BB10BF012
:1002D00075F82A4B0BB10BF08DFE294B0BB1AFF328
:1002E000008000F0C4FE00F09BFD0423217F1B482A
:1002F0002B7001F0C3F8194801F0E4F8174801F039
:10030000DBF8A36801221A70022000F063F80523CD
:100310002B7001F029F900F04DF830B100F02AFD02
:1003200018B900F02FF800F02BFD00F03BFDF2E7CC
:10033000EC220020E42200209023002088230020CB
:10034000DC22002000230020F0220020D422002004
:10035000F82200209423002008230020E00500203C
:10036000F1010108981A020849840108B11C01082A
:10037000F981010800000000BDB30108F5BF0108C4
:100380000000000070B50A4D10262B6803B970BD3F
:10039000EFF3118486F31188284600F0C4FCE4B220
:1003A00084F311880028F0D000F0C8FCEDE700BF0E
:1003B00094230020024B1868003018BF01207047BA
:1003C00094230020024B1B689868AC30704700BF34
:1003D000E4220020022801D103F0CEBA00207047A9
:1003E000002343600B6803600B6813B90860486022
:1003F000704758600860704708B500F061F8DFED9D
:10040000027A37EEC00A08BDDB0FC93FF0B52DED0B
:10041000048B9FED298A9FED299A83B0F0EE408AE4
:100420000024002538EE680A00F072F9B4EEC90A1B
:10043000F1EE10FA2046294607DC0DF07DF800EEBB
:10044000100A03B0BDEC048BF0BD0DF075F800EEA2
:10045000100A00F017F918EE100A8DED010A0CF0E1
:100460007DFD064618EE900A0F460CF077FD024619
:100470000B46304639460CF011FC9DED010A06464C
:1004800010EE100A0F460CF069FD02460B4630468E
:1004900039460CF0E1FE02460B46204629460CF098
:1004A000FDFB0D4604460DF047F800EE100A00F083
:1004B00009FBB0EE408AB5E7000000000000003400
:1004C00008B5FFEE007AB4EEE70AF1EE10FA2DED72
:1004D000028BB0EE408A2FD4F7EE008AB4EEE80A21
:1004E000F1EE10FA28DCB4EE400AF1EE10FA23D156
:1004F00000F00EF9DFED147AB4EEE70AF1EE10FA2F
:1005000013DDB0EE680AA8EE480A00F051FBFFF7D1
:100510007DFFF0EE480ABDEC028BDFED0C7ABDE802
:10052000084037EEC00A00F0A0B8B0EE480ABDECB3
:10053000028BBDE8084069E7BDEC028BDFED047A71
:1005400087EEA70A08BD00BF8FC2353FDB0FC93F4A
:1005500000000000F5EEC00AF1EE10FA08B505DD66
:1005600080EE200ABDE8084000F042B8B5EEC00AAF
:10057000F1EE10FA0DDBF5EEC00AF1EE10FA08D537
:1005800080EE200A00F034F8DFED157A30EE270A0D
:1005900008BDB5EEC00AF1EE10FA0DD5F5EE400A31
:1005A000F1EE10FA15D080EE200A00F021F8DFED10
:1005B0000C7A30EE670A08BD0EDDF5EE400ADFED7D
:1005C000097A9FED090AF1EE10FA08BFB0EE670A4A
:1005D00008BD9FED060A08BD9FED030A08BD00BFD8
:1005E000DB0F4940DB0FC93F00000000DB0FC9BF34
:1005F00008B52DED028BB0EE408AB7EE000AA8EEEA
:10060000080A00F0D5FA88EE000ABDEC028BBDE8BE
:100610000840FFF755BF00B52DED028B83B002A84F
:10062000B0EE408A20ED010A00F0C2F9B5EEC08AB2
:10063000F1EE10FA12DD9DED010A38EE400A00F0ED
:1006400067F8B5EEC00AF1EE10FAC1BFDDED017A30
:10065000B7EE007A77EE877ACDED017A9DED010A4B
:1006600003B0BDEC028B5DF804FB10EE103A10EE07
:10067000902A23F0004302F00042134300EE103AA8
:1006800070470000DFED027A30EE270A00F01ABA58
:10069000DB0FC93F10B5B5EE400AF1EE10FA2DEDB3
:1006A000028BF7EE008A2BD0B5EEC00AF1EE10FAFD
:1006B00048BFB1EE400ABCEEC07A134B9FED138ADF
:1006C000F8EE477A48BF012430EE670A58BF00248D
:1006D00003F12802F7EE007AF3EC016A9342A6EEEA
:1006E000A78A67EE807AF7D117EE100A00F084F837
:1006F00028EE000A0CB188EE800ABDEC028B10BD1A
:10070000B0EE680AF9E700BFEC1A0208000000002A
:10071000B5EEC00AF1EE10FA48BFB1EE400A7047DC
:1007200000B52DED028B83B0B0EE408A01A800F039
:100730003FF9B5EEC08AF1EE10FA0CD5DDED017A85
:10074000B4EEE78AF1EE10FA42BFB7EE007A77EE28
:10075000C77ACDED017A9DED010A03B0BDEC028BA5
:100760005DF804FB00B52DED028B83B001A880EE8F
:10077000200AB0EE608A00F01BF928EE000A03B0F0
:10078000BDEC028B5DF804FB0EB403B503AA52F86E
:10079000041B019200F0ACFA02B05DF804EB03B068
:1007A000704710B52DED028B0446B0EE408A00F084
:1007B00045F8FFF730FFFDEEC07AB7EE000A17EEFE
:1007C000900AC4ED007A00F005F888EE000ABDEC4E
:1007D000028B10BD08B507EE900A2DED028BF8EEE6
:1007E000E70AB0EE408AB0EE000A00F019F920EEF8
:1007F000080ABDEC028B08BD582810B5F7EE007A48
:1008000006D80C4AB0EE670A0023012428B910BDAF
:100810009FED097A87EE870A10BD04FA03F10142C1
:100820001EBFD2ED007A884320EE270A013304323E
:10083000ECE700BF181B02080000000008B500F03C
:1008400007F8DFED027A80EE270A08BD1872313F03
:1008500008B52DED0A8BB0EE40BA9FED328A9FEDC0
:10086000320ADFED329A9FED32AAF7EE007AF0EE0F
:1008700040BAB0EE679AF0EE48AAB0EE40CA37EE42
:10088000807AB4EEC78AF1EE10FA12DC77EEC07A05
:10089000B4EEE78AF1EE10FA0BD4B4EE698AF1EE09
:1008A00010FA36D189EE2A8AB0EE480ABDEC0A8BDE
:1008B00008BDB0EE480AFFF7EDFE70EE4B7A87EE0A
:1008C000800A78EE408AF4EEE98AF1EE10FA1ADC3A
:1008D000F4EE4A8AF1EE10FA48BFF0EE4A8AB0EE22
:1008E000680AFFF715FFB4EEC90AF1EE10FA0DDD44
:1008F000B0EE680AFFF70CFF20EE2B0AF0EE487A04
:10090000B0EE688ABBE7DFED098AE8E7B0EE4C0A93
:10091000F4E7DFED077AB4EE678AF1EE10FAC1D0A2
:10092000C2E700BF00000000000000340000B04239
:100930000000B0C210B501390244904201D100203C
:1009400010BD10F8014B11F8013F9C4202D3F4D9BD
:10095000012010BD4FF0FF3010BD10B5431E0A44FA
:10096000914200D110BD11F8014B03F8014FF7E798
:10097000884210B501EB020308D8421E994200D10B
:1009800010BD11F8014B02F8014FF7E78118D21A98
:10099000D34200D110BD13F8014D01F8014DF7E726
:1009A00002440346934200D1704703F8011BF9E764
:1009B00010B52DED028B0446B0EE408AFFF7A8FE7D
:1009C000DFED157AB4EEE70AF1EE10FA08DB84EDFC
:1009D000008A9FED128AB0EE480ABDEC028B10BD72
:1009E000B0EE480AFFF794FEF7EE007AB4EEE70A9D
:1009F000F1EE10FA55BFFDEEC87ADFED087AF8EE99
:100A0000E77A68EE277A56BFC4ED007AC4ED007A23
:100A100038EE678ADFE700BF0000004B00000000EF
:100A200008B52DED028BB0EE608AFFF711FF20EEC6
:100A3000080ABDEC028BBDE80840FFF72BBE0FB4DF
:100A400013B504AB53F8044B0193FFF7BBFC019AB9
:100A50002146283000F04CF902B0BDE8104004B047
:100A6000704773B50446FFF7ADFC00F12805064654
:100A7000284603F054FB2046294603F074FB041E6D
:100A800015DD02A80A2300F8013D2A46012103F0E2
:100A9000DEFB00280BDD96F846305B0704F101040D
:100AA00007D50121284603F08BFB002801DA4FF01F
:100AB000FF34FFF787FC283003F047FB204602B0E5
:100AC00070BD000008B52DED028B9FED248AF0EE7D
:100AD000480AFFF747FE9FED227A9FED226A224ADD
:100AE000B4EEC70AF1EE10FAF0EE407AF0EE476A83
:100AF000A8BF70EE487A9FED1D7A9FED1D0AF4EEB7
:100B0000C77AF1EE10FA48BF77EE887A0023F4EE48
:100B1000C67AF1EE10FAA8BF76EEE77ADFED156A35
:100B2000F4EEE67AF1EE10FA48BF77EE677A27EE38
:100B3000A77AD2ED006AD90703F1010358BFA6EEE8
:100B4000A70A02F1040248BFA6EEE70A062B67EEE9
:100B5000877AEED1BDEC028B08BD00BFDB0FC94028
:100B6000DB0F4940DB0FC93F341B0208DB0F49C0D4
:100B700000000000DB0FC9BF1FB5044610B90020FC
:100B800004B010BD0021009002AB6A4608460191F6
:100B900000F0E6FD0028F2DA02988442F0D9039AC8
:100BA000024B9A42C8BF0130EAE700BFFF64CD1D87
:100BB00008B52DED028BDFED248AB4EEE80AF1EEE4
:100BC00010FAB0EE408A0AD5FFF700FB212303603C
:100BD000C8EEA87ABDEC028BB0EE670A08BDB4EE91
:100BE000400AF1EE10FAF3D1B7EE007AC7EE287A98
:100BF000B4EE670AF1EE10FAECD0B1EE677AB4EE1B
:100C0000470AF1EE10FAE5D0B5EE400AF1EE10FA1F
:100C100016D003F078FBC8EE007AB6EE007A37EE15
:100C2000800A20EE070AC8EE007A77EE807A27EE77
:100C3000870AC8EE007A77EE807A67EE877AC9E78E
:100C4000F0EE687AC6E700BF0000000040B102463F
:100C5000104612F8013B8B4202D0002BF8D1184607
:100C60007047421E12F8013F11F8010B181A40B2EA
:100C700008B9002BF6D1704703461A78591C0AB9F7
:100C8000181A70470B46F8E708B52DED028BF0EE09
:100C9000408AFFF717FFB0EE408AB0EE680AFFF710
:100CA000F1FC88EE000ABDEC028B08BD10EE102AA4
:100CB000C2F3C753763B1F2B82B010EE100A11DC33
:100CC000082BD8BF01234FF0FF3121FA03F31A425A
:100CD00008D0DFED067A70EE277ACDED017A019A21
:100CE00020EA030200EE102A02B070470000807B69
:100CF0007FB50D461646044690B10146684603F09E
:100D000094FE204603F00BFA29463246684603F06B
:100D1000B1FC0546204603F018FA284604B070BD21
:100D20004FF0FF35F9E703682BB11A68026002B98A
:100D3000426000221A6018467047000001460148D0
:100D400003F0B4BF9C2300200A460146014804F08A
:100D50001FB800BF9C2300200146014804F039B8A9
:100D60009C2300200A460146014804F071B800BFE8
:100D70009C230020014804F04BB900BF9C230020B5
:100D8000014804F070B900BF9C230020044B1B688D
:100D90000360C3F1005303F540330B60704700BF9D
:100DA0004C1B020830BF704708B504F04BFEEFF350
:100DB000148343F0040383F31488134A136823F065
:100DC00040431360A2F5D672136843F470031360B6
:100DD00004F0FEFD04F03AFC0C4B0D4A0021934256
:100DE0000AD30C4A0C4B0D498B4208D305F094F8FA
:100DF00000F063FAFFF7FCF943F8041BEFE752F841
:100E0000040F43F8040BEFE734EF00E0DC050020AB
:100E1000942800208422020800000020DE03002025
:100E200008B50A4B00221A6004F038FD084B0BB1DC
:100E300004F064FB05F017FA03F0DEFE05F080F81D
:100E40000120BDE80840FFF7C5BA00BF0C2500200F
:100E5000FD54010810B50446E42200217030FFF76C
:100E60009FFD236BC4F88030236923F00103C4F88D
:100E700004314FF08073C4F808316FF01603C4F8E2
:100E8000A8300023C4F84C31C4F85031F023C4F822
:100E9000843010BD024B1868003018BF0120704725
:100EA0000C250020072810B50AD800F0B1F800285A
:100EB00008DA4442FFF78AF904604FF0FF3010BDB2
:100EC0000924F7E7002010BD70B58568064675B1A6
:100ED000EC681CB164680CB1A0470446284600F0D9
:100EE00017F9002333607360B360204670BD2C4651
:100EF000FBE710B50446204600F0AEFB0430FAD004
:100F000010BD70470122002103F016BE70B50546E2
:100F1000041D00F1840620461034FFF7D5FFB442CB
:100F2000F9D12846BDE8704000F040BBF8B50C464A
:100F30000646002841D08368002B3ED000293CD0D3
:100F400000F02CFB074608B1FFF7D3FF2046FFF760
:100F5000BBFF051E24DBB568284600F08AF833681D
:100F6000236073686360A560EB681BB90FBB002545
:100F70002846F8BD19680029F8D06A8902F00702EE
:100F8000022A13D1DB6921463046984700280546DE
:100F9000ECDAA06800F0BCF8002323606360A36073
:100FA000002FE5D0384600F019FBE1E720468847DE
:100FB000ECE7384600F012FBD9E76FF00805D7E7F9
:100FC0002DE9F0411C460F469046064600F0E6FA31
:100FD0000546FFF78EFF05EB0413072C05DD2846B9
:100FE00000F0FCFA4FF0FF340DE0103353F8040C1E
:100FF00060B905EB041318615F60C3F80880DE6018
:10100000284600F0EBFA2046BDE8F0810134E4E721
:1010100038B5044600F0C2FA072C05460FD8240163
:101020000319DB685BB1FFF764FF201D2844FFF75D
:101030004BFF0446284600F0D1FA204638BD6FF039
:101040000804FAE738B5044600F0A8FA072C05466C
:101050000CD8FFF74EFF05EB0410002343608360BC
:10106000C3602846BDE8384000F0B8BA38BD00F08B
:101070000DB810B5044640B100F01EF823890133C5
:101080002381BDE8104000F031B810BD10B5084C08
:1010900001220021204603F04FFD4FF6FF736380CD
:1010A0000023A380034B0BB1FFF72BFF10BD00BF44
:1010B00040070020030F010870B500F097FC0A4BB1
:1010C000B3F90220824205461C4603D19A880132B8
:1010D0009A8070BD1E46304600F0BEFA0430FAD049
:1010E00001236580A38070BD400700200748B0F948
:1010F0000430012B02DD013B838070474FF6FF7304
:1011000043800023838000F069BA00BF40070020BD
:1011100010B50446C0B1FFF7CFFFB4F908300BB1EA
:10112000013B2381B4F90830002B09DC63891B07DC
:1011300006D5FFF7DBFF2046BDE8104005F0FFBBFA
:10114000BDE81040FFF7D2BF10BDCB0702D5C36882
:101150009B685BB111F0020106D0C368DB68002B0D
:1011600014BF00216FF00C01084670476FF00C01AE
:10117000FAE70EB470B5064687B030B9FFF726F827
:10118000162303604FF0FF341EE00023019001A8F6
:10119000029303930493059305F0C0FB002804DA3F
:1011A0004442FFF713F80460ECE7029D6B8903F0FB
:1011B0000702012A0ED12846FFF7AAFF0B993046F5
:1011C00005F064FA041EECDB204607B0BDE8704071
:1011D00003B0704713F0050233D1EB68002B30D019
:1011E0000B992846FFF7B1FF002804DA444228464D
:1011F000FFF78EFFD5E713460B992846FFF7E0FE71
:10120000041E20DB694605F072FB0028EEDBEB686C
:101210001E68002ED8D06B8903F00703022B0DD176
:101220004FF4DB730B9A05990098B0470028CBDA8E
:1012300046422046FFF706FF3446D8E70098B047FD
:10124000F4E70624D3E71824D1E710B404688368D0
:10125000E40707D55BB1DB684BB19B683BB15DF838
:10126000044B18476FF00C005DF8044B70476FF0AB
:101270000800F9E7072837B50C4615460BD801A931
:1012800005F035FB002804DB2A4621460198FFF7CC
:10129000DCFF03B030BD6FF00800FAE710B5FFF7D0
:1012A000E9FF041E05DAFEF791FF644204604FF087
:1012B000FF34204610BD0000704710B54FF44020A9
:1012C00004F0D8F90A480B4C04F0D4F90A4804F0A9
:1012D000D1F90A4804F0CEF9204604F0CBF92046B3
:1012E000012104F0B4F90648BDE8104004F0C2B989
:1012F00001000C000408040002000C0003000C00B4
:101300000708040070B50422ADF50A7D46490120A6
:1013100004F08AF80146454800F0FCFE012004F084
:1013200058FF02F03AFE014630B300220024104676
:1013300002F0A8FA009423463D4A3E493E4805F093
:10134000A7FBA0421BDA4FF480713B480BF034F846
:1013500000942346364A3749374805F099FB04463E
:1013600050B94FF4007301461A46344801F03AF878
:101370000146204601F048F90DF50A7D70BD0321B4
:101380002E48FFF7F6FE041E04DA07212B48FFF76C
:10139000F0FE0446002C1ADD03A9284805F099FC4C
:1013A000049BB3F5002F0FD04FF4007200210AA860
:1013B000FFF7F6FA4FF480654FF400720AA9204651
:1013C00005F037FD013DF7D12046FFF76BFD002109
:1013D0004FF480534FF40072184801F003F80146AF
:1013E0000028C9D00026002001F00EF900963346EF
:1013F000134A1449144805F04BFBB042BCDA134DB4
:101400000FCD0AAC0FC495E80F0084E80F000AA9BD
:101410000D480BF015F800963346094A09490A4869
:1014200005F036FBA8E700BF501B0208741B02083A
:101430007D1B0208851B0208901B02089C1B0208EA
:10144000AB1B0208B01B0208BD1B0208541B02089C
:1014500070470120704701207047B1F5003F05D16A
:10146000B2FA82F14909024804F0F1B8704700BFAE
:1014700004080400704700BF0020704770B506469E
:101480004FF4EC7003F03CFE054690B1B06006F0FE
:101490005DFF041E06DA2846FFF750FC0023B36008
:1014A000204670BD01220021A81C03F045FB00244A
:1014B000F6E76FF00B04F3E7836801225A7000200F
:1014C0007047000038B5044680682830FFF71AFDE1
:1014D00003210B48FFF74DFE051E0BD1012105F03E
:1014E0002DF92846022105F029F92046BDE83840AB
:1014F00000F008B801DDFFF7D5FC6FF0160038BD2D
:10150000CC1B020810B50446806803F0BCFA2246E2
:101510000121002005F03AF922460621012005F0BC
:1015200035F922460621022005F030F9002010BDD1
:1015300013B50024FFF7E6FE0094084B08484FF46B
:101540008052642100F03CFAA04204DC40F20D110C
:10155000044804F0ABFE204602B010BD9D01000817
:10156000D91B0208DE1B020813B500240094084BA7
:1015700008484FF40062F02100F02DFAA04204DC8C
:101580004FF4B471044804F091FE204602B010BD3F
:1015900031150108F01B0208DE1B0208024B1B6814
:1015A000986800B128307047E422002030B10388E9
:1015B0001B0401D401230380002070476FF0150045
:1015C000704710B5FFF7F2FF041E05DAFEF7FEFDC7
:1015D000644204604FF0FF34204610BD10B530B3B4
:1015E000EFF31184102383F31188038847F6FF7209
:1015F0001BB2934203D179210E4804F057FE0388B1
:1016000001331BB2038003881BB2002B0ADC0A4B98
:101610001B683BB15A6B9042FAD100225A631846BC
:1016200005F002F8E4B284F31188002010BD6FF0D9
:10163000150010BDFB1B0208DC22002010B5FFF7CF
:10164000CDFF041E05DAFEF7C1FD644204604FF0D1
:10165000FF34204610BD00BF70B5174B1C68EFF378
:101660001185102383F3118818B303881BB2002B54
:1016700009DD0388013B1BB2038000206063EDB2EB
:1016800085F3118870BD626B1AB183210B4804F099
:101690000DFE0388013B1BB20380E66E6063E266C9
:1016A0002046052104F0D0FEE06E00B14042E6661F
:1016B000E5E76FF01500E2E7E4220020101C0208C5
:1016C00010B5FFF7C9FF041E06DAFEF77FFD64427E
:1016D00004604FF0FF3010BD002010BD2DE9F7432E
:1016E0000F460646002834D042681B4B9A4230D839
:1016F000EFF31185102383F31188DFF860806846CB
:10170000D8F8009003F04BFA32460021684600F00A
:1017100069F810F10B0F0446EDB206D185F311887C
:101720000024204603B0BDE8F0837FB101A9304614
:1017300006F0CEFDD8F800300198A3EB09038342F0
:1017400034BFC01A0020394606F0B2FD85F3118877
:10175000E7E76FF01504E4E7FFC99A3B1025002086
:101760007FB51E46CB07144624D5EFF31185102311
:1017700083F3118802A906F0FFFC0028EDB206DA17
:1017800085F311884FF0FF34204604B070BD6A46DF
:1017900002A9204606F0BCFD31466846FFF79EFFD1
:1017A000044685F31188002CEEDAFEF70FFD644243
:1017B0000460E7E731461046FFF790FF0446F2E782
:1017C0008B7E062B0DD1FF2381F85030022381F848
:1017D0005130742381F8523000234B65084604F0E1
:1017E00023BF70472DE9F04F3F4B85B080460F4631
:1017F00091461C6806F0CCFEEFF31186102383F3AC
:1018000011882046D8F8005007F002F805400395EB
:10181000F6B2CDB103A806F0EBFF0146204607F073
:1018200085F8044627B1011D08223846FFF795F8D0
:101830002046257907F056F886F3118806F076FFE2
:10184000284605B0BDE8F08FD8F80030E363B9F161
:10185000000F39D099E8000C00F0D4F9814660629D
:10186000E8B11FA1D1E90001DFF888E01F4A10EBC1
:101870000B0041EBEB71EEFB0A0100230BF0FCFEC9
:1018800001231B4A00940146484600F039FA06211C
:10189000204604F0D9FD606A00F0E0F9656294F832
:1018A000501000231F29E36313D8404603F07BF94F
:1018B00090B194F85050002FBED0082204F150018E
:1018C0003846FFF74AF8B7E70621204604F0BCFD8A
:1018D000E5E76FF00A05EEE76FF00305EBE700BF01
:1018E0007F96980000000000E42200208096980077
:1018F000C117010800CA9A3B10B5FFF773FF041E19
:1019000005DAFEF763FC644204604FF0FF342046C2
:1019100010BD00BF2DE9F34104464FF4AC700E46F4
:101920001746984603F0ECFB0546002841D03146A7
:10193000FFF7A4FD00280ADA44423146284606F0A3
:1019400083FEFEF743FC04604FF0FF302EE0284694
:1019500006F038FD0028EFDB32464146284604F009
:10196000C1FD0028E8DB0096089B134A394628464B
:1019700000F070F80028DFDB099A2146284600F0C5
:10198000CBF82846FFF798FD0028D5DB2846B5F9A7
:101990000C4007F02FF8002807DAFEF717FC07497C
:1019A0000468284602F0A0FBC7E7204602B0BDE865
:1019B000F0810C24C5E700BFD91B0108F8220020E4
:1019C00013B5049C8DE8180013460A460021FFF762
:1019D000A1FF02B010BD13B5049C8DE8180013469A
:1019E0000A460221FFF796FF02B010BD024B1868AD
:1019F00008B1B0F90C007047E4220020F8B50646A3
:101A000006F0C6FD1148124A102101270388013350
:101A10001BB2002B0380D8BF012303F00F05D8BFF2
:101A2000078052F835404CB942F8356002EBC502E8
:101A30009380B38106F07AFE2046F8BD0139E5D1E6
:101A400006F074FE4FF0FF30F8BD00BF9023002079
:101A5000082300202DE9F04104460E4690461F461B
:101A6000FFF7CCFF054610BBA38BC4F8108023F012
:101A700003029DF81830676103F003031343F1B2CA
:101A8000A38304F13802217661760146032006F033
:101A9000E9FE2046A576FFF7DDF906F079FD054958
:101AA0002046FEF79DFC0423A37606F03FFE284661
:101AB000BDE8F081F82200202DE9F04104460E46F1
:101AC00090461F46FFF79AFF0546F8B9A38BC4F866
:101AD000108023F0030343F00103F1B2A38304F168
:101AE00038022176617667610146032006F0BAFE6E
:101AF0002046A576FFF7AEF906F04AFD05492046D7
:101B0000FEF76EFC0423A37606F010FE2846BDE81F
:101B1000F08100BFF82200202DE9F74F80462D48C4
:101B20001646FFF7A9F8451C26BBB14609F1020489
:101B3000A4006119404604F040FD0746002846D045
:101B4000044404602348FFF797F8054621492046DE
:101B5000013502F07FFF25443B46043E4FF0000A6A
:101B6000D1451ED1002044F8040CC8F8547103B0CC
:101B7000BDE8F08F4FF0000940F2011456F829003B
:101B80000028D3D0FFF778F8D8F828300130054482
:101B90009D4219D209F10109A145EFD16FF006006C
:101BA000E5E743F8045F70680193FFF765F8834643
:101BB00056F8041F28460BF1010B02F04BFF5D4461
:101BC0000AF1010A019BCBE76FF05A00CFE76FF0F3
:101BD0000B00CCE7251C020810B5094B1B68D3F895
:101BE0005411012040F2011451F8202012B95B6910
:101BF000984703E00130A042F6D1012006F0D4FB63
